:1000000000800020BD0100008DD5000045D5000016
:1000100045D5000045D5000045D5000045D5000078
:1000200045D5000045D5000045D500008DD5000020
:100030008DD5000045D500000DCC000011CD00008D
:100040008DD500008DD500008DD500008DD5000028
:100050008DD500008DD500008DD500008DD5000018
:100060008DD500008DD500008DD500008DD5000008
:100070008DD500008DD500008DD500008DD50000F8
:100080008DD500008DD500008DD500008DD50000E8
:100090008DD500008DD500008DD500008DD50000D8
:1000A00049B1000055B100008DD500008DD500008C
:1000B0008DD500008DD500008DD500008DD50000B8
:1000C0008DD500008DD500008DD500008DD50000A8
:1000D0008DD500008DD500008DD500008DD5000098
:1000E0008DD500008DD500008DD500008DD5000088
:1000F0008DD50000F9F500008DD5000025F7000032
:100100008DD5000065DF00008DD500008DD5000085
:100110008DD500008DD500008DD500008DD5000057
:100120008DD500008DD500008DD500008DD5000047
:100130008DD500008DD500008DD500008DD5000037
:100140008DD500008DD500008DD500008DD5000027
:10015000FDCD000011CE000025CE000039CE0000FC
:100160008DD5000081E200008DD500008DD5000006
:100170008DD500008DD500008DD500008DD50000F7
:100180008DD500008DD500008DD500008DD50000E7
:100190008DD500008DD500008DD500008DD50000D7
:1001A0008DD500008DD500008DD500008DD50000C7
:1001B0008DD500008DD500008DD50000564B4CF23A
:1001C000205210B51A804DF628121A8000BF00BFC9
:1001D0000DF0E0F9514B4FF010621A60504A9A60EE
:1001E000504ADA60504A136813F4807304D14F49BF
:1001F0000B604FF4A85313604D4B1A78110703D5C9
:100200001A7842F008021A704A4B4B492A221A7097
:100210004A4A4B4B8B4204D252F8040F43F8040B6A
:10022000F8E7484B484900228B4202D243F8042B9E
:10023000FAE74649464A002352F8230041F82300D2
:1002400001336F2BF8D1434B434A802103F8011B44
:100250009342FBD1414B3D4A1A60414B8A221A70AE
:10026000A3F5805324225A70A0221A709A7992071B
:10027000FCD59A79D406FCD43A4A937903F00C035E
:10028000082B384BF9D103221A7140225A719A79FE
:100290009006FCD5334A9179324B4906FBD5324A58
:1002A000324911600221516020221A709A7902F0BD
:1002B0000C020C2AFAD12E4B2E4A1A602E4B2F4AD2
:1002C0001A6000225A60072243F8042C2C4AC3F813
:1002D0000C2D62B60DF00EFD144B1B68DA0705D528
:1002E00028480DF0DBFA284B284A1A60284B1B7867
:1002F0005B0609D5244C254B22689A4204D121483B
:100300000DF0CCFA0023236010F0C6FC0DF048F984
:100310000DF076F8FEE700BF0E2005403080044067
:10032000823F04000100002B10D0034014D0034092
:1003300002D0074000E00740EC9BFF1FC4450100CE
:100340004088FF1FEC9BFF1F10A4FF1F0082FF1FB0
:100350000000000000E400E05FE400E008ED00E0E1
:100360000050064000400640448004400000030165
:1003700004800440C010050014E000E0FF76010096
:1003800000002020DD763F5F1CE00340A5C3945AA7
:1003900000F00740FFFFFFFFFFFFFFFFFFFFFFFF32
:1003A000FFFFFFFFFFFFFFFFFFFFFFFFFFFFFFFF5D
:1003B000FFFFFFFFFFFFFFFFFFFFFFFFFFFFFFFF4D
:1003C000FFFFFFFFFFFFFFFFFFFFFFFFFFFFFFFF3D
:1003D000FFFFFFFFFFFFFFFFFFFFFFFFFFFFFFFF2D
:1003E000FFFFFFFFFFFFFFFFFFFFFFFFFFFFFFFF1D
:1003F000FFFFFFFFFFFFFFFFFFFFFFFFFFFFFFFF0D
:10040000FFFFFFFFFFFFFFFFFFFFFFFFDEF9FFFF23
:1004100010B5054C237833B9044B13B10448AFF33E
:1004200000800123237010BDEC9BFF1F0000000023
:10043000C8450100084B10B51BB108490848AFF387
:1004400000800848036803B910BD074B002BFBD0A0
:10045000BDE81040184700BF00000000F09BFF1FE0
:10046000C8450100EC9BFF1F0000000038B50446A2
:10047000104621700A491D4610F0F0F901464FF070
:100480007E5010F09FFA074910F0E8F9E5606060CF
:10049000256165610DF0BEFBE061204638BD00BFFF
:1004A000DB0FC9400024744938B50446104621705A
:1004B00009491D4610F0D2F901464FF07E5010F068
:1004C00081FA064910F0CAF9E5606060256165614E
:1004D0000DF0A0FBE06138BDDB0FC940002474497A
:1004E00038B503780446032B20D8DFE803F01A1848
:1004F0001002C168406910F0A7F80D490546606810
:1005000010F060FA0146284610F05CFA38BD084940
:10051000406810F057FAE16810F0A0F938BDC068E3
:1005200038BDC168406910F08FF838BD002038BD73
:100530000024744970B504460E460DF06BFB054669
:10054000E069281A10F036F9E3682361E561666115
:10055000A0610146606810F035FA0146A0601048BD
:1005600010F030FA0FF006FD0FF0A6F910F018F8B1
:10057000054601464FF07E5010F066F8616910F0B4
:100580006DF921690646284610F068F901463046A3
:1005900010F05CF8E0602046BDE87040FFF7A0BFB7
:1005A000000080BF38B50E201C4C0CF003FE2188E3
:1005B0001B4B884205461A881DDA0023511AB1F5F3
:1005C000805FAABF1B03C3EB03330131142093FBED
:1005D000F1F10DF075F9134B1988F1B923889D429B
:1005E00010DAC3F57F630F33282091FBF3F1BDE8E8
:1005F00038400DF065B99042D4BFC1EB0003C1EBA8
:100600000203DBE740F6FF718D42D4BFC3EB050167
:10061000C3EB0101C1EB0131E3E738BDE09CFF1FF3
:10062000A29EFF1F509EFF1F10B504460CF0C4FB96
:10063000204610BD70B44C88A04220D9012301335C
:10064000DBB21CB2660031F8144084421D46F6D37A
:10065000A04211D005F10045013D965B31F815101F
:1006600032F81530401AF21A00FB02F0641A90FBBF
:10067000F4F4E01870BC7047905B70BC70470226C1
:100680000125E5E700280CDA064A434282FB0320F5
:10069000DA17C2EB600000EB4000A3EB8000C0F172
:1006A0000C007047ABAAAA2AF0B40E8886420DD27D
:1006B00003F10043013B31F81350854202D9F0BCED
:1006C000FFF7B8BF32F81300F0BC70471088F0BCD9
:1006D000704700BF094B1B880C2B09D8084A80B211
:1006E00052F8232028B143F6FE73984203D9108CA8
:1006F0007047108870470349FFF79CBF429CFF1F5B
:1007000010200100AC2101004B4B4C4A2DE9F04771
:100710001E8814684A4BB442B3F80080494B33DB5F
:100720004445A8BF4446A6421C60C8BF00202DDD3A
:10073000C6EB0807B7F5804F33DB80037B1C90FBCB
:10074000F3F0FFF7C7FF404A404B15881B88C0F302
:10075000C61909FB05F57F2D8246A8BF7F252BB35F
:10076000A64253DC4445D4BFC6EB0404C6EB0804E0
:100770009F42CCBF03FB04445C43354BC8BF0137E9
:1007800094FBF7F71F6013E034461E60C6EB0807C2
:10079000A045D4BFC6EB0800C6EB0400B7F5804FF8
:1007A000CBDAC0EB803090FBF7F0CAE7284A136041
:1007B000284C2368994508D0274B1B88002B34D13F
:1007C000264B1B886BBBC4F80090254C23689A45C8
:1007D00006D0214B1B885A1F032A19D9C4F800A040
:1007E000204C23689D420FD01F4B188848B11A4BEC
:1007F0001E4A1B88D35C834203D0C0B2E9B208F022
:10080000E1FD2560BDE8F087BDE8F0870024AFE793
:10081000164AD05C2030C0B20AF07F0108F0D2FD49
:10082000DCE7484608F042FECDE7104A4946D05C76
:1008300008F0C8FDC4E700BFE09CFF1F4C9EFF1FEF
:10084000A29EFF1F109CFF1F249CFF1F269CFF1FC2
:10085000A89EFF1F849CFF1F349EFF1FD29CFF1F7A
:100860003C9CFF1FD49CFF1F429EFF1F048AFF1F5A
:100870002DE9F04F012089B00DF0E0FBAF4B18607F
:1008800000200DF0DBFBAE4BAE4A1B8810600C2B3A
:1008900000F03B81AC4BAD4A19880093AC4B52F849
:1008A000214000221A70AB4BAB4D1B88AB4A2E88FF
:1008B000013B32F91370002E5CD0A94BA94A1B886A
:1008C000A9491278013B31F91380002A40F0DF80FA
:1008D00011200DF0B3FBA54B0193D3F800A0064601
:1008E000B24540F3DF80A24BDFF8A4921B88A14AF7
:1008F000012BD9F80030B2F800B09F4A029220468E
:10090000C8EB030800F09A820FF054FF029A52F8E5
:100910002B100FF0A3FF014600200FF095FE10F002
:1009200063F9CAEB0802B045B8BFB0469042CAEBC3
:10093000080880F2968200FB0888013298FBF2F0EA
:100940008E4BDFF850820293D8F80030034403EB5B
:10095000D3735B10C8F800302B88012B12D1884B61
:10096000DFF834B20393874BDBF8005004934FF069
:10097000000A47E07D4B0193DFF814927F4BDFF8CC
:10098000148202937E4B03931D460F200DF056FBFD
:100990002B689842824641DA754A1288012A00F093
:1009A0001D82744A05931288734D049220460FF0FD
:1009B00001FF049ADFF8E0B155F82210DBF800508F
:1009C0000FF04CFF014600200FF03EFE10F00CF936
:1009D000EF1B059B5745A7EB0302B8BF5746FF1A0D
:1009E0009042BABF013200FB0777474397FBF2F70B
:1009F000D8F80020634B0493BB1803EBD3735B1050
:100A0000C8F80030604B1B88013B032B00F2B0821A
:100A1000DFE813F06301A901C4008601594B049378
:100A20001B68984240F3C281514A1288012A00F0A3
:100A3000A682504A079311884F4A06912046059294
:100A40000FF0B8FE059A0699DFF84CB152F8211064
:100A5000DBF800500FF002FF10F0C6F8079B2F44A0
:100A60005745A7EB0302A8BF5746FF1AD8F8003036
:100A70009042BABF00FB07770132474397FBF2F77A
:100A80003B4403EBD3735B10C8F80030BAE7152082
:100A90000CF090FB354B0193D3F800A00646B2450D
:100AA0003FF721AF354B0293D3F800A0B24580F257
:100AB00089812F4BDFF8D8901B882E4A012BD9F85B
:100AC0000030B2F800B02C4A03922046984400F05F
:100AD00070820FF06FFE039A52F82B100FF0BEFEDB
:100AE00010F082F8B045CAEB0802A8BFB046CAEBC6
:100AF00008089042B6BF00FB088800FB08F80132E6
:100B000098FBF2F0DFF88C801EE7204B1B78002B5F
:100B10003FF4C0AE0C4B0D4A198800930C4B52F8B1
:100B2000210001221A700FF045FE4FF07C510FF0AA
:100B300095FE10F059F80446B5E600BF749CFF1FFF
:100B40007A9EFF1FC89EFF1F7A9CFF1F8489FF1F8C
:100B50001A9CFF1F108AFF1FEC9DFF1F102501002C
:100B6000608AFF1F009EFF1F642101006C9CFF1F15
:100B7000BE9CFF1F609CFF1F28250100AC9CFF1F2F
:100B80006C9EFF1FE09DFF1F5A89FF1F309CFF1FB7
:100B9000089CFF1F849EFF1F689EFF1F28460FF0C2
:100BA00009FEB2490FF05AFE054650460FF002FE0C
:100BB000AF490FF053FE014628460FF047FD10F0F5
:100BC00013F80546CBF80050D9F800000FF0F2FDFD
:100BD000A6490FF043FE074630460FF0EBFDA4494F
:100BE0000FF03CFE014638460FF030FD0FF0FCFFE1
:100BF000C9F800009F4AA04B168819889F4AA04B4D
:100C000012681B889F4FC6EB050E3544039EC6F83D
:100C100000E0461A084404990D6001990E6002999B
:100C20003E8808609A4280F289810025C3EB060E57
:100C3000954974450F6880F27681611C9F4205FBDF
:100C400001F50EF1010E95FBFEF5C0F2BE81BE422C
:100C5000A8BF3E46F61A01FB06F494FBFEF49A4246
:100C600000F33681BB42C0F23381884C20680FF01C
:100C7000A1FD87490FF0F2FD86490FF0E7FC0FF068
:100C8000B3FFA0F5FF531C3B082B98BF4FF4005057
:100C9000D8F80030184400282060C0F24281B0F536
:100CA000804F80F252817C4B1B781BB1B0F5005F06
:100CB00040F05381794D2B78002B40F05481784DD2
:100CC00020682B68714C984204D080B208F058FC20
:100CD00023682B6009B0BDE8F08F28460FF06AFD4D
:100CE00070490FF0BBFD054650460FF063FD6E499D
:100CF0000FF0B4FD014628460FF0A8FC0FF074FF7A
:100D00000546CBF80050D9F800000FF053FD6549B7
:100D10000FF0A4FD074630460FF04CFD62495FE737
:100D200028460FF047FD5A490FF098FD05465046FA
:100D30000FF040FD5D490FF091FD014628460FF090
:100D400085FC0FF051FF0546CBF80050D9F80000A4
:100D50000FF030FD4E490FF081FD074630460FF091
:100D600029FD52493CE728460FF024FD50490FF079
:100D700075FD054650460FF01DFD4E490FF06EFD06
:100D8000014628460FF062FC0FF02EFF0546CBF817
:100D90000050D9F800000FF00DFD45490FF05EFD41
:100DA000074630460FF006FD424919E7D8F80030F3
:100DB000DFF810B103EBD3735B10DBF80050C8F819
:100DC00000301FE6DFF80081DFF80091D8F800302E
:100DD00003EBD3735B10C8F80030BDE5364A0693C9
:100DE0001188364A059120460492DFF8D8B00FF0FA
:100DF000E1FC049A0599DBF8005052F821100FF03D
:100E00002DFD0FF0F1FEEF1B069B5745A7EB0302EC
:100E1000B8BF5746FF1AD8F800309042BABF013227
:100E200000FB0777474397FBF2F73B4403EBD37391
:100E3000234A04925B10C8F80030E3E50FF0BAFCD7
:100E4000029A52F82B100FF009FD0FF0CDFECAEBFD
:100E50000802B045B8BFB0468242CAEB08083FF767
:100E60006AAD00FB08F898FBF2F069E5CDCC4C3F89
:100E7000CDCC4C3E128AFF1F5889FF1F749CFF1F68
:100E8000489EFF1F589CFF1FC89EFF1FB889FF1F69
:100E90009A99193FCDCC4C457E9FFF1FD09CFF1FD8
:100EA0002089FF1F3333733FCDCC4C3DCDCCCC3E9E
:100EB0006666663FCDCCCC3D609CFF1F28250100B7
:100EC000E09DFF1F689EFF1F849EFF1F089CFF1F61
:100ED000009B1B88002B3FF4C8AE2B1B002BB8BF18
:100EE0005B42092B47DD05F500500130001B0FF078
:100EF00061FC3B493B4C0FF0B1FC054620680FF00C
:100F000059FC39490FF0AAFC014628460FF09EFB18
:100F10000FF06AFED8F80030184400282060BFF6B1
:100F2000BEAE002213E09F4205FB04F5B8BF0021CE
:100F300095FBFEF54BDA91FBFEF490E6B242D4BF8E
:100F4000C3EB0205C3EB060570E643F6FF72274BC1
:100F500022601B78002B3FF4ADAE05F0B3FC244BB0
:100F600001221A70ABE605F0A9FC00232B70A6E65F
:100F7000D9F800003EE64FF400501A4C88E61D49AF
:100F80001D4A069320460D8805920FF013FC059A22
:100F9000DFF868B052F82510DBF800500FF05EFC67
:100FA000014600200FF050FB0FF01EFE2F44069B61
:100FB00056E50FF0FFFB039A52F82B100FF04EFC92
:100FC000014600200FF040FB8AE51E4642E6B7428C
:100FD000D4BFC3EB0701C3EB060104FB01F1AAE791
:100FE000CDCCCC3EB889FF1F9A99193F7E9FFF1F39
:100FF000D09CFF1F609CFF1F28250100689EFF1FDB
:1010000008B5244B1B88FBB1234B1B78FBB1234B4A
:101010001B78E3B1224B1B78CBB1224B1B78B3B1C9
:10102000214B22481A78C2B9214A224900881288E5
:1010300009680244B1EB620F09DD01221A706420D5
:10104000BDE8084005F052BC174A117801B908BD47
:101050001370BDE8084008F05DBA154A16490088CB
:10106000128809680244B1EB620FF0DD00221A70A9
:1010700008F050FA642005F039FC642005F036FCD5
:10108000642005F033FC4FF41670BDE808400CF006
:10109000E3BD00BFEE9DFF1F9E9EFF1F9F9EFF1F93
:1010A000A09EFF1FA19EFF1F409CFF1F589CFF1F7B
:1010B000489EFF1F749CFF1FC89EFF1F38B5114C30
:1010C000232025780CF076F80F4A42F82500131FEC
:1010D00002F1C400002253F8041F83420A44FAD1EB
:1010E00023780A4907480A4C0133DBB2322B81FBD3
:1010F000025108BF0023D217C2EB211203702260F5
:1011000038BD00BF289CFF1FF09CFF1F1F85EB51BF
:10111000449EFF1F2DE9F04FB84CB94D2068B94FE0
:1011200083B00FF047FBB8490FF098FB064610203C
:101130000CF084FF0FF03EFBB4490FF08FFB3146FB
:101140000FF084FA0FF050FD2988206088423B8818
:1011500043DA9E465B1A7F2B4FF0000247DDD20137
:101160005E1C92FBF6F2AA4EDFF8C882B6F800C009
:10117000C8F80020BCF1190F00F0DF80BCF11A0F95
:1011800000F01781BCF11E0F00F020810126B1464E
:10119000A04A1288002A00F09D808842C0F2078190
:1011A0007045D4BFC1EB0000C1EB0E009A42BABF3C
:1011B00002FB00000133504390FBF3F3964A1360A7
:1011C000964B1888C0B9964A1288AAB9954B1978D7
:1011D00001B11A7003B0BDE8F08F9842D4BFC1EBE3
:1011E0000002C1EB03029E465B1A7F2BB7DCC2EB09
:1011F000C21292FBF3F2B6E72988D4F800E0DFF8D8
:101200000082DFF8F8A171456CDCDFF818C29CF8A9
:101210000020002A2ED14FF0010B04288CF800B0DA
:1012200028D1002E40F094817D4B18880028D1D021
:10123000B9F1000FCED023682C883A88A34280F2FF
:1012400065810023141B7E2C774DD5BFC3EB831320
:10125000C3EBC3135B00013493FBF4F42B6801343C
:10126000A34203D0C0B2E1B208F0ACF82C6003B0E6
:10127000BDE8F08F012800F0F680022800F0EB8036
:101280000328D1D1694B1B88092BCDD0002ECBD0A0
:1012900023682E883A88B34280F27B810023961B14
:1012A0007E2EDFF88CA1D5BFC3EB8313C3EBC31332
:1012B0005B00013693FBF6F6DAF800300136B342F4
:1012C00003D0F1B24A2008F07DF8CAF80060ABE71D
:1012D00016469146BCF11E0F7FF472AF0022DFF874
:1012E00058817EE04F4B1A78002A3FF473AF0024F8
:1012F00001281C7000F0A480022840F00E81002E0E
:1013000000F0A3804A4D2B68002B00F09E80042043
:10131000214608F057F8424B2C60188800283FF40B
:1013200059AFB9F1000F3FF455AFC0B2002108F03A
:1013300049F83D4B00221A604CE7DFF8FC8098F832
:101340000020C2B1DFF8D890B9F800A0BAF1000FC0
:1013500011D0DFF8E89099F800B0934578D05FFAA3
:101360008AF07F2108F02EF898F80030B6F800C017
:1013700089F8003010E0DFF8C49099F800A0924599
:1013800066D0274B0021187808F01CF898F8003038
:10139000B6F800C089F800301E4B1A88002A97D092
:1013A000BCF11E0F40F006810026B14619E0002076
:1013B000FCE6DFF8848098F80020002A0BBF0126A5
:1013C00000264FF000094FF00109E1E6DFF86880E0
:1013D000104B98F800601A88B6FA86F676094FF036
:1013E000000998F80030002B3FF4E8AE2988B7F8E0
:1013F00000E02068C1EB0E03CFE600BF689CFF1F32
:10140000F49DFF1FF09DFF1F9A99193FCDCCCC3E54
:101410007A9EFF1FAC9EFF1FE89CFF1F729CFF1F60
:101420008A9EFF1F7F9EFF1F4C9CFF1F349EFF1F45
:10143000EC9CFF1F609EFF1F309CFF1F2C9CFF1F1A
:101440001EB1614D2B68002B7BD1604B188865E77E
:101450000026B1469CE6002E3FF4E6AEDFF868A118
:10146000DAF800202EE0002E3FF4DEAEB7F8008060
:10147000F045D4BFC1EB0802C1EB0E02C1EB080876
:10148000B8F17E0FDFF840A1D5BFC2EB8212C2EBEC
:10149000C212520008F1010892FBF8F8DAF80020B5
:1014A00008F10108424506D05FFA88F10120009357
:1014B00007F088FF009B1888CAF8008002287FF494
:1014C000DFAE42462168B5F800803888414559DAD8
:1014D0000021C8EB0008B8F17E0FD3BFC1EB81112A
:1014E000C1EBC11108F10108490091FBF8F808F1BE
:1014F0000108904506D05FFA88F10420009307F0B8
:1015000061FF009B1888CAF80080B9E69342D4BFF7
:10151000C4EB0303C4EB020394E6032827D12C4B4E
:101520001B88092B91D0002E8FD0274D2B68002BC4
:101530008BD04A20214607F045FF244B2C601888A9
:10154000ECE6214607F03EFF204B2C601888E5E6CC
:1015500040207F218DE80C0007F034FF019B009AAA
:10156000188858451CD002287FF48AAE76E70428F4
:101570007FF46BAF002E3FF468AF2146402007F0A8
:1015800021FF62E78142D4BFC8EB0101C8EB000133
:101590009FE79342D4BFC6EB0303C6EB02037EE68C
:1015A000B8F80010DAF800E0B7F800808E45FFF6D2
:1015B00065AF5DE72988B7F800E020680026C1EB39
:1015C0000E03B146E9E500BFEC9CFF1F8A9EFF1F9A
:1015D000349EFF1F08B5114B1B88022B09D0052B29
:1015E00007D0032B15D0042B0BD00D4B01221A7002
:1015F00008BD7F21412007F0E5FE094B01221A704A
:1016000008BD7F21092007F0DDFE054B01221A707D
:1016100008BD4021092007F0D5FEE6E7E69CFF1F44
:10162000969CFF1F38B5244B1B881D2B40D0234BA5
:101630001B88012B25D0224A224B14881B68224A82
:10164000A342128828DB214909889342D4BFC4EB06
:101650000303C4EB0203121B914224DA01FB0333A0
:10166000541C93FBF4F41A4B1A4D1B88052B06D01F
:101670002B689C4203D0E1B2052007F0A3FE2C604A
:1016800038BD154B154A1B681488154AC3F53B63D2
:101690000833A3421288D6DA0C490988121B9142FA
:1016A0004FF00003DADB03FB01F393FBF2F4DAE71C
:1016B000064B1C88D7E700BF7A9EFF1FEC9DFF1FDB
:1016C000929CFF1F1C9CFF1F789EFF1F809EFF1F88
:1016D000E69CFF1F149CFF1FF89DFF1FE49CFF1F4B
:1016E000649EFF1F38B5124D124C2B88052B12D06B
:1016F00022684AB9022B0ED0033B012B13D90E4AA4
:1017000000231370236038BD0021052007F05AFE26
:101710002B88022B04D10021412007F053FEEEE775
:10172000052BE9D1F7E70021092007F04BFEE6E79A
:10173000E69CFF1F149CFF1F969CFF1F08B5284BBB
:101740001B78ABB115200BF035FD264A264B1288CD
:1017500018601D2A15D0254A1288DAB1012A2BD02B
:10176000234B1B78002B3AD0BDE80840FFF7BABFE7
:1017700011200CF063FC1B4A1B4B128818601D2AB9
:10178000E9D11C4B1B88002BEAD01B4B1B78002B8C
:10179000E6D008E0174A1288002AE1D0174A1B68F1
:1017A00012889A42DCDC124B1B780BB9FFF712FF50
:1017B000BDE80840FFF736BF0F200CF03FFC0D4B93
:1017C0000F4A1B88106033B10E4BC0F53B601B887D
:1017D00008309842E7DA064B1B78002BC4D108BDCD
:1017E000009EFF1F7A9EFF1F1C9CFF1FEC9DFF1F8A
:1017F000969CFF1FE69CFF1F309CFF1F929CFF1FC3
:10180000F89DFF1FE49CFF1FF8B510200CF016FC9C
:10181000C830B0F5FA7FC0F29680B0F57A6F014615
:10182000A8BF4FF47A6101F51673B3F57A6FA8BFBC
:101830004FF47A639BB289B2914A924C1180222074
:10184000238007F043FF21888F4D904C242007F020
:101850003DFF0E200BF0AEFC40F6FF71C830884211
:10186000A8BF084620EAE07000F5FA6283B28A4217
:10187000A8BF0A460220194622802B8007F026FFC7
:101880002188042007F022FF01200CF0D7FB04463A
:1018900000200CF0D3FBA042B8BF204600F1C801E5
:1018A000B1F5FA7FC0F2D180B1F57A6FA8BF4FF4DD
:1018B0007A6101F54873B3F57A6FA8BF4FF47A6384
:1018C0009BB289B2724A734C11800A20238007F0C0
:1018D000FDFE21880C2007F0F9FE0F200CF0AEFB76
:1018E000C0F53F610431B1F5AF6FC0F2AB80B1F527
:1018F000FA6FA8BF4FF4FA6189B2674BC0F5436035
:10190000B0F5AF6F1980C0F29A80B0F5FA6FA8BF3A
:101910004FF4FA6083B2614CA420238007F0D6FE16
:101920002188A62007F0D2FE15200BF043FC00F51D
:101930009671B1F52F7F0BDB41F25C23994240F3A6
:101940008980194608E040F24C434FF4FA7173E77E
:1019500040F214534FF42F71514A1180514C524DA3
:101960002380062007F0B2FE2188504E082007F0A1
:10197000ADFE00274FF4AF74F9B24D4809F058FCA2
:1019800055F8043BC3F5967300FB03F086FB002378
:10199000C017C0EB6310844207F10107A8BF0446DB
:1019A000062FE9D1434F414E0025E9B2424809F0E4
:1019B0003FFC57F8043BC3F5967300FB03F086FB2E
:1019C0000023C017C0EB6310844205F10105A8BFD6
:1019D00004460C2DE9D1394F344E0025E9B2384880
:1019E00009F026FC57F8043B304AC3F5967300FB18
:1019F00003F086FB0013C017C0EB6310844205F1AF
:101A00000105A8BF04460C2DE8D1A4F11401312929
:101A100031DD40F23A73A4F5B97403FB04F482FBA0
:101A20000432E417A4EB621289B232322548264B05
:101A300001801A602A20BDE8F84007F047BE4FF445
:101A4000AF6368E74FF4AF6157E740F214534FF4C8
:101A5000FA7137E7124A00F5617089B2B0F52F7F4D
:101A60001180B8BF4FF42F73FFF678AF8342A8BF41
:101A700003469BB272E740F26C723221D6E700BF98
:101A8000F49DFF1FF09DFF1FE09CFF1FA29EFF1F04
:101A9000489EFF1F589CFF1FE49CFF1F649EFF1F72
:101AA000929CFF1F789EFF1F488AFF1FB5814E1B27
:101AB000449CFF1F188AFF1F789CFF1F2889FF1F67
:101AC000D89CFF1F9C9EFF1F008AFF1F2DE9F84F27
:101AD0000C200BF03BFB0C200BF0F0FFBF49142057
:101AE0000BF0FCFFBE49BF4809F034F80221032087
:101AF0000CF08AF8022104200CF086F8022105205F
:101B00000CF082F8022106200CF07EF801210A2058
:101B10000CF07AF8012109200CF076F801210D2053
:101B20000CF072F8012128200CF06EF8012114202D
:101B30000CF06AF8012116200CF066F8172001213C
:101B40000CF062F804200CF051F800283DD005207C
:101B50000CF04CF8044600283ED000242046A24D4C
:101B6000287006F0CBF92E785EBB204607F0D8FD32
:101B70009E4B9F491B880F889E4ADFF8DCE29E4DF2
:101B8000A3F5AF7140F23A7303FB01F382FB03123A
:101B9000DB17A3EB6213323301210D20CEF80030A6
:101BA0002F700CF01DF864200CF056F84FF41671ED
:101BB0000A200BF085FE5D21904809F075FB90B975
:101BC000FEE7BDE8F84F08F0D5BE06200CF00EF891
:101BD0000028BCD10124C2E703200CF007F8B0FABA
:101BE00080F04009BBE764200CF036F831460A204B
:101BF0000BF066FE4FF4967109200BF061FE5C213C
:101C00007F4809F051FB00B9FEE764200CF024F88E
:101C1000314609200BF054FE4FF4967116200BF05C
:101C20004FFE5B21774809F03FFB00B9FEE76420D7
:101C30000CF012F8314616200BF042FE4FF496716C
:101C400017200BF03DFE64200CF006F831461720FB
:101C50000BF036FE64200BF0FFFF31460D200BF039
:101C6000BFFF694A69481268DFF8F0B1DFF8A4A144
:101C7000674FDFF8EC91DFF8EC8100230121FEF7DC
:101C800013FC0123CAF800603E60C9F800608BF8BD
:101C9000003004260F200CF0D1F9D9F800300344AD
:101CA0000E20C9F800300BF085FADAF800309BF806
:101CB00000200344CAF800301520002A7DD00BF024
:101CC00079FA3B681844386006F0010080F00100A2
:101CD00004F0FCFDB8F80030002B14BF4B20DC20D2
:101CE0000BF0BAFF013ED5D1D9F80030DAF8002068
:101CF00048493868DFF870E1474E002BB8BF03331E
:101D0000002AB8BF033292100A604449444A098845
:101D100012880028B8BF03309B10801038605F1A0B
:101D200019443160CEF800703E4E3F4F3F49C9F82C
:101D30000030C2EB000E0244C7F800E032600B60D6
:101D40000CB1FFF761FDB8F800305BB94FF4FA70E1
:101D500004F0CCFD04F0B6FD06F0D8FB4FF4AF6004
:101D60000BF07AFF324B012404201C600BF03EFF85
:101D700010B9304B28701C702F4B1B881C2B23D0A4
:101D80002E4C04F1C80523200BF014FA44F8040F7C
:101D900001200BF061FFA542F5D1294A294B1078AB
:101DA000187007F0C7FB04F089FD45F6BF522649BD
:101DB0002648BDE8F84F0AF0B5BF11200CF03EF9F7
:101DC0003B68184438607FE7214B18880028D7D03B
:101DD000204BC0B2197807F0F5FAD1E7001B37465F
:101DE00040420F00F890FF1F489CFF1F9C9EFF1F62
:101DF0000C9EFF1FB5814E1BA89CFF1F449CFF1F1C
:101E0000D89CFF1F789CFF1F2489FF1F109EFF1F77
:101E1000089CFF1F209CFF1FE09DFF1F128AFF1FD1
:101E20005889FF1FAC9CFF1F6C9CFF1FB49EFF1FB7
:101E3000749EFF1F319CFF1F7A9EFF1FEC9CFF1FAB
:101E4000FC9DFF1FDB9DFF1FA5050000949EFF1F4B
:101E5000B09CFF1F649CFF1F008AFF1F009EFF1F96
:101E6000689EFF1F3E9EFF1F6C9EFF1F2DE9F04FD7
:101E7000AD4C2678012E95B000F05582C0F00B8253
:101E8000022E00F0D880A949A94A91F80080117863
:101E9000A84ADFF83CE3A84DA84FA948A94B0292F5
:101EA000A94A0092A94A9EF800B001922D78A84A4A
:101EB0003F7890F800E01B78DFF818A3DFF818C32C
:101EC000DFF818930392012E84BF00222270A14AEA
:101ED000A1481370A14A80F800B01570A048A14A2B
:101EE000077082F80080A048A04A03709CBF0136AA
:101EF00026701170BEF1000F40F074819C4A10886A
:101F00000D2800F0B9819B4C002020700246044649
:101F10002DB197480088002840F0BA8105469648C0
:101F200006882544002E40F067819448944C019E19
:101F30000078367824780130A0EB4600002C40F081
:101F40005682039C94F800E0CEEB0004BEF1000F33
:101F500040F076820026DFF874E202989EF800E0F6
:101F60000078A41BA4EB4E043C44CBEB040410B15A
:101F7000B7FA87F040099CF800602718BC1B1EB117
:101F80001EF1000618BF0126009F99F8000097F87F
:101F900000909AF800C07B4FC6EB040EC0EB0E0019
:101FA000A0EB49008044C3EB0803A3EB41010C23E1
:101FB00013FB0C113960744B744F754C75481B88BA
:101FC0000088D7F800C0744E2788744C3688D4F83F
:101FD00000E0033BC0EBC00403EB4303C7EBC700C7
:101FE00001EB830364446E4F334470446D4E57F8E5
:101FF000244056F820000C3B1D44254405440AB1FA
:10200000694B1960694A13689D4200F03181684B41
:10201000684819680791079901601B68089366482A
:10202000089B008815605B1A834284BF634B1D6068
:1020300015B0BDE8F08FDFF8A881614E08AF00252C
:10204000E9B2604809F0F4F858F8043BC3F5967318
:1020500000FB03F086FB00230135C017C0EB6310C3
:102060000C2D47F8040BEBD1574B384D0195384DEB
:10207000B3F800C00395109D09980F99404EDFF802
:10208000C0A0DFF8B490DFF8BC80654511AA8CCA07
:10209000AE46ACBF4FF0000E4FF0010E8445D4BFEA
:1020A0000020012030708C4528480B9D1F4E8AF877
:1020B00000E0D4BF00210121017094452449DFF8DC
:1020C00014A1D4BF002201220A709C453F4AD4BF0C
:1020D00000230123BC45AB46D4BF00270127137062
:1020E000AC45164B0C9D1F70D4BF4FF0000B4FF04A
:1020F000010B374B0F4A0292AC45DFF834C0124A4D
:1021000083F800B0D4BF0025012589F8005098F865
:1021100000309CF8001096F80080DFF8BCC02678EC
:10212000DFF8B8900092CEE6DA9DFF1F309EFF1FC9
:10213000329EFF1FC09CFF1FD09EFF1F949CFF1F5D
:10214000D59EFF1F319EFF1F7D9EFF1F8D9EFF1F8F
:102150008E9EFF1FCF9EFF1FF39DFF1FD19EFF1F6F
:10216000D29EFF1FD39EFF1FD49EFF1F7E9EFF1F88
:10217000D69EFF1F309CFF1F189CFF1F148AFF1F55
:10218000C09EFF1F389EFF1F549EFF1FE89CFF1F2D
:10219000989CFF1F709EFF1F2A9CFF1FA89EFF1F79
:1021A00024230100601D0100B89EFF1F8C9CFF1FAF
:1021B000BC9FFF1F7C9CFF1F889EFF1FC49EFF1FAC
:1021C000B5814E1BD89CFF1F9C9EFF1F8F9EFF1F3B
:1021D000959CFF1FE59DFF1FCE9EFF1F7C9EFF1F4E
:1021E0002889FF1FAF4AB04814880122182C0270BA
:1021F00040F2058100248BE6012E00F08F81022E33
:1022000000F0EE81032EA94B00F01F811E78009B89
:102210009CF800E01C78019B99F800C01878029B9C
:1022200093F80080039B1F78A6EB4E03A4EB840475
:10223000CCEB030CC0EB80760CEB0403C0EB860008
:10224000034403EB480303EB810327B19849097862
:10225000002940F0608201269AF800109548C1F1EB
:10226000060101EB4101334403EB81010160A2E669
:102270009149924B0968D0E6002D3FF444AE894A5B
:10228000894E14880122182C327040F2B8807446AE
:10229000A0F10D0543E6DFF87092894F0DF120089B
:1022A0000025E9B2874808F0C3FF59F8043BC3F59D
:1022B000967300FB03F087FB00230135C017C0EBCA
:1022C0006310062D48F8040BEBD17F4BDFF83CA2DE
:1022D00019880D9B00228B428AF8002080F2A28090
:1022E0007A4B8AF800507A497A4A7B4891F8008004
:1022F00011787A4A1D7002920378794ADFF810C289
:10230000DFF810920092774A774E784D784892F82D
:1023100000E0784A0192784A96F800B02D78077864
:1023200026780392CFE5DFF8F081654E08AF0025EF
:10233000E9B2724808F07CFF58F8043BC3F5967385
:1023400000FB03F086FB00230135C017C0EB6310D0
:102350000C2D47F8040BEBD15B4B0C9D1F885F4B9A
:1023600002935F4B00930B9B0A98099ADFF8A0C178
:10237000089EDFF8A0910F99BB429E46ACBF4FF07C
:10238000000E4FF0010EAF42D4BF00250125874259
:10239000109B8CF80050D4BF00200120504D89F8CC
:1023A00000009742D4BF00220122B742D4BF4FF0B1
:1023B00000084FF001082A709F42474A4448474EA0
:1023C00080F80080D4BF002301231370129A414883
:1023D00086F800E08F42D4BF0021012197420170AE
:1023E0001ADC00224648DFF824A102708BE7039C28
:1023F00046B12678002E40F06081441EABE50C3CCF
:10240000012285E594F800E00138CEEB0004BEF12E
:10241000000F7FF4A0AD9DE5119A9742D4BF002232
:102420000122DFE70C9A374B9142CCBF01220022F8
:102430001A7040F3458105258AF80050234B52E776
:10244000002E3FF487AD012685E51C78009B02989D
:1024500093F80080019B9CF800601B7890F800C006
:1024600099F800700398A4EB4604E71B90F800E08D
:10247000C3EB8374A8EB88003844C3EB84030344A4
:1024800003EB4C0303EB8103BEF1000F40F04881E6
:1024900001269AF80010074833440C2414FB01313C
:1024A000016088E57A9EFF1F309CFF1F148AFF1F82
:1024B0008F9EFF1F389EFF1F7C9CFF1FBC9FFF1F2E
:1024C000B5814E1B449CFF1F9C9EFF1FF29DFF1F6A
:1024D000309EFF1F329EFF1F319EFF1FC09CFF1FBB
:1024E0007D9EFF1FD59EFF1F959CFF1FD09EFF1F47
:1024F000949CFF1F8D9EFF1F8E9EFF1F789CFF1FC9
:102500005E9CFF1FA19EFF1F488AFF1FE59DFF1FC6
:10251000CE9EFF1F7C9EFF1F188AFF1FA34CDFF873
:102520009CE2207805909EF8004001980494059C58
:10253000007801900134A4EB40040498002840F096
:10254000AF80039890F800E00498261ACEEB0600BE
:102550000390BEF1000F40F09E8074460298944EA6
:1025600000780290039836780496041BA4EB460486
:1025700002983C44CBEB0404002800F08780B7FAB3
:1025800087F040099CF800602044871B1EB1049826
:10259000061C18BF0126009C99F800002478BE1B79
:1025A000301AA0EB440080440198C3EB0803A3EB6E
:1025B0004103002867D1BEF1000F40F0BB80734497
:1025C000002C5ED100290CBF00206FF009009AF8A2
:1025D0000010784C03440C2010FB01312160EAE428
:1025E000039E019C36780396009E247801943478EB
:1025F0006F4E714899F800E0009496F800906F4C87
:102600009DF80C6086709DF80460067080F806E006
:102610009DF8006080F803909CF800C02478DFF8F3
:10262000B491DDF804E080F80880077180F805C0F7
:10263000C671417244704FF00008012000950021DE
:102640005D4C0D465FFA88FC4F46764607E002284F
:1026500009D00A290BD014F8016F17F8010F864230
:1026600001F10101F3D101350A29EDB2F3D1092DB0
:1026700072D808F10108B8F1100F36D019F80A0F16
:10268000DDE70020A3E74FF0000E98E7029879E716
:10269000CEEB040003900198041C18BF01245DE7F1
:1026A000019800284ED0039890F800E0BEF1000F8A
:1026B000EED1601E0390744650E7841B01264AE465
:1026C0000B9A3F4B9142CCBF012200221A703EDC94
:1026D0000A9A3C4B9142CCBF012200221A7052DD73
:1026E00003258AF80050384BFDE530483749047817
:1026F000C86B0299009D097801342044CBEB00009F
:10270000084400219AF800402A4B401A0C2111FB82
:10271000040119604FE41BF1000618BF01269BE578
:102720002349097800293FF4B3AE1BF1000618BF16
:102730000126AEE6049800280CBF4FF0000E4FF0C3
:10274000090E3CE7039890F800E03046FDE60425CA
:102750008AF800501C4BC6E514481C49047851F80F
:1027600028000299009D097801342044CBEB000039
:1027700066460844002BC4D0002EC2D1BBF1000F26
:10278000BFD00121BEE7099A114B9142CCBF012273
:1027900000221A7004DD02258AF800500A4BA2E5D7
:1027A000089B994218DD01259AE500BF148AFF1F96
:1027B0008F9EFF1F389EFF1FB49CFF1FC09EFF1FF0
:1027C000A09EFF1F9F9EFF1FF29DFF1FC089FF1F3E
:1027D0009E9EFF1FD0210100134B1D78012D21D992
:1027E000124A8AF800501288002A3FF47CAD104A41
:1027F0001288013A92B2062A3FF675AD0D4A127858
:10280000002A3FF470AD0C4A1268012A7FF46BADC8
:102810000A4A0B4E10680C2290FBF2F102FB1102E7
:10282000328060E535465EE5F29DFF1FCC9EFF1FBE
:10283000FE9DFF1FE29CFF1F749EFF1FC49EFF1F93
:102840003C9EFF1F2DE9F04F3A4B1B788BB0002BBD
:102850006BD10E200AF0AEFC0DF0ACFF01463648FD
:10286000364E374DFDF766FE3348FDF739FE0EF064
:10287000BBF980F30C003060FFF7F8FA2C68012CEC
:102880007AD0022C00F09D82032C00F0AB832D4EF9
:102890002D4C33682D4A2E4E0993099B31681288BE
:1028A0002360591A013A9142274F00F28582294E3E
:1028B00032689A1A0D2A00F27882274E32689A1AE4
:1028C000132A00F26D82254E32689A1A252A1AD9E7
:1028D000234B1B88002B40F05481224B1B78002B8C
:1028E00040F04F81FEF7EAFB1F4B1B881B3B9BB25E
:1028F000022B04D81D4B1B78002B40F0458104F0BF
:1029000007F8236833601A4D2A689B1A502B00F28F
:102910000382184B1B88012B00F01B8206F0E6FD9A
:1029200006F014FC0BB0BDE8F08F07F0ABFE0BB067
:10293000BDE8F08F489CFF1F109EFF1F4C9EFF1F9D
:10294000749EFF1FBC9FFF1F089EFF1FBC89FF1FB7
:10295000DC9CFF1FC89CFF1FA09CFF1FA49CFF1FA7
:10296000EE9DFF1F409CFF1F7A9EFF1F309CFF1FA4
:10297000E89DFF1F509EFF1FDFF80C939C4AB9F89B
:1029800000001378834204D0C3B21846137006F0D7
:10299000E9FCDFF8F082974AB8F8003011789942E4
:1029A00004D0954F3978002940F0DA86934A33688D
:1029B0001288934E9A42C0F2F180924A1278002A0D
:1029C00040F0EC80DFF8C4A2BAF8003023B98E4B97
:1029D0001B88002B00F0E3848C4A8D4B11881B88E8
:1029E0008C4A0B4412685B1093428B4A126880F247
:1029F000858400219342B4BF01230B4604910093C8
:102A0000ACBF4FF0010B8B4605910E200AF0D2FBB4
:102A1000824B834A1B68176803930133A7F2523233
:102A2000002B8446029240F3C286802BA8BF8023ED
:102A30007C4A7D4912780191002A00F0B98009781A
:102A4000914200F0B580B8F80010DFF838E2994202
:102A500001F0D7806849AEF80030744B4FF0010E9A
:102A600081F800E01978DFF828E2019B8EF8001069
:102A70001A70009B002B00F00D81BAF80030002B7B
:102A800000F008816A4B1B685A1C002A40F39386A9
:102A9000802A00F38F86674C674968482488098834
:102AA00000682144B0EB610FC1F22083A3F148021A
:102AB0000F2A02D8473BA9F800300E200AF07AFB13
:102AC0006FF454731F44874202DC5D4B00221A707E
:102AD0005C4B1B88002B00F009845B4B5B4A1B7826
:102AE0001178994240D0002B3ED059490C78002CE7
:102AF00000F01D87574991F800C0BCF1000F40F06D
:102B00001487554F0097554F55480297524F0078FC
:102B100087F800C0514F4FF0010E87F800C081F8D0
:102B200000E0002841F0C4804E490978002900F0F7
:102B3000E0874D4903910C460978002940F0D6877B
:102B40004A48464F0078397001210297217058B1E8
:102B5000414840490090002008700099029F087089
:102B6000039901243C7008701370414B1B88A3F13A
:102B70001B02012A40F2B8851D2B00F002863D4C55
:102B800087E6FEF73DFAADE63B4B1B78002B3FF4A2
:102B9000B6AE2B68012B7FF4B2AEB2E63168374A8D
:102BA000069106983649106002220B602A6009E7F8
:102BB0001E49DFF8DCE0097800293FF456AF9EF8A3
:102BC000000081423FF451AF03984B2840F3E08767
:102BD0001833802BB8F80000A8BF802398423FF438
:102BE00044AF284803800448012303703DE700BF39
:102BF000DB9DFF1FA89CFF1F319CFF1FE09CFF1F58
:102C0000BC9FFF1F409CFF1FCE9CFF1F589CFF1FB7
:102C1000489EFF1F749CFF1FC89EFF1FB89EFF1F8A
:102C2000209CFF1FAE9EFF1F889CFF1FAF9EFF1FB3
:102C3000389EFF1FF49DFF1FF09DFF1F689CFF1F24
:102C4000E49DFF1FFE9DFF1F5E9CFF1F0C9CFF1F4E
:102C5000D29EFF1F409EFF1F8C9EFF1FE29CFF1F06
:102C6000D39EFF1FCF9EFF1F0D9CFF1F309CFF1F99
:102C70007A9EFF1F089EFF1F7E9EFF1F9C9CFF1FCA
:102C8000049EFF1F0C9EFF1FFC9DFF1F909CFF1FBB
:102C9000899CFF1F029B9C45BFF60FAF864B1B888C
:102CA000002B3FF40AAFBBF1000F7FF4EBAE834B78
:102CB0001B881BB1059B002B7FF4E4AE049B002B0B
:102CC0003FF4FBAE7E4B1A78002A7FF4F6AEDFF8B5
:102CD000649299F8004001221A70002C40F02C8375
:102CE000784B1B78002B02F0C680774B1B78002BAB
:102CF00002F09A83754B1B78002B7FF4DEAE744B89
:102D00001B78002B3FF4D9AEB8F8003071490A3B6C
:102D1000A8F800300A70D0E605F038F96E4B1B7841
:102D200073B96E4B1B785BB96D4B1B7843B96D4B18
:102D30001B782BB96C4B1B7813B903F0BFFD01E076
:102D400003F0C8FD23682B60684B1B88012B7FF4C0
:102D5000E5AD674A674B116867481A78A1F1180317
:102D60002A2101FB03F10160002A00F0A982634CD3
:102D70002368994200F3528310DA61480278002AEE
:102D800040F07C875F4A1068D0F17F0048BF033075
:102D9000801001301B1A994242F3BF86216091E2F4
:102DA000FEF7CCFC236833608DE5FDF761FDFEF78F
:102DB000B1F92368336080E5FDF7A6FC3B6833601A
:102DC00075E5514A34681188A14204DB464B1B78F3
:102DD000002B00F05D834D4E4D48336807934D4BFB
:102DE000079A00681B88121A9A4200F2A980002BE9
:102DF00000F0A680484B1A88002A3FF4C0AE474B2B
:102E000047481B680088A342B8BF2346994241F354
:102E10006681444B1960DFF8208188F80020344F28
:102E2000FDF772FC38687F2840F371853E4B7F3890
:102E300083FB0032C317C3EB620303EB4303A0EB36
:102E400083007330394B01931B883860002B40F0AE
:102E5000CA86234B00931B78002B00F0C683344CAA
:102E60002378002B00F0C183DFF8D090DFF8B8A002
:102E70004FF0000B0CE003F17300C0B298F80010A3
:102E800006F0C8FA23780BF1010B5B4540F3AD83E4
:102E90003B6859F8040F1844A0F17F038AFB032113
:102EA000DA17C2EB610202EB42027F28A3EB820336
:102EB000E1DCFDF7E7FBE0E7CE9CFF1F029EFF1F72
:102EC000E49DFF1FCF9EFF1FF39DFF1FD19EFF1F9D
:102ED000D29EFF1F319CFF1FE29CFF1F409EFF1FE1
:102EE0008C9EFF1F0D9CFF1F409CFF1F509EFF1FCD
:102EF000C49EFF1F969CFF1FA49EFF1F389CFF1FB0
:102F0000909EFF1F149CFF1FE09CFF1FBC9FFF1F94
:102F10009C9CFF1FCC9CFF1F2E9CFF1F049EFF1F2D
:102F2000A29EFF1F109CFF1FABAAAA2A709CFF1F26
:102F30008089FF1FE59DFF1FC19CFF1F5889FF1F50
:102F4000554B564A1B681088554AA342B8BF2346C2
:102F5000994200F37A82534C12888342A8BF0346F9
:102F60002360002A7FF457AF9942C8BF134640F34D
:102F70007382401AB0F5804FAABF9B03C3EB833323
:102F8000013093FBF0F0FDF7A5FBC0F3C6100DF088
:102F900011FC454B044618880DF00CFC43490746CC
:102FA00020460DF05BFC014638460DF057FC2146EB
:102FB0000DF04CFB4FF07E5104460DF0EDFD002866
:102FC00041F071803A4920460DF004FE002840F09F
:102FD000698620460DF02EFEC0B2DFF8F48088F836
:102FE00000001CE7334B34681988A14274DD324B72
:102FF0001B78002B70D1DFF8DC9099F800007F2857
:1030000040F33886A3F155337F3803F1004383FB47
:103010000032C317C3EB620303EB4303A0EB83004F
:103020007330264B01931B88C0B289F80000002B37
:1030300041F03580224B00931B78002B00F0A484D4
:10304000204C2378002B00F09F841F4FDFF87C80FA
:103050004FF0000A0AE003F17300C0B206F002FA72
:1030600023780AF1010A534540F38E8457F8043F50
:1030700099F800001844A0F17F0388FB0321DA17B8
:10308000C2EB610202EB42027F28A3EB8203E2DC87
:10309000FDF7F8FAE1E700BF049EFF1FA29EFF1FA5
:1030A0002E9CFF1F109CFF1FB09EFF1FCDCCCC3D60
:1030B0000000FE42E09CFF1F409CFF1F709CFF1F12
:1030C0008C9EFF1F8089FF1F5889FF1FABAAAA2A69
:1030D000C19CFF1F369EFF1FB34F38687F2800F347
:1030E000C281FDF7CFFADFF8249399F800A082455A
:1030F00000F02182AD4B1B88002B43D1AC4AAD4878
:1031000012680088914205DC8242D4BFC1EB020301
:10311000C1EB0003411AB1F5804FA6BF9B030131FB
:10312000C3EB833393FBF1F0FDF7D4FAC0F3C61081
:103130000DF040FBA04B044618880DF03BFB9F4967
:10314000804620460DF08AFB014640460DF086FB86
:1031500021460DF07BFA4FF07E5104460DF01CFD28
:10316000002840F08F87964920460DF033FD002857
:1031700040F0958520460DF05DFDC0B2DFF89082ED
:1031800088F80000BAF17F0F40F3BD838D48AAF1A3
:103190007F0A80FB0A304FEAEA73C3EB600000EB62
:1031A0004000AAEB80007330874B00931B78C0B2BD
:1031B00089F80000002B40F01A83844B03931B789E
:1031C000002B40F04B85824B02931B78002B40F084
:1031D0007E87804B0193029B1B78FBB17E4B1B8843
:1031E000012B00F0C385022B01F05380032B01F06B
:1031F0009281042B01F09D83052B01F03E84062B68
:1032000001F00D86072B01F0C187082B02F07880B2
:10321000092B02F08C810A2B02F0C283009B1B78E1
:10322000002B00F07684019B6A4C1988002900F07D
:10323000FD8438687F2840F36383624B7F3883FBCB
:103240000032C317C3EB620303EB4303A0EB83001D
:1032500073303860002940F0AC84009B1B78002B51
:1032600000F075815D4C2378002B00F07081DFF851
:10327000A4A1DFF89C814FF0000B0CE003F1730078
:10328000C0B298F8001006F0C5F823780BF1010BD6
:103290005B4540F35C813B685AF8040F494A184487
:1032A000A0F17F0382FB0321DA17C2EB610202EB7C
:1032B00042027F28A3EB8203E0DCFDF7E3F9DFE7BE
:1032C000474B1960474B1B68A92202FB03F3002BF5
:1032D000BCBF03F57F533F339B13543B194481F329
:1032E0000C0128200AF0ECFAFFF718BB384C3E48D6
:1032F0003549364A237003700B7035E493424FF022
:10330000000B80F2BD800123CDF800B0CDF814B0E1
:103310000493FFF77ABB354B1B78002B7FF4CDABC2
:10332000039B334A243B83F34703D9B25B201360EA
:1033300006F048F899F80040032C30D1DFF8D88027
:1033400098F80030002B42F0BE812A4F3B78002BCA
:1033500042F0AC81254C2378002B42F09A81264B19
:103360001B78002B42F08881244A1380244B1B7861
:10337000002B42F04E820D4B7F221A8098F80030CD
:103380006BB93B785BB923784BB91E4A7F21072084
:10339000138006F017F87F210B2006F013F81A4B64
:1033A0001F68FFF78ABB00BFC49EFF1F2E9CFF1F34
:1033B000109CFF1FA29EFF1FB09EFF1FCDCCCC3DD7
:1033C0000000FE42ABAAAA2A8C9EFF1F0D9CFF1F85
:1033D000E29CFF1F709CFF1FFE9DFF1F8089FF1F47
:1033E000389CFF1FB889FF1F409EFF1FD29EFF1F02
:1033F000549CFF1FD19EFF1FF39DFF1FD29CFF1FF8
:10340000D39EFF1F349EFF1F209CFF1F369EFF1F71
:10341000C19CFF1F5889FF1FCF9EFF1FBA4A10781B
:10342000002840F05983B94A1268D2F17F0248BFA0
:10343000033203EBA202531CB54A23609942B8BF82
:103440001160FFF63FAF19463CE7B24B1288196096
:10345000002A7FF4E0AC0B469842D4BFC1EB0003D6
:10346000C1EB030385E5AC4B7F3883FB0032C31708
:10347000C3EB620303EB4303A0EB8300733032E63C
:103480000123CDF810B0CDF800B00593FFF7BDBA19
:1034900001232B60A14EA24CFFF7FBB9029B1B78C6
:1034A000FBB1A04B1B88012B00F0E284022B00F043
:1034B0006F86032B01F0A580042B01F05F82052BA2
:1034C00001F05283062B01F0A284072B01F0068540
:1034D000082B01F04C87092B02F04A800A2B02F0DE
:1034E0002882019B1B88002B00F06C83009B1B78BB
:1034F0003BB9039B1B7823B9029B1B78002B01F07F
:103500000080894B1B78002B00F0288187490B78BD
:10351000082B00F2238186483A680068854C013305
:10352000DBB25F1E101A44F827000B70824B346820
:10353000198889F80020A142784EBFF620AB326886
:103540007E4B0892089A764C1A60FFF7A2B9039B4B
:103550001B78002BA2D03B68A3F10C007F2840F31E
:103560006C836D488B3B80FB0320DA17C2EB600055
:1035700000EB4000A3EB800303F17300DFF8D08180
:10358000C0B298F8001005F045FF009B1B78002B97
:1035900084D0664C2378002B80D0DFF8B8A14FF0A0
:1035A000000B0CE003F17300C0B298F8001005F0B6
:1035B00031FF23780BF1010B5B457FF76FAF3B6861
:1035C0005AF8040F544A1844A0F18B0382FB0321DC
:1035D000DA17C2EB61020C3802EB42027F28A3EB40
:1035E0008203DFDCFDF74EF8DEE74F4B1B78002B44
:1035F00040F0EE823B68524A1278002A45D0A3F18F
:103600000C007F2840F33383434A8B3B82FB03212A
:10361000DA17C2EB610202EB4202A3EB820303F171
:103620007300C0B298F8001005F0F4FE009B1B7800
:1036300053B33E4C23783BB3DFF81891DFF8D8A0A2
:103640004FF0000B0BE003F17300C0B298F80010CC
:1036500005F0E0FE23780BF1010B5B4514DD3B68C0
:1036600059F8040F1844A0F18B038AFB0321DA17E1
:10367000C2EB61020C3802EB42027F28A3EB82030B
:10368000E1DCFCF7FFFFE0E73B682E4A1278FAB175
:10369000244A1288012A00F07284022A00F07786F8
:1036A000032A01F02F80042A01F08C81052A01F001
:1036B000CE82062A01F0D883072A01F0B484082AB2
:1036C00001F0CD86092A01F098870A2A02F0F980D4
:1036D000019A1288002A00F08D821B4A104C137048
:1036E00003232B60FFF7D5B8DFF86C8098F8003023
:1036F000002B40F01081154F3B78002B40F0F984EF
:10370000074C3B70FFF7C5B8909EFF1F149CFF1F2E
:10371000389CFF1F109CFF1FABAAAA2ABC9FFF1F4B
:10372000089EFF1FFE9DFF1F409EFF1F8089FF1FF9
:10373000349CFF1F5C89FF1FE09CFF1F689FFF1FD9
:103740000D9CFF1FE29CFF1F369EFF1F2C9CFF1F3E
:10375000C19CFF1F5889FF1F309CFF1F3A68E5E698
:10376000DBB21846137005F00BFEAC4BAC491A46A1
:10377000AC4B184600230B703B7013700370FFF7BF
:1037800015B9DFF8BC8298F80030002B40F0CF81EB
:10379000A54F3B78002BB3D0A44BA54C1988A22091
:1037A00005F094FF98F800303B70FFF772B80123E2
:1037B000FFF73EB980249F499F4BA04A09881B8888
:1037C00012680B44B2EB630FBFF677A99C4B1B78D2
:1037D000002B40F01C82B8F800309A4AA3423FF414
:1037E0006CA9994B148001221A70FFF766B9974BA8
:1037F00001931B88002B42F08A818A4B0393944BE0
:103800000293944C23786BB3DFF85C82DFF848A214
:103810004FF0000B09E003F17300C0B205F022FE87
:1038200023780BF1010B5B451CDD58F8043F99F838
:1038300000001844A0F17F038AFB0321DA17C2EBD2
:10384000610202EB42027F28A3EB8203E3DCFCF778
:1038500019FFE2E77E4B029305F004FE009B1B7804
:10386000002BCED1039B1B78002B3FF4B4AC99F80E
:103870000030A3F10C007F2840F3ED8176488B3BAC
:1038800080FB0320DA17C2EB600000EB4000A3EBE3
:10389000800303F17300C0B205F0E4FD009B1B78C8
:1038A000002B00F0CD816B4C2378002B01F0C082FF
:1038B000DFF8B481DFF8A0A14FF0000B0AE003F1BC
:1038C0007300C0B205F0CEFD23780BF1010B5B4510
:1038D0007FF781AC58F8043F99F800001844A0F134
:1038E0008B038AFB0321DA17C2EB61020C3802EB6F
:1038F00042027F28A3EB8203E1DCFCF7C3FEE0E792
:10390000FCF7C0FEA5E45046FCF7BCFE4CE4FCF717
:10391000B9FEFFF797BA514A1278002A40F0D581D4
:10392000414F434C3B70FEF7B4BF002008704C4938
:10393000087840B1394900910978002900F0B58133
:10394000009F002139704749097800297FF4F1A8C8
:10395000002C40F0CE80002840F0CB80384C2F4F18
:1039600094F800E02F4C0394394C02942D4C2C49D0
:103970002070374C0097087038702070BEF1000F2F
:103980007FF4E9A8FFF7F0B8264B1B78002B6DD029
:1039900099F80030A3F10C007F2840F3CC832E4A25
:1039A0008B3B82FB0321DA17C2EB610202EB42027E
:1039B000A3EB820303F17300C0B205F053FD009B3B
:1039C0001B78002B52D0234C2378002B4ED0264F4F
:1039D000DFF884804FF0000A09E003F17300C0B201
:1039E00005F040FD23780AF1010A53453EDD57F802
:1039F000043F99F800001844A0F18B0388FB0321D1
:103A0000DA17C2EB61020C3802EB42027F28A3EB0B
:103A10008203E2DCFCF736FEE1E700BF8C9EFF1F6D
:103A2000409EFF1F0D9CFF1F2C9CFF1F809EFF1FB1
:103A3000089EFF1FF49DFF1FF09DFF1F689CFF1F46
:103A4000309CFF1F0C9EFF1F319CFF1F709CFF1FAF
:103A5000E29CFF1F8089FF1FABAAAA2A7E9EFF1F40
:103A6000D39EFF1FCF9EFF1F5889FF1FA84B1B78B7
:103A7000FBB1A84B1B88012B00F0D486022B00F071
:103A8000CF87032B01F04A81042B01F0E481052B41
:103A900001F01B84062B01F0DA84072B01F01F864E
:103AA000082B01F0DD86092B01F0C9870A2B01F0F4
:103AB000A687019B1B88002B00F0EC82964B1B789D
:103AC000002B40F0E282954B954A1988346800201B
:103AD000012310602B602EE50130C0B2022886BFA2
:103AE0000021117010701946FFF7ECBB03980021FC
:103AF00001708C49097800293FF436A88449029165
:103B00000978002900F0B287029800210170FFF7C0
:103B10002BB8039B1B78002B7FF485AB029B1B7893
:103B2000002B7FF480AB019B1988FFF782BB7E4A94
:103B30001278002A3FF4F4AE7C4F387802F052FF3E
:103B40007B4B1B78002B00F0BB8439887E2900F268
:103B5000B784784CDFF80C922368D9F800209B1AC0
:103B60000F2B40F29680744B01311B8889B239804B
:103B70002BB1052B03D0C9B2052005F023FC6F4FF4
:103B8000226898F80030C9F800203B70FEF781BE2B
:103B9000243B002BB8F8000040F3788498423EF4B0
:103BA00064AF9BB26648A8F8003001230370FEF7AB
:103BB0005CBFDFF89081C0B298F8001005F02AFCD5
:103BC000FFF74BBB5F4B3878197805F023FC8DE489
:103BD0007F21402005F0F6FB5B495C4A3B680B60A7
:103BE0000021117007E5C0B298F8001005F012FC32
:103BF000FFF72FB9D8B298F8001005F00BFC3B681E
:103C00006BE5534BDFF860E11978FEF72EBF4B2CC4
:103C100040F34C821834802CB8F800304D4AA8BFCD
:103C20008024A3427FF4DDADFEF747BF99F8000082
:103C300005F018FC2188FFF7FCBAFCF723FD9DE492
:103C4000029B1B78002B7FF4C9AA039B1B78002BD7
:103C50007FF4E9AA67E7FCF715FD1CE63E4B0193EC
:103C60001B88002B7FF4F6AD294B0293FFE5FCF790
:103C700009FDD6E4FCF706FDFFF7D3B90132D2B255
:103C8000022A40F25E82002202701946FFF71ABB38
:103C9000284C2A4F98F800303B70FEF7FABD7F2081
:103CA000FFF76CBA7F20FFF798B9194F1A490297AE
:103CB0004FF0000C81F800C0009F02994FF0010EF8
:103CC00087F800E081F800C03DE6244F387802F024
:103CD00089FE174B1B78002B00F03A8239887E2929
:103CE00000F23682134CDFF87C902368D9F800206C
:103CF0009B1A0F2BCDD91A4B0131188889B2398004
:103D0000002800F04182C9B2C0B205F05BFB36E783
:103D1000E29CFF1FFE9DFF1F409EFF1FE09CFF1FB8
:103D2000109CFF1F309CFF1F7E9EFF1F809EFF1F69
:103D3000D49EFF1F089EFF1FE69CFF1F2C9CFF1FA9
:103D4000319CFF1FC19CFF1F349CFF1F8089FF1FF8
:103D5000AF9EFF1F0C9EFF1F709CFF1F649CFF1FE8
:103D6000B09CFF1FBC9EFF1F899CFF1FDFF8B4A300
:103D700099F80000BAF80030E34AE44CC31A82FB19
:103D8000031ED917C1EB6E0101EB4101A3EB8103C7
:103D900003EB430354F8233018447F2840F3AE84E8
:103DA0007F3882FB0032C317C3EB620303EB43038C
:103DB000A0EB83007330DFF870B3C0B205F052FBA4
:103DC000BBF80030022B7FF629AA99F80010BAF848
:103DD0000030CD4ACB1A82FB030ED817C0EB6E0021
:103DE00000EB4000A3EB800303EB430304EB8303EE
:103DF000586808447F2840F320877F3882FB0032D0
:103E0000C317C3EB620202EB4202A0EB82007330E5
:103E1000C0B205F027FBBBF80030032B7FF6FEA9EC
:103E200099F80010BAF80030B74ACB1A82FB030E9B
:103E3000D817C0EB6E0000EB4000A3EB800303EB50
:103E4000430304EB8304A06808447F2840F3708197
:103E50007F3882FB0032C317C3EB620202EB4202DF
:103E6000A0EB82007330C0B205F0FCFAFFF7D6B9C0
:103E7000DFF8B0A23868BAF80030A34AA34CC31ADE
:103E800082FB031ED917C1EB6E0101EB4101A3EBCD
:103E9000810303EB430354F8233018447F2840F395
:103EA00029847F3882FB0032C317C3EB620303EB24
:103EB0004303A0EB83007330DFF87082DFF868B251
:103EC00098F80010C0B205F0A5FABBF80030022B3C
:103ED0007FF607AB3968BAF800308B4ACB1A82FB01
:103EE000030ED817C0EB6E0000EB4000A3EB80037D
:103EF00003EB430304EB8303586808447F2840F333
:103F000098867F3882FB0032C317C3EB620202EB54
:103F10004202A0EB82007330C0B298F8001005F0A6
:103F200079FABBF80030032B7FF6DBAA3968BAF8C0
:103F30000030754ACB1A82FB030ED817C0EB6E0017
:103F400000EB4000A3EB800303EB430304EB83048B
:103F5000A06808447F2840F3F8807F3882FB003255
:103F6000C317C3EB620202EB4202A0EB8200733084
:103F700098F80010C0B205F04DFAFFF7B2BADFF8BA
:103F8000A4A16149BAF80020604C9A1A81FB020E84
:103F9000D017C0EB6E0000EB4000A2EB800202EBFA
:103FA000420254F8220018447F2840F32284A0F1F2
:103FB0007F0381FB0321DA17C2EB610000EB4000B5
:103FC000A3EB80007330DFF860B198F80010C0B246
:103FD00005F020FABBF80030022B50D93968BAF846
:103FE0000030494ACB1A82FB030ED817C0EB6E0093
:103FF00000EB4000A3EB800303EB430304EB8303DC
:10400000586808447F2840F385867F3882FB003259
:10401000C317C3EB620202EB4202A0EB82007330D3
:10402000C0B298F8001005F0F5F9BBF80030032B8A
:1040300025D93868BAF80030334AC31A82FB031E08
:10404000D917C1EB6E0101EB4101A3EB810303EB37
:10405000430304EB8304A36818447F286EDD7F3894
:1040600082FB0032C317C3EB620202EB4202A0EBF9
:1040700082007330C0B298F8001005F0CBF93B68AD
:10408000FFF726BB0120FFF779B80021402005F09B
:1040900099F918E599F8000005F0E4F90EE505F046
:1040A000E1F9FEF7C7BF0120FEF797BF243C002CC3
:1040B000B8F8003040F3C585A3423EF4FEACA4B28C
:1040C000134BA8F8004001221A70FEF7F6BC114B02
:1040D00001931B88002B7FF4BFABFFF77CB80E4920
:1040E0008342A8BF03460B60FEF795BE1446FFF758
:1040F0006DBB0A4B0A4C19886A2005F0E7FA98F85C
:1041000000303B70FEF7C5BBABAAAA2AD420010041
:10411000319CFF1F709CFF1F109CFF1F649CFF1FA2
:10412000089EFF1F3C9EFF1F469CFF1FC19CFF1F58
:10413000FCF7A8FA97E6FCF7A5FA3DE4FCF7A2FA2B
:1041400098E702701946FFF7BDB8FCF79BFA0FE736
:10415000D14B1B78002B3FF49BAD3B88CF4F002BFE
:104160003FF496ADCE4CDFF848932268D9F80010A2
:10417000521A0F2A7FF68DADCA4A013B108899B2B8
:10418000398000287FF4BFADC8B205F08FF9F6E49E
:10419000DFF820A33868BAF80030C34AC34CC31A0A
:1041A00082FB031ED917C1EB6E0101EB4101A3EBAA
:1041B000810303EB430354F8233018447F2840F372
:1041C00025847F3882FB0032C317C3EB620303EB05
:1041D0004303A0EB83007330DFF8DC82DFF8DCB24E
:1041E00098F80010C0B205F015F9BBF80030022BAA
:1041F0007FF677A93968BAF80030AB4ACB1A82FB50
:10420000030ED817C0EB6E0000EB4000A3EB800359
:1042100003EB430304EB8303586808447F2840F30F
:104220000E867F3882FB0032C317C3EB620303EBB9
:104230004303A0EB83007330C0B298F8001005F080
:10424000E9F8BBF80030032B7FF64BA93868BAF8C1
:104250000030954AC31A82FB031ED917C1EB6E01C9
:1042600001EB4101A3EB810303EB430304EB830464
:10427000A36818447F287FF768AF7F3882FB00323D
:10428000C317C3EB620303EB4303A0EB830073305C
:104290006EE6DFF820A299F80000BAF80030824AF2
:1042A000824CC31A82FB031ED917C1EB6E0101EBCE
:1042B0004101A3EB810303EB430354F8233018447B
:1042C0007F2840F3A7837F3882FB0032C317C3EBFC
:1042D000620303EB4303A0EB83007330DFF8DCB130
:1042E000C0B205F0BFF8BBF80030022B7EF696AFE7
:1042F00099F80010BAF800306B4ACB1A82FB030E13
:10430000D817C0EB6E0000EB4000A3EB800303EB7B
:10431000430304EB8303586808447F2840F39385E4
:104320007F3882FB0032C317C3EB620303EB430306
:10433000A0EB83007330C0B205F094F8BBF80030F6
:10434000032B7EF66BAF99F80010BAF80030564A8E
:10435000CB1A82FB030ED817C0EB6E0000EB4000B7
:10436000A3EB800303EB430304EB8304A06808443E
:104370007F287FF7DDAE7F3882FB0032C317C3EBA7
:10438000620303EB4303A0EB830073306BE5DFF8BC
:1043900024A14549BAF80020444C9A1A81FB020E28
:1043A000D017C0EB6E0000EB4000A2EB800202EBE6
:1043B000420254F8220018447F2840F32E83A0F1D3
:1043C0007F0381FB0321DA17C2EB610000EB4000A1
:1043D000A3EB80007330DFF8E4B098F80010C0B2AF
:1043E00005F018F8BBF80030022B7FF648AE3968AC
:1043F000BAF800302C4ACB1A82FB030ED817C0EB58
:104400006E0000EB4000A3EB800303EB430304EBDF
:104410008303586808447F2840F319857F3882FB5E
:104420000032C317C3EB620303EB4303A0EB83002B
:104430007330C0B298F8001004F0ECFFBBF8003005
:10444000032B7FF61CAE3868BAF80030164AC31A40
:1044500082FB031ED917C1EB6E0101EB4101A3EBF7
:10446000810303EB430304EB8304A36818447F2810
:104470007FF764AE7F3882FB0032C317C3EB620361
:1044800003EB4303A0EB83007330F3E501283EF414
:10449000ECAA0123FFF786BBD39EFF1F649CFF1F7E
:1044A000089EFF1FB09CFF1FABAAAA2ACC230100C5
:1044B000BC9EFF1F3C9EFF1FC19CFF1F469CFF1F11
:1044C000CE4B1B78002B3FF4E3AB3B88CC48002B52
:1044D0003FF4DEABCB4CDFF83C932268D9F80010F8
:1044E000521A0F2A7FF6D5ABC74A013B128899B200
:1044F0000180002A3FF443AB052A7FF43CABFFF771
:104500003EBB4FF47A43013BFDD199F8000004F023
:10451000A9FFFEF7F6BFDFF800A399F80000BAF88C
:104520000030BA4ABA4CC31A82FB031ED917C1EB3A
:104530006E0101EB4101A3EB810303EB430354F84C
:10454000233018447F2840F3E8817F3882FB003213
:10455000C317C3EB620202EB4202A0EB820073308E
:10456000DFF8B8B2C0B204F07DFFBBF80030022B18
:104570007EF654AE99F80000BAF80030A34AC31A88
:1045800082FB0321DA17C2EB610202EB4202A3EBCA
:10459000820303EB430304EB83035B6818447F2827
:1045A00040F31F847F380C2290FBF2F302FB1300D0
:1045B0007330C0B204F056FFBBF80030032B7EF618
:1045C0002DAE99F80000BAF80030904AC31A82FB69
:1045D0000321DA17C2EB610202EB4202A3EB820372
:1045E00003EB430304EB8304A36818447F287FF79D
:1045F0009FAD7F380C2290FBF2F302FB1300733067
:1046000031E4DFF814A23868BAF800307F4A804CF1
:10461000C31A82FB031ED917C1EB6E0101EB4101E6
:10462000A3EB810303EB430354F8233018447F28A2
:1046300040F370817F3882FB0032C317C3EB620204
:1046400002EB4202A0EB82007330DFF8D481DFF886
:10465000CCB198F80010C0B204F0DCFEBBF800301A
:10466000022B7EF63EAF3868BAF80030674AC31AAC
:1046700082FB0321DA17C2EB610202EB4202A3EBD9
:10468000820303EB430304EB83035B6818447F2836
:1046900040F3AB837F380C2290FBF2F302FB130054
:1046A0007330C0B298F8001004F0B4FEBBF80030CC
:1046B000032B7EF616AF3868BAF80030534AC31A97
:1046C00082FB0321DA17C2EB610202EB4202A3EB89
:1046D000820303EB430304EB8304A36818447F289D
:1046E0007FF733AD7F380C2290FBF2F302FB13000F
:1046F00073303DE4FBF7C6FFFFF7DEBBFBF7C2FFFD
:10470000FFF759BBDFF810A14049BAF80020404C30
:104710009A1A81FB020ED017C0EB6E0000EB40002E
:10472000A2EB800202EB420254F8220018447F28D8
:1047300040F3F680A0F17F0381FB0321DA17C2EB7F
:10474000610101EB4101A3EB81007330DFF8CCB0D4
:1047500098F80010C0B204F05DFEBBF80030022BE8
:104760007FF68DAC3868BAF80030284AC31A82FB4D
:104770000321DA17C2EB610202EB4202A3EB8203D0
:1047800003EB430304EB83035B6818447F2840F387
:1047900038837F380C2290FBF2F302FB1300733056
:1047A000C0B298F8001004F035FEBBF80030032BBF
:1047B0007FF665AC3868BAF80030144AC31A82FB39
:1047C0000321DA17C2EB610202EB4202A3EB820380
:1047D00003EB430304EB8304A36818447F287FF7AB
:1047E000ADAC7F380C2290FBF2F302FB1300733068
:1047F00040E4FBF747FFFFF7E6BB00BFD39EFF1F78
:10480000809EFF1F089EFF1FE69CFF1FABAAAA2ADF
:104810005C240100BC9EFF1F3C9EFF1F469CFF1FA7
:10482000C19CFF1FDFF838A399F80000BAF80030E8
:10483000C34AC44CC31A82FB0317D917C1EB6701E3
:1048400001EB4101A3EB810303EB430354F8233055
:1048500018447F286ADD7F3882FB0032C317C3EB20
:10486000620202EB4202A0EB82007330DFF8F4B286
:10487000C0B204F0F7FDBBF80030022B7FF619A997
:1048800099F80000BAF80030AD4AC31A82FB032140
:10489000DA17C2EB610202EB4202A3EB820303EBE5
:1048A000430304EB83035B6818447F2840F3AC8226
:1048B0007F380C2290FBF2F302FB13007330C0B27E
:1048C00004F0D0FDBBF80030032B7FF6F2A899F876
:1048D0000000BAF800309A4AC31A82FB0321DA17A3
:1048E000C2EB610202EB4202A3EB820303EB430340
:1048F00004EB8304A36818447F2814DD7F380C225E
:1049000090FBF2F302FB13007330C0B204F0AAFD77
:10491000FFF7CFB8FBF7B6FE97E6FBF7B3FE1FE64F
:10492000FBF7B0FE12E7FBF7ADFEEEE7FBF7AAFEE2
:104930009CE7DFF82CA299F80000BAF80030804A12
:10494000814CC31A82FB031ED917C1EB6E0101EB28
:104950004101A3EB810303EB430354F823301844D4
:104960007F28DADD7F3882FB0032C317C3EB620396
:1049700003EB4303A0EB83007330F1E5DFF8E0A124
:104980003868BAF800306E4A6F4CC31A82FB031EB7
:10499000D917C1EB6E0101EB4101A3EB810303EBDE
:1049A000430354F8233018447F28B3DD7F3882FB5B
:1049B0000032C317C3EB620303EB4303A0EB830096
:1049C000733042E6DFF898A15D49BAF800205E4CEA
:1049D0009A1A81FB020ED017C0EB6E0000EB40006C
:1049E000A2EB800202EB420254F8220018447F2816
:1049F00096DDA0F17F0381FB0321DA17C2EB610092
:104A000000EB4000A3EB800073309FE6FBF73AFE1B
:104A1000FFF7E2BBFBF736FE60E4FBF733FEDAE4B8
:104A2000DFF83CA199F80000BAF80030444A474C3E
:104A3000C31A82FB0317D917C1EB670101EB4101D0
:104A4000A3EB810303EB430354F8233018447F287E
:104A50007FF76CAF7F3882FB0032C317C3EB620372
:104A600003EB4303A0EB83007330FFE6384800906C
:104A7000384839490390FEF76EB8DFF8E4A099F89A
:104A80000000BAF800302E4A344CC31A82FB0321CE
:104A9000DA17C2EB610202EB4202A3EB820303EBE3
:104AA000430354F8233018447F2840F3A7817F380C
:104AB0000C2290FBF2F302FB13007330DFF8A4B07A
:104AC000C0B204F0CFFCBBF80030022B19D999F822
:104AD0000000BAF800300C22C11A91FBF2F302FB7D
:104AE000131302FB03435B6818447F2840F385845B
:104AF0007F3890FBF2F302FB13007330C0B204F076
:104B0000B1FCBBF80030032B7EF688ABBAF800305E
:104B100099F800000C22C11A91FBF2F302FB131367
:104B200002FB0344A36818447F287FF701AB7F385A
:104B300090FBF2F302FB13007330FFF794B900BF50
:104B4000ABAAAA2AD4200100E0250100CC23010051
:104B50008C9EFF1F0D9CFF1F409EFF1F70220100B7
:104B60003C9EFF1F469CFF1FDFF864A33868BAF81D
:104B70000030CE4ACE4CC31A82FB0321DA17C2EBB7
:104B8000610202EB4202A3EB820303EB430354F8FE
:104B9000233018447F2840F32E817F380C2290FB6D
:104BA000F2F302FB13007330DFF82883DFF828B339
:104BB00098F80010C0B204F02DFCBBF80030022BB6
:104BC0001AD93868BAF800300C22C11A91FBF2F3F6
:104BD00002FB131302FB03435B6818447F2840F376
:104BE000C3837F3890FBF2F302FB13007330C0B233
:104BF00098F8001004F00EFCBBF80030032B7EF692
:104C000070ACBAF8003038680C22C11A91FBF2F38C
:104C100002FB131302FB0344A36818447F287FF7A9
:104C200094AA7F3890FBF2F302FB13007330FFF776
:104C30009FB9FBF727FDFFF76FB9FBF723FDFFF7E0
:104C4000E7B8012B3DF439AF0124FFF739BADFF89B
:104C500080A29649BAF80020954C9A1A81FB02105E
:104C6000D117C1EB600101EB4101A2EB810202EB24
:104C7000420254F8220018447F2840F3B980A0F182
:104C80007F030C2093FBF0F200FB12307330DFF84F
:104C900048B298F80010C0B204F0BCFBBBF800307A
:104CA000022B1AD93868BAF800300C22C11A91FBCD
:104CB000F2F302FB131302FB03435B6818447F28E3
:104CC00040F34F837F3890FBF2F302FB1300733005
:104CD000C0B298F8001004F09DFBBBF80030032B25
:104CE0007FF6CDA9BAF8003038680C22C11A91FBC2
:104CF000F2F302FB131302FB0344A36818447F285A
:104D00007FF71CAA7F3890FBF2F302FB130073308D
:104D1000FFF7B0B9FBF7B6FCFFF782B9DFF8B0A137
:104D200099F80000BAF80030604A624CC31A82FB5E
:104D30000321DA17C2EB610202EB4202A3EB82030A
:104D400003EB430354F8233018447F2846DD7F38B3
:104D50000C2290FBF2F302FB13007330DFF878B102
:104D6000C0B204F07FFBBBF80030022B19D999F8D0
:104D70000000BAF800300C22C11A91FBF2F302FBDA
:104D8000131302FB03435B6818447F2840F38B80B6
:104D90007F3890FBF2F302FB13007330C0B204F0D3
:104DA00061FBBBF80030032B7EF683AEBAF800300F
:104DB00099F800000C22C11A91FBF2F302FB1313C5
:104DC00002FB0344A36818447F287FF7ACAD7F380B
:104DD00090FBF2F302FB1300733096E5FBF752FCF5
:104DE000BCE7FBF74FFCFFF7E4BBFBF74BFC58E4D9
:104DF000FBF748FC4BE7FBF745FCD5E6FBF742FC2D
:104E00005CE6FBF73FFCCBE4FBF73CFC57E5DFF847
:104E1000C0A03868BAF80030244A274CABE6DFF867
:104E2000B0A099F80000BAF80030204A224C2CE6D5
:104E3000029B1B78002B7EF4D1A9FEF7F4B9FBF797
:104E400021FCFFF7F9B9FBF71DFCFFF774BAFBF77C
:104E500019FCFFF7EEBADFF878A099F80000BAF86D
:104E60000030124A154C61E7DFF864A00F49BAF828
:104E70000020114CF1E6124B1B78002B00F0C18290
:104E8000104B1B78002B7DF418AE0F4B1B78002BBA
:104E90003DF413AEB8F800300C490A33A8F80030DE
:104EA0000A70FDF70ABEFBF7EDFB77E7ABAAAA2A6B
:104EB000702201005C24010050250100E025010062
:104EC000F39DFF1FD19EFF1FD29EFF1F319CFF1F2E
:104ED0003C9EFF1FC19CFF1F469CFF1FA44C2388C4
:104EE000002B40F0BE83DFF8A0B2A249A24A098895
:104EF000D7F80080B2F800E0A048C1EB080C0C2203
:104F00009CFBF2F102FB11C14FF0900C0CFB0EFE6A
:104F100002FB01E16FF00B0E405880440EFB038052
:104F20007F2840F30285A0F17F0393FBF2F002FBA0
:104F300010307330924BC0B2197804F06BFABBF8A2
:104F4000002023881344022B23DD8A4A8A4B1188D0
:104F50003868B3F800C0DFF824E2411A0C2291FB54
:104F6000F2F302FB1311902303FB0CF302FB01335A
:104F700073445B6818447F2840F3AD857F3890FB0D
:104F8000F2F302FB130073307D4BC0B2197804F0CA
:104F900041FABBF8002023881344032B23DD754A14
:104FA000754B11883868B3F800C0DFF8D0E1411ABA
:104FB0000C2291FBF2F302FB1311902303FB0CF381
:104FC00002FB013373449B6818447F2840F35D85DE
:104FD0007F3890FBF2F302FB13007330684BC0B2D2
:104FE000197804F017FABBF8002023881344042B27
:104FF0007EF777AA634B1B88012B7EF472AA3A686E
:10500000A2F10C007F2840F38F828B3A0C2092FB98
:10501000F0F300FB13207330594BC0B2197804F041
:10502000F9F9FEF75EBA524C2288002A00F0D782C6
:105030005449DFF854B10988BBF8000003318842B5
:1050400027DD4C484C490088B1F800E0DFF82CC15E
:10505000181A0C2190FBF1F901FB19004FF090098F
:1050600009FB0EFE01FB00E06FF00B0E5CF8000088
:1050700003440EFB02307F2840F3B7847F3890FB57
:10508000F1F301FB13007330C0B298F8001004F084
:10509000C1F9BBF8002023881344022B23DD354BD4
:1050A000354A38681B88B2F800C0DFF8D0E0C31A70
:1050B0000C2193FBF1F201FB1232902303FB0CF362
:1050C00001FB023373445B6818447F2840F3E48497
:1050D0007F3890FBF1F301FB13007330C0B298F8F6
:1050E000001004F097F9BBF8002023881344032B29
:1050F00023DD204B204A38681B88B2F800C0DFF857
:105100007CE0C31A0C2193FBF1F201FB12329023D5
:1051100003FB0CF301FB023373449B6818447F28A4
:1051200040F3C1847F3890FBF1F301FB130073302F
:10513000C0B298F8001004F06DF9BBF80020238885
:105140001344042B7EF79BAF0E4B1B88012B7EF480
:1051500096AF3A68A2F10C007F287EF7EFAF8B3A4A
:105160000C2092FBF0F300FB13207330FEF782BF9C
:10517000C49CFF1F3C9EFF1FE69DFF1FD01D01002A
:10518000C19CFF1F629CFF1F469CFF1FCE4C2388C3
:10519000002B40F02782DFF864B3CC49CC4A098861
:1051A00099F80000B2F800E0DFF85483C1EB000C7E
:1051B0000C229CFBF2F102FB11C14FF0900C0CFB96
:1051C0000EFE02FB01E16FF00B0E58F801100844CF
:1051D0000EFB03007F2840F30484A0F17F0393FBC0
:1051E000F2F002FB10307330C0B204F03BF9BBF8B0
:1051F000002023881344022B22DDB44AB44B1188CB
:1052000099F80000B3F800C0DFF8F4E2411A0C226C
:1052100091FBF2F302FB1311902303FB0CF302FB4F
:10522000013373445B6818447F2840F3E5837F387B
:1052300090FBF2F302FB13007330C0B204F012F9DA
:10524000BBF8002023881344032B22DD9F4AA04B88
:10525000118899F80000B3F800C0DFF8A4E2411A01
:105260000C2291FBF2F302FB1311902303FB0CF3CE
:1052700002FB013373449B6818447F2840F3028487
:105280007F3890FBF2F302FB13007330C0B204F0DE
:10529000E9F8BBF8002023881344042B7DF7BEAF48
:1052A0008C4B1B88012B7DF4B9AF99F80020A2F13B
:1052B0000C007F287EF73CAF8B3A0C2092FBF0F37A
:1052C00000FB13207330FEF7CEBDDFF800A299F883
:1052D0000000BAF80030804CC11A0C2291FBF2F3A6
:1052E00002FB131302FB03F3E35818447F287FF7F4
:1052F00075AD7F3890FBF2F302FB130073302DE5A0
:10530000764B1B88182B12D099F800201344A3F178
:1053100018007F2840F3DC830C20973B93FBF0F2CE
:1053200000FB123303F17300C0B204F09BF86C4A27
:105330006C4B127833F81230182B3DF46FAF99F89C
:1053400000201344A3F118007F287EF7F1AE0C2053
:10535000973B93FBF0F200FB123303F17300FEF76F
:1053600082BDFBF78FF9B3E4FBF78CF93FE45B4BAD
:105370001A88182A13D03B681344A3F118007F2819
:1053800040F37D830C20973B93FBF0F200FB12333C
:1053900003F17300544BC0B2197804F03BF8504B42
:1053A00050491A78022A94BF013200221A701A78E2
:1053B00031F81200182810D10424022A02F1010049
:1053C000C2B288BF002231F81200182804D1013C73
:1053D000F3D11A70FEF785B81A703B680344A3F145
:1053E00018007F2840F3A0800C20973B93FBF0F23D
:1053F00000FB123303F173000EE6FBF743F9FFF7EE
:105400007DBB3A4B1B78002B7DF485AF384B1B7866
:10541000002B3DF452ABB8F8003036490133A8F800
:1054200000300A70FDF749BB304B1B78002B7DF430
:1054300044AB2F4B1B78002B3DF43FABB8F800304A
:105440002C49013BA8F800300A70FDF736BBDFF8A5
:105450007CA099F80000BAF80030274C3CE71F4ABE
:105460001288182A12D01344A3F118007F2840F3A1
:10547000C0820C20973B93FBF0F200FB123303F148
:105480007300C0B298F8001003F0C4FF144B154924
:105490001A78022A94BF013200221A701A7831F861
:1054A000120018282FD10424022A02F10100C2B2EE
:1054B00088BF002231F81200182823D1013CF3D113
:1054C0001A703B68FEF704B9C49CFF1F3C9EFF1F87
:1054D000E69DFF1F629CFF1F70220100529CFF1F70
:1054E000C29CFF1F589EFF1FC19CFF1FD19EFF1F24
:1054F000D29EFF1F319CFF1F50250100469CFF1FBD
:10550000D01D01001A703B680344A3F118007F28E6
:105510007EF714AE0C20973B93FBF0F200FB1233A6
:1055200003F17300FEF7A6BDFBF7ACF874E5BF4BC3
:105530001B88182B12D099F800201344A3F11800EF
:105540007F2840F3AD820C20973B93FBF0F200FBE9
:10555000123303F17300C0B203F084FFB44AB54BB9
:10556000127833F81230182B7FF4E9AEFDF756BEEF
:10557000AE4B1A88182A13D03B681344A3F11800C5
:105580007F2840F386820C20973B93FBF0F200FBD0
:10559000123303F17300A84BC0B2197803F03AFF3D
:1055A000A34BA4491A78022A94BF013200221A7030
:1055B0001A7831F8120018287FF40FAF0424022A59
:1055C00002F1010294BFD2B2002231F81200182871
:1055D0007FF402AF013CF2D11A70FDF782BFDFF811
:1055E0007CB22EE5954ADFF874B21288BBF8001041
:1055F000033291427FF7FBADCFE58C4A1288182A1F
:1056000012D01344A3F118007F2840F35E820C20CF
:10561000973B93FBF0F200FB123303F17300C0B22F
:1056200098F8001003F0F6FE814B82491A78022A9E
:1056300094BF013200221A701A7831F8120018282B
:105640007FF461AF0424022A02F1010294BFD2B2B6
:10565000002231F8120018287FF454AF013CF2D137
:105660002EE7764ADFF8F4B11288BBF80010033257
:1056700091427FF764AC38E4714B01227F2107200F
:105680001A8003F09FFE7F210B2003F09BFEFDF7A5
:105690006DBE6C4B04227F2107201A8003F092FE1E
:1056A00000210B2003F08EFEFDF759BE654B022250
:1056B0007F2107201A8003F085FE7F210B2003F055
:1056C00081FEFDF747BE5F4B002107201C8003F0E1
:1056D00079FE7F210B2003F075FEFDF736BE5A4C94
:1056E0002388002B40F0E681DFF870B1574999F824
:1056F0000000574A09881788DFF858E1411A0C2240
:1057000091FBF2FC02FB1C114FF0900C0CFB07F715
:1057100002FB01716FF00B075EF80110014407FBFB
:1057200003107F2840F3C3817F3890FBF2F302FB24
:1057300013007330C0B203F095FEBBF8002023883D
:105740001344022B21DD414B414A99F800001B888C
:10575000B2F800E03F4FC31A0C2193FBF1F201FBBA
:105760001232902303FB0EF301FB02333B445B68D0
:1057700018447F2840F3C8817F3890FBF1F301FB88
:1057800013007330C0B203F06DFEBBF80020238815
:105790001344032B21DD2D4B2D4A99F800001B8863
:1057A000B2F800E02B4FC31A0C2193FBF1F201FB7E
:1057B0001232902303FB0EF301FB02333B449B6840
:1057C00018447F2840F39D817F3890FBF1F301FB63
:1057D00013007330C0B203F045FEBBF800202388ED
:1057E0001344042B7EF765A9144B1B88012B7EF410
:1057F00060A999F80020A2F10C007F287FF793A8F8
:105800008B3A0C2092FBF0F300FB13207330FFF770
:105810007CB8114B00227F2107201A8003F0D2FDB3
:105820007F210B2003F0CEFDFDF7A8BD5A9CFF1F82
:10583000C29CFF1FC89DFF1FC19CFF1F629CFF1FD2
:10584000D29CFF1F349EFF1FC49CFF1F3C9EFF1F66
:10585000E69DFF1FD01D01002E9CFF1F469CFF1FD1
:10586000B04B1B88182B12D099F800201344A3F1D9
:1058700018007F2840F33C810C20973B93FBF0F20B
:1058800000FB123303F17300C0B203F0EBFDA64A34
:10589000A64B127833F81230182B3EF40AA999F867
:1058A00000201344A3F118007F287FF73CA80C20A8
:1058B000973B93FBF0F200FB123303F17300FFF709
:1058C00024B89B4A1288182A12D01344A3F1180056
:1058D0007F2840F307810C20973B93FBF0F200FBFD
:1058E000123303F17300C0B298F8001003F092FD78
:1058F0008D4B90491A78022A94BF013200221A7007
:105900001A7831F8120018287FF4FDAD0424022A19
:1059100002F1010294BFD2B2002231F8120018281D
:105920007FF4F0AD013CF2D1CAE5FAF7ABFEFFF728
:1059300001BB7F4B1A88182A13D03B681344A3F18C
:1059400018007F2840F3DA800C20973B93FBF0F29D
:1059500000FB123303F17300774BC0B2197803F0E8
:1059600059FD714B73491A78022A94BF0132002203
:105970001A701A7831F8120018287FF42EAD04241A
:10598000022A02F1010294BFD2B2002231F81200C1
:1059900018287FF421AD013CF2D11A70FDF7A1BDAA
:1059A000634B1B88182B12D099F800201344A3F1E5
:1059B00018007F2840F393800C20973B93FBF0F274
:1059C00000FB123303F17300C0B203F04BFD564AE3
:1059D000584B127833F81230182B7FF4B0ACFDF727
:1059E0001DBCFAF74FFEFFF7FFBBFAF74BFEFFF7C0
:1059F0004BBBFAF747FE44E5FAF744FE1DE44C4B77
:105A00001B88182B11D099F800201344A3F118001B
:105A10007F286ADD0C20973B93FBF0F200FB1233EA
:105A200003F17300C0B203F01DFD3F4A414B1278F1
:105A300033F81230182B7FF432AFFEF73AB83F4BF1
:105A40001B88182B11D099F800201344A3F11800DB
:105A50007F2850DD0C20973B93FBF0F200FB1233C4
:105A600003F17300C0B203F0FDFC2F4A344B1278EF
:105A700033F81230182B7FF412AFFEF71AB8FAF78A
:105A800001FE87E4FAF7FEFD00E4FAF7FBFDFFF7FD
:105A9000A5BAFAF7F7FD7EE5FAF7F4FDFFF71EBBAE
:105AA000FAF7F0FD57E5FAF7EDFDFFF741BBFAF71E
:105AB000E9FD3FE6234ADFF898B01288BBF80010F2
:105AC000033291427FF739AE10E6FAF7DBFDA6E527
:105AD000FAF7D8FD28E4FAF7D5FDFFF755BAFAF73B
:105AE000D1FD71E7FAF7CEFDFDE6FAF7CBFD99E7B8
:105AF000FAF7C8FDC8E6FAF7C5FDB3E7FAF7C2FD45
:105B00002AE7FAF7BFFD65E6FAF7BCFD3AE60E4B69
:105B100003930E4B0293FDF79FBE23601946FDF7DA
:105B2000D1BB00BF529CFF1FC29CFF1F589EFF1F8E
:105B30005C9CFF1FD09DFF1FC19CFF1F5A9CFF1F35
:105B4000C89DFF1F629CFF1F0D9CFF1FE29CFF1F53
:105B5000469CFF1F38B507F0C9FB0E4805F000FB57
:105B60000D4805F0FDFA0D4805F0FAFA00234FF054
:105B70007E5201210A48FAF779FC0A4B0A4A0B497E
:105B8000802400251C7118461D60BDE838400BF0CC
:105B900071B800BF449CFF1F789CFF1FD89CFF1F5B
:105BA000109EFF1F949EFF1F1C89FF1F29060000E7
:105BB00010B50446A4206368198803F087FDE368E4
:105BC000A6201988BDE8104003F080BD43682A2054
:105BD000198803F07BBD00BF10B50446222063681E
:105BE000198803F073FDE36824201988BDE810408C
:105BF00003F06CBD10B504460A206368198803F0F1
:105C000065FDE3680C201988BDE8104003F05EBD17
:105C100010B5044606206368198803F057FDE36851
:105C200008201988BDE8104003F050BD10B50446A7
:105C300002206368198803F049FDE368042019888D
:105C4000BDE8104003F042BD70B50E4C84B0122583
:105C50000422012306460390029320468DE8240087
:105C60001423102106F080FC0622092302930396D8
:105C70000195204600921423102106F075FC04B013
:105C800070BD00BF049FFF1FF8B5B04CB4F90030E1
:105C9000032B00F01281002B6AD0022B00F08A80C7
:105CA000052B00F0B580012B00F0DD80042B00D027
:105CB000F8BDA74FA74E00254FF4AF74E9B2A64830
:105CC00005F0B6FA57F8043BC3F5967300FB03F0F2
:105CD00086FB0023C017C0EB6310844205F1010569
:105CE000A8BF0446062DE9D19C4F9A4E0025E9B283
:105CF0009B4805F09DFA57F8043BC3F5967300FBEB
:105D000003F086FB0023C017C0EB6310844205F14B
:105D10000105A8BF04460C2DE9D1924F8D4E0025F8
:105D2000E9B2914805F084FA57F8043B894AC3F573
:105D3000967300FB03F086FB0013C017C0EB6310E3
:105D4000844205F10105A8BF04460C2DE8D1A4F159
:105D50001401312900F3A38040F26C723221834890
:105D6000834B01801A602A20BDE8F84003F0AEBCE6
:105D70000E2007F01FFA40F6FF71C8308842A8BF16
:105D8000084620EAE07000F5FA6283B28A42794D53
:105D9000794EA8BF0A460220194633802A8003F0B4
:105DA00095FC2988042003F091FCB4F90030022B03
:105DB0007FF476AF012008F041F90546002008F095
:105DC0003DF9A842B8BF284600F1C801B1F5FA7FF5
:105DD000C0F2B480B1F57A6FA8BF4FF47A6101F5D3
:105DE0004873B3F57A6FA8BF4FF47A639BB289B258
:105DF000624A634D11800A202B8003F067FC2988DA
:105E00000C2003F063FCB4F90030052B7FF44BAF9A
:105E10000F2008F013F9C0F53F630433B3F5AF6FFB
:105E2000C0F28980B3F5FA6FA8BF4FF4FA6399B254
:105E3000544BC0F54360B0F5AF6F198061DBB0F52E
:105E4000FA6FA8BF4FF4FA6083B24F4DA4202B80A5
:105E500003F03CFC2988A62003F038FCB4F900309C
:105E6000012B7FF423AF152007F0A4F900F59671FC
:105E7000B1F52F7F4DDB41F25C23994263DC434A4D
:105E800000F5617089B2B0F52F7F1180B8BF4FF473
:105E90002F7344DB8342A8BF03469BB23FE040F22E
:105EA0003A73A4F5B97403FB04F482FB0432E417DB
:105EB000A4EB621289B2323251E7102008F0BEF82A
:105EC000C830B0F5FA7F1FDBB0F57A6F0146A8BF86
:105ED0004FF47A6101F51673B3F57A6FA8BF4FF4EA
:105EE0007A639BB289B22A4A2A4D118022202B80E4
:105EF00003F0ECFB2988242003F0E8FBB4F9003020
:105F0000C9E64FF4AF63A0E740F24C434FF4FA7197
:105F1000E9E740F214534FF42F711C4A11801E4DD3
:105F200006202B8003F0D2FB2988082003F0CEFB4B
:105F3000B4F90030BAE64FF4AF6179E740F2145398
:105F40004FF4FA7154E71946E7E700BFDE9EFF1FE2
:105F5000488AFF1FB5814E1B449CFF1F188AFF1FF4
:105F6000789CFF1F2889FF1FD89CFF1F9C9EFF1F46
:105F7000008AFF1FA29EFF1FE09CFF1F489EFF1F7D
:105F8000589CFF1FE49CFF1F649EFF1F929CFF1FF5
:105F9000F49DFF1FF09DFF1F789EFF1F2DE9F0412C
:105FA000224D82B0012602B284B2009228460196A8
:105FB0007823192106F01EFA04F10C0212B28DE8C2
:105FC00044002846A7197823192104F1020806F095
:105FD00011FA3FB20FFA88F819233A4628461946B3
:105FE0000196CDF8008006F005FA78233A46284657
:105FF0001946CDF80080019604F10A070B3406F02B
:10600000F9F93FB224B278233A46284619468DE87A
:10601000500006F0EFF9192300943A4601962846FD
:10602000194606F0E7F902B0BDE8F081049FFF1FB2
:1060300030B583B000230C4605B2009326225B23C3
:106040001C210C4805F026FF294601232622094879
:1060500005F030FA002C24B205DB2146012326226C
:10606000044805F027FA044A044B15801C8003B04D
:1060700030BD00BF049FFF1F628AFF1F648AFF1F9D
:106080002DE9F041B44C237882B01BB1B34B4FF6ED
:10609000FF721A80B24BB3F90030CBB9B14AAF4BA3
:1060A0001068B3F9002080F30C005B2303FB00F0C1
:1060B00000131C30824244D04FF0FF31FFF7B8FF8D
:1060C000A94805F04BFF0023237002B0BDE8F08122
:1060D000012B1BD0022B53D0032B38D0042B00F004
:1060E0008C80052BEFD10F2007F0A8FFC0F53B6097
:1060F0000830B0F5AF6F41DBB0F5FA6FA8BF4FF4D1
:10610000FA60A0F5AF625B2398482EE0984B1A68BE
:10611000B2F52F7F32DB41F25C239342A8BF1346D6
:10612000A3F52F735B22934802FB03F380FB03204C
:10613000DB17C3EBA0201C30884BB3F9003083423F
:10614000BAD18D4BB3F900300133B5D1BBE78B4BDE
:106150001B68B3F5FA7F11DBB3F57A6FA8BF4FF474
:106160007A638748A3F5FA725B2303FB02F380FB93
:106170000320DB17C3EB20201C30DDE71C20DBE70E
:10618000804B1B68B3F5FA7F33DBB3F57A6FA8BF9A
:106190004FF47A63A3F5FA7279485B2303FB02F3A9
:1061A00080FB0320DB17C3EB20201C30764B1B68E1
:1061B000B3F5FA7F1FDBB3F57A6FA8BF4FF47A63AC
:1061C000A3F5FA726E495B2303FB02F381FB032103
:1061D000DB17C3EB21211C31604BB3F90030834244
:1061E0007FF46CAF644BB3F900308B427FF466AF41
:1061F00069E71C20DAE71C21EEE7252200258DE85F
:10620000240076231C215848604E614FDFF89881A6
:1062100006F0F0F816E0B0F5AF7FA8BF4FF4AF700E
:10622000323802FB00F088FB0031C017C0EB61116F
:106230001C3109B201231D4425224B4805F03AF9CF
:106240000C2D14D0E9B2534804F0F2FF56F8043B89
:10625000C3F5967300FB03F087FB0013C017C0EB78
:10626000631031284FF05B02D5DC1C21E2E72622C7
:1062700000258DE8240076231C213B48464E444FE0
:10628000DFF8248106F0B6F816E0B0F5AF7FA8BFBE
:106290004FF4AF70323802FB00F088FB0031C017BA
:1062A000C0EB61111C3109B201231D4426222E4886
:1062B00005F000F90C2D14D0E9B2384804F0B8FF0D
:1062C00056F8043BC3F5967300FB03F087FB0013FD
:1062D000C017C0EB631031284FF05B02D5DC1C21E6
:1062E000E2E7272200258DE8240076231C211E48A2
:1062F0002B4E274FDFF8B08006F07CF817E0B0F5A2
:10630000AF7FA8BF4FF4AF70323802FB00F088FBBC
:106310000031C017C0EB61111C3109B201231D44CB
:106320002722114805F0C6F8062D3FF4C9AEE9B2A0
:106330001C4804F07DFF56F8043BC3F5967300FB40
:1063400003F087FB0013C017C0EB631031284FF038
:106350005B02D4DC1C21E1E7D89EFF1F628AFF1F8D
:10636000DE9EFF1F4C9EFF1F049FFF1F37800B6D9B
:106370001C9CFF1FD3058541648AFF1F689CFF1F7B
:10638000011FB812749CFF1FC89EFF1F188AFF1FB1
:10639000B5814E1B789CFF1F2889FF1FD89CFF1FCB
:1063A000488AFF1F449CFF1F4B48371B2DE9F041D3
:1063B000044682B056482768E56805F0C3FC112002
:1063C000FFF7ECFD012619234FF028081946242277
:1063D0004F480196CDF8008006F00CF87823194656
:1063E00024224B480196CDF8008006F003F8314690
:1063F000474806F095FB02221921454806F08CFB20
:1064000038460BF0FDF939460246414806F01EFDBC
:106410003F4806F031FD142200213D4806F07CFB88
:1064200003223C493A4806F011FD394806F024FDA4
:1064300023220021364806F06FFB032236493448F8
:1064400006F004FD324806F017FD7DB12F20FFF75E
:10645000A5FD322200212E4806F05EFB03222F49C3
:106460002B4806F0F3FC2A4806F006FD01232C4ACF
:1064700018461370FFF7E8FB2189638962685B1A8D
:106480005C2B128832DD521A02EB4202C2EB42123E
:10649000013392FBF3F31B33224A1D48138001267C
:1064A0001A221BB28DE844001946142205F0A2FFFF
:1064B000CDB1218A638AE2685B1A5C2B12881DDCED
:1064C000511A5C2202FB01F292FBF3F31B33164AD2
:1064D0000F481380012438221BB28DE8140019469E
:1064E000322205F087FF02B0BDE8F081511A5C222C
:1064F00002FB01F292FBF3F31B33CDE7521A02EBDE
:106500004202C2EB4212334492FBF3F31B33DEE749
:10651000049FFF1F482701004C270100502701005E
:106520007D9FFF1FDA9EFF1FDC9EFF1F2DE9F041BC
:106530001E4682B014461AB3052A054600F09C8018
:10654000099B6F4A00EBC305012C6F892989686894
:10655000A7EB010382FB03E21A444FEAE373C3EBA8
:10656000A213028829D0042C69D0664A022CB2F901
:10657000001060D0082C65D0012002B0BDE8F08189
:10658000614D624A2B681268CB1A93420F466FD94D
:106590005F4A338811785F48012918BF01241470BD
:1065A000089A06321BB212B28DE814001946BDF9E2
:1065B000202005F01FFF2F60DEE79BB2D31A99421F
:1065C00003DC9F423946A8BF1946089A0180B6F9F4
:1065D0000030BDF920804F48971D4FF0000E3FB2AC
:1065E000194642460097CDF804E005F003FF2989DB
:1065F0006A896B68521A1B885C2AA3EB010377DD5A
:1066000003EB43030132C3EB431393FBF2F303F1B8
:106610001B0213B2012032801946424601900097B6
:106620003C4805F0E7FE3A4B00221A70354A022C2E
:10663000B2F900109ED14B1C1BB2138004E012FA79
:1066400083F3BCE700231380994295D0089AB6F9EA
:10665000003030480632012412B2009219460194EB
:10666000BDF9202005F0C6FE204602B0BDE8F0814D
:10667000204602B0BDE8F081072400265A232322D9
:106680008DE850001A21234805F082FE012121489F
:1066900006F046FA01211F4806F048FA2322352168
:1066A0001C4806F039FA22461B491A4806F0CEFB70
:1066B000184806F0E1FB174805F050FC4FF4FA606B
:1066C00007F0CAFAFFF7E0FA5A2323221A218DE8CD
:1066D0005000104805F05CFE0E4805F03FFC2846CF
:1066E000FFF764FE0D4B01221A70FFF7C9FC43E768
:1066F0005C2101FB03F393FBF2F21B3289E700BF3D
:10670000C94216B2E29EFF1F689FFF1F703601004C
:106710007D9FFF1F049FFF1F54270100D89EFF1F6E
:106720002DE9F04F5A4E5B4DB6F900704C7855F894
:10673000277085B08146984604B10C78DFF874A1C3
:106740001AB99AF80030002B39D0534D002338463F
:106750002B808AF80030FFF729FE504A504BB5F9DC
:106760000000012111704FF6FF721A8060B30128FA
:106770005ED0012032232246019000934946494BC6
:106780003846FFF7D3FE00240346B5F90020022A5D
:1067900039DD00222A80B6F900203D49002A3BDB82
:1067A000052AC4BF00220A80B8F1000F39D1002C9D
:1067B0000CBF18464FF0FF3005B0BDE8F08F364DE6
:1067C000B5F900000028D2D1DFF8ECB0364ADBF88A
:1067D00000301268C3EB0903934227D9334B1A7870
:1067E000012A18BF01201870FFF72EFA0123CBF8F9
:1067F0000090012C2AD0042C35D0022C3AD0082C41
:106800003ED00024C1E7C6D1FA68002AC1D0B6F94B
:1068100000201F49002AC3DA05220A80B8F1000FC0
:10682000C5D00393FFF72CFC039BC0E70346E0E7CA
:106830004FF0000E142322468DE8084049461C4BB9
:1068400038467446FFF772FE03469EE732888AF8A0
:106850000040013232807A6982B1002438460393C5
:106860009047039B91E732880121013A32808AF8F0
:106870000010F0E701222A8000248CE7144684E708
:106880007A69002129804FF0FF34002AE6D182E79F
:10689000DE9EFF1F688AFF1FE29EFF1FD89EFF1F1C
:1068A000628AFF1FDC9EFF1F703601007D9FFF1F65
:1068B000DA9EFF1FE09EFF1F689FFF1F01210D2032
:1068C00007F08EB900210D2007F08AB901460D208E
:1068D00007F086B908B50D2007F088F9B0FA80F105
:1068E00049090D20BDE8084007F07AB910B500212C
:1068F00044080D2007F074F9204607F0ADF90D208B
:10690000012107F06DF92046BDE8104007F0A4B959
:106910002D4A2E4B10881B68984210B549DA2C4A34
:106920001288141A9A42A8BF1A46B4F5157F36DAAF
:10693000121A40F2532303FB02F393FBF4F10531E7
:106940000A2006F0BDFF234B1978C9B3224B234917
:106950001B6840F2271283F3070302FB03F381FB5A
:1069600003211944DB17C3EBA1110531092006F0FF
:10697000A7FF1B4B1968F1B181F3070140F2271201
:10698000164802FB01F380FB03211944DB17C3EB1C
:10699000A11105311620BDE8104006F091BF131A71
:1069A0004FF41572611C02FB03F393FBF1F1053107
:1069B000C6E70021C4E71620BDE8104006F080BFFE
:1069C000092006F07DFFD4E7E09CFF1F109CFF1F0D
:1069D000A29EFF1F969CFF1F149CFF1F09040281AB
:1069E000609EFF1F7F2838B5A8BF7F200F4C4FF453
:1069F000167202FB00F284FB02311144D2170546E5
:106A0000C2EBA1110A2006F05BFF7F3D4FF49673A5
:106A100003FB05F384FB03211944DB17A3EBA1114E
:106A20000920BDE8384006F04BBF00BF09040281D1
:106A3000C368B3F9003030B583EAE374A4EBE374C0
:106A4000002BA0B218DB012300E0134603EB830206
:106A500052009442F9DA0A4D90FBF3F285FB03E40D
:106A600003FB1200DB173032D3EBA40380B201F832
:106A7000012BF1D10B7030BD2D230B700131E2E7FA
:106A80006766666638B5094D8224204602F038FEF6
:106A900035F8021B00B28842204601D002F016FEF3
:106AA0000234A4B28A2CF0D138BD00BFD09DFF1FA4
:106AB000024B8020198802F009BE00BF5C9CFF1FBA
:106AC00038B5094D7824204602F01AFE35F8021B2D
:106AD00000B28842204601D002F0F8FD0234A4B290
:106AE000802CF0D138BD00BFC89DFF1F024B76201F
:106AF000198802F0EBBD00BF5A9CFF1F38B5094D45
:106B00004624204602F0FCFD35F8021B00B2884204
:106B1000204601D002F0DAFD0234A4B24E2CF0D1AE
:106B200038BD00BF589EFF1F024B4420198802F059
:106B3000CDBD00BF529CFF1F024B4E20198802F0B2
:106B4000C5BD00BF709CFF1F024B9A20198802F040
:106B5000BDBD00BFC49CFF1F024B9820198802F0E6
:106B6000B5BD00BF629CFF1F024B8C20198802F04C
:106B7000ADBD00BFE69DFF1F024B9C20198802F0AF
:106B8000A5BD00BF469CFF1F024BA020198802F044
:106B90009DBD00BFCC9EFF1F024B9620198802F0BE
:106BA00095BD00BF3C9EFF1F024B8A20198802F052
:106BB0008DBD00BFFE9DFF1F08B5034B1020198837
:106BC00002F084FD012008BDFC9DFF1F024B102038
:106BD000198802F07BBD00BFFC9DFF1F024B2C20DB
:106BE000198802F073BD00BF429CFF1F024B1E209C
:106BF000198802F06BBD00BF609CFF1FC3680E20A8
:106C0000198802F063BD00BF024B2820198802F0EA
:106C10005DBD00BF549EFF1F024B6420198802F027
:106C200055BD00BF509EFF1F024B5A20198802F02D
:106C30004DBD00BF249CFF1F024B1620198802F097
:106C400045BD00BF2E9CFF1F024B2E20198802F06D
:106C50003DBD00BFCC9CFF1F024B3020198802F0C5
:106C600035BD00BFB09EFF1F024B9E20198802F069
:106C70002DBD00BFBC89FF1F024B1820198802F0F0
:106C800025BD00BFE69CFF1F024BA220198802F021
:106C90001DBD00BF809EFF1F024B1A20198802F005
:106CA00015BD00BF7A9CFF1F024B1C20198802F003
:106CB0000DBD00BF729CFF1F024B6620198802F0B9
:106CC00005BD00BF8A9EFF1F024B7220198802F08B
:106CD000FDBC00BFAC9EFF1F024B2020198802F0B4
:106CE000F5BC00BF889EFF1F024B3220198802F0BE
:106CF000EDBC00BF7A9EFF1F024B6820198802F08E
:106D0000E5BC00BFB09CFF1F024B6C20198802F04D
:106D1000DDBC00BF189CFF1F024B6E20198802F0DB
:106D2000D5BC00BFD69EFF1F024B5220198802F02F
:106D3000CDBC00BF5A89FF1F024B5020198802F0BA
:106D4000C5BC00BF108AFF1F024B5420198802F0F7
:106D5000BDBC00BF128AFF1F024B5C20198802F0E5
:106D6000B5BC00BF608AFF1F024B5E20198802F08D
:106D7000ADBC00BF5889FF1F024B6020198802F08C
:106D8000A5BC00BFEC9DFF1F024B5620198802F0E6
:106D90009DBC00BFBE9CFF1F244B1B880B2B43D800
:106DA000DFE803F00B10151A1F24292E33383D0697
:106DB000084604221E490AF0E1BD084604221D4986
:106DC0000AF0DCBD084604221B490AF0D7BD08467C
:106DD00004221A490AF0D2BD0846042218490AF0D2
:106DE000CDBD0846042217490AF0C8BD0846042252
:106DF00015490AF0C3BD0846042214490AF0BEBD75
:106E00000846042212490AF0B9BD08460422114975
:106E10000AF0B4BD084604220F490AF0AFBD084687
:106E200004220E490AF0AABD704700BF3C9EFF1F16
:106E300024330100D4300100882F0100703001009C
:106E40008C2F010030340100902F0100942F01009D
:106E50000C320100982F0100303301009C2F0100FB
:106E6000064B074A10B41C88064B0846002C14BF7A
:106E700011461946042210BC0AF080BD909CFF1FE9
:106E8000A02F0100A42F0100064B074A10B41C8854
:106E9000064B0846002C14BF11461946042210BCAC
:106EA0000AF06CBDCE9CFF1FA02F0100A42F010093
:106EB000064B074A10B41C88064B0846002C14BF2A
:106EC00011461946042210BC0AF058BDEE9DFF1F62
:106ED000A02F0100A42F0100064B074A10B41C8804
:106EE000064B0846002C14BF11461946042210BC5C
:106EF0000AF044BD3E9EFF1FA02F0100A42F0100F9
:106F0000064B074A10B41C88064B0846002C14BFD9
:106F100011461946042210BC0AF030BDD29CFF1F56
:106F2000A02F0100A42F01001B4B1B880A2B0AD89D
:106F3000DFE803F00A0E12161A1E22262A2E060079
:106F4000164B186808607047154B18680860704742
:106F5000144B186808607047134B18680860704736
:106F6000124B186808607047114B1868086070472A
:106F7000104B1868086070470F4B1868086070471E
:106F80000E4B1868086070470D4B18680860704712
:106F90000C4B186808607047FE9DFF1FCC2F010046
:106FA000A42F0100A82F0100AC2F0100B02F010079
:106FB000B42F0100B82F0100BC2F0100C02F010029
:106FC000C42F0100C82F0100F0B52B4E2B4FDFF866
:106FD000C4E005460FCE87B06C460FC496E80300A8
:106FE0003B68274A274F44F8040B40F6CC308342D5
:106FF000C8BF3A46BEF800602180012E1188927801
:10700000ADF80D108DF80F202AD032D340F6CA0209
:10701000022E18BF00229A4226DAA3F698031A49D4
:107020001A4AC3EB031381FB03011944DB17C3EBBB
:107030006123243382FB0321DA17C2EBA10202EBA6
:107040008201A3EB4103303330328DF813308DF8D9
:1070500011206946284616220AF090FC07B0F0BDC0
:1070600040F698029A42D8DB094B1868CDF8110017
:10707000EFE740F6FC02CEE7E02F0100449EFF1F41
:10708000D42F0100D02F01003B773B9867666666DE
:10709000D82F0100D89DFF1FF8B5174C174E227846
:1070A000174D33782F888E46003218BF01220146D3
:1070B0007046FFF735FB002398423370237015DBD1
:1070C00014BF012000202B889F420ED040F23A725C
:1070D000A3F5AF730B490C4C02FB03F381FB0312C6
:1070E000DB17A3EB621332332360F8BD074901229B
:1070F00018460A702270E6E7348BFF1FF59EFF1FCB
:107100009C9EFF1FB5814E1B008AFF1F7C9FFF1FA7
:10711000014B187802F072BA649FFF1F014B187878
:1071200002F086BADC90FF1F134BB3F9003030B584
:1071300083EAE374A4EBE374002BA0B218DB012311
:1071400000E0134603EB830252009442F9DA0B4D40
:1071500090FBF3F285FB03E403FB1200DB173032F4
:10716000D3EBA40380B201F8012BF1D10B7030BD39
:107170002D230B700131E2E7DC90FF1F6766666626
:10718000144BB3F9003070B583EAE375A5EBE375F2
:10719000002BACB21ADB012300E0034603EB8300B3
:1071A00040008542F9DA0C4E94FBF3F086FB03E5D0
:1071B00003FB1044DB173030D3EBA503A4B201F876
:1071C000010BF1D105480B70106070BD2D230B70C1
:1071D0000131E0E7249CFF1F67666666F82F010017
:1071E000134BB3F9003030B583EAE374A4EBE374D6
:1071F000002BA0B218DB012300E0134603EB83024F
:1072000052009442F9DA0B4D90FBF3F285FB03E454
:1072100003FB1200DB173032D3EBA40380B201F87A
:10722000012BF1D10B7030BD2D230B700131E2E742
:10723000BC89FF1F67666666134BB3F9003030B533
:1072400083EAE374A4EBE374002BA0B218DB012300
:1072500000E0134603EB830252009442F9DA0B4D2F
:1072600090FBF3F285FB03E403FB1200DB173032E3
:10727000D3EBA40380B201F8012BF1D10B7030BD28
:107280002D230B700131E2E7809EFF1F6766666663
:10729000134BB3F9003030B583EAE374A4EBE37425
:1072A000002BA0B218DB012300E0134603EB83029E
:1072B00052009442F9DA0B4D90FBF3F285FB03E4A4
:1072C00003FB1200DB173032D3EBA40380B201F8CA
:1072D000012BF1D10B7030BD2D230B700131E2E792
:1072E0005A89FF1F67666666134BB3F9003030B5E5
:1072F00083EAE374A4EBE374002BA0B218DB012350
:1073000000E0134603EB830252009442F9DA0B4D7E
:1073100090FBF3F285FB03E403FB1200DB17303232
:10732000D3EBA40380B201F8012BF1D10B7030BD77
:107330002D230B700131E2E7108AFF1F6766666636
:10734000134BB3F9003030B583EAE374A4EBE37474
:10735000002BA0B218DB012300E0134603EB8302ED
:1073600052009442F9DA0B4D90FBF3F285FB03E4F3
:1073700003FB1200DB173032D3EBA40380B201F819
:10738000012BF1D10B7030BD2D230B700131E2E7E1
:10739000128AFF1F67666666134BB3F9003030B57B
:1073A00083EAE374A4EBE374002BA0B218DB01239F
:1073B00000E0134603EB830252009442F9DA0B4DCE
:1073C00090FBF3F285FB03E403FB1200DB17303282
:1073D000D3EBA40380B201F8012BF1D10B7030BDC7
:1073E0002D230B700131E2E7608AFF1F6766666636
:1073F000134BB3F9003030B583EAE374A4EBE374C4
:10740000002BA0B218DB012300E0134603EB83023C
:1074100052009442F9DA0B4D90FBF3F285FB03E442
:1074200003FB1200DB173032D3EBA40380B201F868
:10743000012BF1D10B7030BD2D230B700131E2E730
:107440005889FF1F6766666608B5702002F058F914
:10745000044B1988884204D07020BDE8084002F02F
:1074600035B908BDD89DFF1F08B5742002F048F952
:10747000044B1988884204D07420BDE8084002F00B
:1074800025B908BD709EFF1F054B1B8808460422C6
:1074900013B904490AF072BA03490AF06FBA00BF7F
:1074A000709CFF1F00300100FC2F01000E4B1B8859
:1074B000032B17D8DFE803F0110C0702084604225B
:1074C0000A490AF05BBA0846042209490AF056BA8A
:1074D0000846042207490AF051BA08460422064920
:1074E0000AF04CBA704700BFE69DFF1F1030010044
:1074F0000C300100083001000430010010B40A4BC8
:107500000A4C0A4693E8030083B0238802AC04E9DE
:10751000030004EB8303104653F8081C052203B054
:1075200010BC0AF02BBA00BFEC270100509EFF1FD1
:1075300030B40A4B0A4D0C4693E8070084B02B8800
:1075400004AD05E9070005EB8303204653F80C1C46
:10755000042204B030BC0AF011BA00BFF4270100C5
:10756000D89DFF1FF0B40C4D0C4F0E460FCD8CB0C4
:1075700001AC0FC40FCD0FC495E807003B8884E829
:1075800007000CAA02EB8303304653F82C1C04229C
:107590000CB0F0BC0AF0F2B900280100349EFF1FC5
:1075A000F0B40B4D0B4F0E460FCD86B06C460FC49A
:1075B00095E803003B8884E8030006AA02EB8303F6
:1075C000304653F8181C042206B0F0BC0AF0D6B9B5
:1075D0003C280100E69CFF1FF0B40A4D0A4F0E46FE
:1075E0000FCD86B001AC0FC42A683B88226006AA82
:1075F00002EB8303304653F8141C0C2206B0F0BC97
:107600000AF0BCB954280100729CFF1FF0B40B4D66
:107610000B4F0E460FCD86B06C460FC495E80300A5
:107620003B8884E8030006AA02EB8303304653F844
:10763000181C042206B0F0BC0AF0A0B968280100AA
:10764000709EFF1F164B1B880BB31BB283EAE370BF
:10765000A0EBE370002B30B584B21DDB012300E00A
:10766000134603EB830252009042F9DA0D4894FB73
:10767000F3F280FB03E503FB1244DB173032D3EB5C
:10768000A503A4B201F8012BF1D10B7030BD08465F
:10769000042205490AF072B92D230B700131DDE790
:1076A000B09CFF1F6766666614300100F0B40A4D97
:1076B0000A4F0E460FCD86B001AC0FC42A683B8836
:1076C000226006AA02EB8303304653F8141C0422FE
:1076D00006B0F0BC0AF052B980280100189CFF1FC8
:1076E000054B1B881BB9054B186808607047084696
:1076F000042203490AF042B9C49CFF1FA42F0100D1
:10770000A02F0100164B1B880BB31BB230B583EAC8
:10771000E374A4EBE374002BA0B21CDB012300E0B4
:10772000134603EB830252009442F9DA0D4D90FBAD
:10773000F3F285FB03E403FB1200DB173032D3EBDB
:10774000A40380B201F8012BF1D10B7030BD064BC0
:107750001868086070472D230B700131DEE700BF09
:10776000609CFF1F67666666A42F0100164B1B888E
:107770000BB31BB230B583EAE374A4EBE374002BC4
:10778000A0B21CDB012300E0134603EB830252008E
:107790009442F9DA0D4D90FBF3F285FB03E403FB11
:1077A0001200DB173032D3EBA40380B201F8012BB7
:1077B000F1D10B7030BD064B1868086070472D235F
:1077C0000B700131DEE700BF429EFF1F67666666F1
:1077D000A42F0100164B1B880BB31BB230B583EAF4
:1077E000E374A4EBE374002BA0B21CDB012300E0E4
:1077F000134603EB830252009442F9DA0D4D90FBDD
:10780000F3F285FB03E403FB1200DB173032D3EB0A
:10781000A40380B201F8012BF1D10B7030BD064BEF
:107820001868086070472D230B700131DEE700BF38
:107830002E9CFF1F6766666618300100174B1B8879
:107840001BB31BB270B583EAE375A5EBE375002BA0
:10785000ACB21EDB012300E0034603EB83004000D3
:107860008542F9DA0E4E94FBF3F086FB03E503FB49
:107870001044DB173030D3EBA503A4B201F8010BA1
:10788000F1D108480B70106070BD074B1868086094
:1078900070472D230B700131DCE700BFCC9CFF1F2C
:1078A000676666661C300100A42F0100164B1B881A
:1078B0000BB31BB230B583EAE374A4EBE374002B83
:1078C000A0B21CDB012300E0134603EB830252004D
:1078D0009442F9DA0D4D90FBF3F285FB03E403FBD0
:1078E0001200DB173032D3EBA40380B201F8012B76
:1078F000F1D10B7030BD064B1868086070472D231E
:107900000B700131DEE700BFB09EFF1F6766666641
:10791000A42F0100164B1B880BB31BB230B583EAB2
:10792000E374A4EBE374002BA0B21CDB012300E0A2
:10793000134603EB830252009442F9DA0D4D90FB9B
:10794000F3F285FB03E403FB1200DB173032D3EBC9
:10795000A40380B201F8012BF1D10B7030BD064BAE
:107960001868086070472D230B700131DEE700BFF7
:107970008A9EFF1F67666666A42F0100164B1B8850
:107980000BB31BB230B583EAE374A4EBE374002BB2
:10799000A0B21CDB012300E0134603EB830252007C
:1079A0009442F9DA0D4D90FBF3F285FB03E403FBFF
:1079B0001200DB173032D3EBA40380B201F8012BA5
:1079C000F1D10B7030BD064B1868086070472D234D
:1079D0000B700131DEE700BFAC9EFF1F6766666675
:1079E000A42F0100174B1B881BB31BB270B583EA91
:1079F000E375A5EBE375002BACB21EDB012300E0C1
:107A0000034603EB830040008542F9DA0E4E94FBF7
:107A1000F3F086FB03E503FB1044DB173030D3EBB8
:107A2000A503A4B201F8010BF1D108480B70106056
:107A300070BD074B1868086070472D230B7001312B
:107A4000DCE700BF889EFF1F676666661C3001008A
:107A5000A42F0100074B1B88022B06D0012B0CBF63
:107A6000054B064B186808607047054B186808609E
:107A7000704700BFEC9DFF1F24300100283001003B
:107A800020300100054B1B881BB1054B18680860AE
:107A90007047044B18680860704700BFBE9CFF1F0A
:107AA000303001002C300100184B1A8852B3184AAC
:107AB000128830B50A80B3F90030002B83EAE374F2
:107AC000A4EBE374BCBF2D238B70A0B2ACBF02311A
:107AD0000331012300E0134603EB8302520094427A
:107AE000F9DA0C4D90FBF3F285FB03E403FB120083
:107AF000DB173032D3EBA40380B201F8012BF1D1B4
:107B00000B7030BD044B1868086070477A9CFF1FEB
:107B10003430010067666666A42F010070B53C4DE5
:107B20002B780646002B35D11C4673780BB92046BE
:107B300070BDFAF79BF9374A374B384812783178DD
:107B40001B78007802EB43034A1E03EB80030E2AE6
:107B5000EDD801A050F822F0C17B0000E37B0000CB
:107B60002F7B0000C17B00002F7B00002F7B0000DB
:107B70002F7B0000AF7B00002F7B00002F7B0000DD
:107B80002F7B00002F7B00002F7B00002F7B00004D
:107B9000AB7B0000AE21224803F084FE204804F0B5
:107BA000D1F800232B700124BFE706F067FBAF215B
:107BB0001B4803F077FE1B4A012313702B70B6E7B6
:107BC00083B91948038804294FF6FF7103F1FF3286
:107BD0000CBF01230B46134403F07F0301330380E2
:107BE0000FE073B1013B114A32F813304BB10E4E26
:107BF0000F481049104A33800123002606700B708D
:107C00001370084A0221012311702B70204670BDA9
:107C1000348BFF1F8D9EFF1F8E9EFF1F8F9EFF1FA9
:107C2000049FFF1F7C9FFF1F0C9EFF1FB89DFF1F1F
:107C3000A89CFF1F319CFF1F7F9FFF1F10B5064BA5
:107C4000064C1A882046012101F02EFD2188422091
:107C5000BDE8104001F03ABD909CFF1F509CFF1FF3
:107C600010B5064B064C1A882046022101F01CFD77
:107C700021884220BDE8104001F028BDCE9CFF1FA6
:107C8000509CFF1F10B5064B064C1A882046042155
:107C900001F00AFD21884220BDE8104001F016BD28
:107CA000EE9DFF1F509CFF1F10B5064B064C1A8817
:107CB0002046002101F0F8FC21884220BDE8104058
:107CC00001F004BD3E9EFF1F509CFF1F08B512200F
:107CD00001F016FD054B1988884206D0122001F0EC
:107CE000F5FCBDE8084001F009BC08BD349EFF1F4B
:107CF00008B5582001F004FD054B1988884206D0CC
:107D0000582001F0E3FCBDE8084001F0F7BB08BDD6
:107D1000429EFF1F08B5142001F0F2FC054B1988A4
:107D2000884206D0142001F0D1FCBDE8084001F0E3
:107D3000E5BB08BDD29CFF1FF0B480EAE075A5EB5F
:107D4000E0750028ACB21FDB1DBF2B230B704E1C4F
:107D50000E46012300E0134603EB830252009542D6
:107D6000F9DA0B4F94FBF3F287FB030503FB124494
:107D7000DB173032D3EBA503A4B206F8012BF1D107
:107D800033700846F0BC70472D230B704E1CE0E7A3
:107D900067666666084B188828B10D2807D00D382D
:107DA00000B2FFF7C9BF054A106808607047044A6F
:107DB00010680860704700BFD69EFF1FA42F010007
:107DC00038300100174B18880C2813D0192815D00B
:107DD0001A2817D01B2819D01C281BD01D281DD0ED
:107DE0001E2803D00C3800B2FFF7A6BF0E4A106859
:107DF000086070470D4A1068086070470C4A1068A8
:107E0000086070470B4A1068086070470A4A10689B
:107E100008607047094A106808607047084A10688F
:107E2000086070477A9EFF1F543001003C3001000B
:107E30004030010044300100483001004C30010066
:107E400050300100034B1888A0EB8000400000B2C6
:107E5000FFF772BF649FFF1F024B1888033800B200
:107E6000FFF76ABF549EFF1F024B18880C3800B200
:107E7000FFF762BF2A9CFF1F024B1888183800B218
:107E8000FFF75ABF5C9CFF1F024B1888183800B2DE
:107E9000FFF752BF5A9CFF1F024B1888183800B2D8
:107EA000FFF74ABF529CFF1FC3681888183800B2FA
:107EB000FFF742BF054B1B881BB9054B18680860CC
:107EC000704708460422034909F058BDCC9EFF1FA5
:107ED000A42F0100A02F0100054B1B881BB9054BE7
:107EE00018680860704708460422034909F046BD37
:107EF000629CFF1FA42F0100A02F010030B5134C7E
:107F000085B001252B463C2202212046009503F036
:107F10003FFD204603F016FF00224021802320462B
:107F20000191009311460A4B029504F0B9FB2046DB
:107F300004F014F807480849084A002303608380C6
:107F40000B608B801360938005B030BD049FFF1FD2
:107F50000C2B0100E49EFF1FFC9EFF1F6C9FFF1F68
:107F600010B500EBC00000F10F02D2B293B284B0A2
:107F70009C1E981C3D2303918DE81900392102486D
:107F800004F0F2FA04B010BD049FFF1F014B012260
:107F90001A707047F59EFF1FF0B5694B694C6A4F28
:107FA0006A4E6B4D85B004228DE80C00029320468A
:107FB000684B4022802103F0F3FA2046664A674965
:107FC000674C08F057FE674A674B9761674FD76168
:107FD000674F9F61674FDF61674FB761674FF76119
:107FE000674FAF61674FEF61674FA7616748684FA1
:107FF000E761684F87616849684FC761684F8F6163
:10800000684A694FCF61694F9761694B694FD76182
:10801000694F9F61694E6A4FDF616A4F6A4DB76170
:108020006A4FF7616A4F6B4CAF616B4FEF616B4FFB
:108030006B48A7616B4FE7616B4F6C4987616C4F71
:10804000C7616C4F6C4A8F616C4FCF616C4F6D4B49
:1080500097616D4FD7616D4F6D4E9F616D4FDF61C1
:108060006D4FB7616D4D6E4FF7616E4FAF616E4CE6
:108070006E4FEF616E4FA7616E486F4FE7616F4FB4
:1080800087616F496F4FC7616F4F8F616F4A704F44
:10809000CF61704F9761704B704FD761704F9F6188
:1080A000704E714FDF61714FB761714D714FF76164
:1080B000714FAF61714C724FEF61724FA76172489F
:1080C000724FE761724F73498761734FC761734F96
:1080D000734A8F61734FCF61734F744B9761744FC5
:1080E000D761744F744E9F61744FDF61744F754D4B
:1080F000B761754FF761754F754CAF61754F764835
:108100007649EF61764F774DA761DFF808E2E561C8
:10811000754F764D764C774A774B8761C5618C6198
:10812000764E774F774D784CC1F81CE07748784908
:108130009761D5619C61D861B16005B0F0BD00BFA9
:1081400040420F00049FFF1F697E0000A48EFF1FA6
:108150009C8CFF1FF890FF1F1C89FF1FF9B50000C2
:10816000588FFF1FBC8DFF1F348FFF1FFD6B00005A
:10817000597E0000096C0000616E00003D7C00002B
:10818000896E0000617C0000B16E0000988DFF1FB9
:10819000857C0000FD740000088DFF1F196C000035
:1081A000D96E0000748DFF1FA97C0000457E000081
:1081B000508DFF1F1171000029710000108FFF1FEB
:1081C0001D71000031750000308CFF1F49740000E4
:1081D00065750000C48FFF1FCD7C00006D77000027
:1081E000E48CFF1FF17C000081710000EC8BFF1F0D
:1081F000296C0000016F00003090FF1F157D00000A
:10820000D5770000C08CFF1F396C00003D7800005E
:10821000E08DFF1F496C0000AD780000788CFF1FD7
:10822000596C0000E17100005C8BFF1F696C00005D
:10823000A1750000C88AFF1F796C00003972000028
:108240002C8DFF1F896C0000A97A0000EC8EFF1FA7
:10825000996C0000D9750000B890FF1FA96C000050
:1082600015790000808EFF1FB96C00007D79000039
:10827000808BFF1FC96C00000D760000E88FFF1F88
:1082800069740000E5790000C88EFF1FD96C0000FA
:10829000C57D0000A48BFF1FE96C0000457600003F
:1082A000388BFF1FF96C0000AD760000808AFF1F3D
:1082B000096D0000957D00008890FF1F196D00007A
:1082C00091720000548CFF1F296D0000E9720000BC
:1082D000108BFF1F396D0000C88BFF1F7C8FFF1FA5
:1082E00041730000496D000099730000596D000052
:1082F000F1730000EC8AFF1FA48AFF1FAC90FF1FE0
:10830000557A0000796D0000857A0000896D0000C3
:108310009D880000696D0000F0B5461C83B00D46D5
:108320000127032336B22AB2044631468DE888007D
:108330002448ADB204F0AEF80C23AA1C12B200938C
:108340000197052321B21F4804F0A4F81E4A1F4BD1
:1083500012881B68BA422AD023D3022A10D11C4C9F
:10836000A3F6CA0384FB03241C44DB17C3EB2414C9
:108370000A2CA8BF0A2424EAE474A2B223B202E0C1
:1083800000231A461C460D35AA1A012000930190BD
:1083900012B2314603230B4803F0FAFF204603B024
:1083A000F0BD0C4CA3F6FC0384FB0324DDE7084C72
:1083B000A3F6980384FB03241C44DB17C3EBE404FB
:1083C000D6E700BF049FFF1FD89DFF1F449EFF1FDD
:1083D000898888881F85EB512DE9F0438FB283B0DF
:1083E000DFF84C80BD1D461D2DB204B236B24FF0F1
:1083F00001090AB22346314640460095CDF8049063
:1084000003F0F8FF2A463346214640468DE8200215
:1084100003F0F0FF07F10C020095334612B221463B
:10842000CDF80490404603F0E5FF03B0BDE8F083CB
:10843000049FFF1F2DE9F043804685B0002956D1E7
:108440000121304804F06CFB2F4998F8062098F879
:10845000083011F80290994522DA4FEA89064D4614
:108460000C24D8F80C3027489B595F6822B20021B1
:1084700004F052FB384609F0C3F939460246214858
:1084800004F0E4FC1F4804F0F7FC98F808300135CC
:108490000934AB42A4B206F1040601DD422CE0D15E
:1084A000B9F1000F13D109F1060999450CDA3C2303
:1084B00001213B22039102930093019239233F2231
:1084C0003A21104804F050F805B0BDE8F0830F23BE
:1084D00001213B22039102930093019239230C2244
:1084E0003A21084804F040F898F80830DBE700210A
:1084F0003423009301913F230C22024803F048FFEC
:108500009EE700BF049FFF1FFC9EFF1F10B5104C8D
:108510000121204604F00AFB2046012104F000FB63
:1085200020463422552104F0F7FA20460222094958
:1085300004F08CFC20460522074904F087FC204605
:1085400004F09AFC2046BDE8104003F007BD00BFD0
:10855000049FFF1F583001005C30010070B50D46CC
:10856000064609F04DF900EB40008400002D36D09E
:10857000284609F045F900EB4000400023185B1045
:1085800003F16001091A282209B21748C3F16004F7
:1085900004F0C2FA0121144804F0C2FA284609F096
:1085A0002FF929460246104804F050FC0E4804F00A
:1085B00063FC02210C4804F0B3FA21B221220A48DC
:1085C00004F0AAFA304609F01BF931460246064883
:1085D00004F03CFC0448BDE8704004F04DBC64105D
:1085E000C4F16004E5E700BF049FFF1F184B70B59E
:1085F000B3F9003083EAE374A4EBE374002B82B098
:10860000A1B21EDB68466D46012300E0134603EB72
:10861000830252009442F9DA0E4E91FBF3F286FB8C
:1086200003E403FB1211DB173032D3EBA40389B24E
:1086300005F8012BF1D119462B70FFF78FFF02B01F
:1086400070BD2D238DF800300DF101056846DBE784
:10865000FC9DFF1F6766666610B50D4B1B5C51F8ED
:108660002340237884B013B1012004B010BD04AAC4
:1086700001A942F8103D2046A3699847A38A9B07A9
:10868000F2D401A80099FFF769FF012004B010BDE2
:10869000E49EFF1F2DE9F04F2F4DDFF8CCB0DFF83F
:1086A000C4A0DFF8C8900FCD91B003AC0FC40FCDBC
:1086B0000FC40FCD0FC42B6823600025A8462F469A
:1086C0002E4600E09846BAF8003024495BF8232093
:1086D00028461123F7F7E8FF00EBC00400EB840005
:1086E00089FB00340444C017C0EB6434C4F13C007F
:1086F000C6F13C0207F14101012600B208F1410335
:1087000000901BB2019612B209B2154803F072FE36
:1087100008EB060305F211153C2B2646ADB2474681
:10872000D0D134226B210E4804F0F6F900210C4818
:1087300004F0F6F90B4B1B8810AA02EB830353F8E5
:10874000344C204609F05CF802460548214611B039
:10875000BDE8F04F04F07ABB94280100AC21010081
:10876000049FFF1F429CFF1F102001000900028090
:1087700010B5424C424882B003F0E4FA2378C3B902
:1087800006213F4804F0CCF92378012B37D90A227F
:10879000022B11463A486BD004F0BEF93949032246
:1087A000374804F053FB364802B0BDE8104004F0EF
:1087B00063BB354B1A7801210523002A35D101917D
:1087C000009311462E4803F065FE304B1A78002ABC
:1087D00036D0052301220192009300220A21284865
:1087E00003F0D6FD2A4B1A78002A35D10121052342
:1087F000019100931421224803F04CFEC0E7254C60
:108800002388092B32D9632B8CBF0A211F210A220E
:108810001B4804F081F92188194804F07DFB1848B1
:1088200002B0BDE8104004F027BB00220191009384
:108830001146134803F0ACFD144B1A78002AC8D136
:1088400005230121019100930A210D4803F022FE26
:108850000F4B1A78002AC9D00122052301920093F8
:1088600000221421064803F093FD89E73021CEE76A
:1088700004F052F90322084992E700BF7F9FFF1FCF
:10888000049FFF1F683001008D9EFF1F8E9EFF1FFB
:108890008F9EFF1F0C9EFF1F64300100F8B56D4DC9
:1088A000287840B96C4B1B6899425CD36B4A012312
:1088B00013702B70F8BD0C4600266948664F03F014
:1088C00041FA04F6AC53324665483B6031212E70C4
:1088D00004F022F901216248624D04F027F9314683
:1088E0005F4804F01DF905225F495D4804F0AEFAC7
:1088F0005B4804F0C1FA0C221021594804F00CF92D
:108900000B225A49564804F0A1FA05225849544806
:1089100004F09CFA524804F0AFFA564B50481C68D9
:10892000A4F69803C3EB031385FB03251D44102114
:10893000DB172022C3EB652504F0EEF840F6CC33BC
:108940009C4205F124054FF022014FF004000BDC9E
:10895000FFF7E2FC484B1C88064674B3012C46D056
:10896000022C41D00120F8BDFFF736FD0922434912
:108970003B4804F06BFA2A221021394804F0CCF865
:108980003F4C374884FB0534EB17C3EBA404214666
:1089900004F0C2FA01223B49314804F057FA04EBD3
:1089A0008401A5EB41012E4804F0B6FA01223649B4
:1089B0002B4804F04BFA0120F8BD34491022284816
:1089C00004F044FA264804F057FA2A2210212448D9
:1089D00004F0A2F83146224804F09EFA07222C49FE
:1089E0001F4804F033FACBE70C222A49E7E70C22B0
:1089F00029491B4804F02AFA194804F03DFA2A22B2
:108A00001021174804F088F8314615481C4E04F030
:108A100083FA07221E49124804F018FA86FB05362D
:108A2000EB17C3EBA60631460D4804F075FA224653
:108A300014490B4804F00AFA06EB8601A5EB410144
:108A4000074804F069FA22460F49054804F0FEF988
:108A50002046F8BD348BFF1FEC9EFF1F7C9FFF1F3D
:108A6000049FFF1F3B773B986C300100743001007E
:108A70005C300100449EFF1FD89DFF1F8030010025
:108A800067666666FC3701006C3701008C300100B8
:108A9000A0300100B8300100A83001002DE9F041FC
:108AA000754C2278002A05460F4614BF4FF0010886
:108AB0004FF000084ED1714E3368CB1AB3F5FA6F00
:108AC00004D86B78A3B94046BDE8F0816C4B6D4883
:108AD0006D49DFF8D0E11A70012303700988237013
:108AE00026208EF8002000F0F1FD6B78002BEAD0F4
:108AF0003760F9F7BBF9654A654B66491278287803
:108B00001B78097802EB4303421E03EB81030E2A14
:108B1000D9D801A151F822F0098C0000D58B0000B2
:108B2000C78A0000098C0000C78A0000C78A0000BD
:108B3000C78A0000BD8B0000C78A00006F8B000051
:108B4000C78A0000C78A0000C78A0000C78A0000E1
:108B50006B8B0000AF215048484E02F0A3FEFFF798
:108B600007FE002337602370ABE705F087FB4A4818
:108B700003F0E8F80221484803F0D2FF0F22232136
:108B8000454803F0C9FF05224449434804F05EF913
:108B9000414804F071F91E2223213F4803F0BCFF35
:108BA00005223F493C4804F051F93B4804F064F980
:108BB000394803F0D3F900F0ADFC84E7394D2B7848
:108BC000012B50D9304B2620198800F07FFD00235F
:108BD0002B7078E7002B3FF476AF013B324A32F836
:108BE0001330002B3FF46FAF274C304825492D4AF6
:108BF00023804FF001080023037081F8008082F881
:108C00000080FFF7B5FD5EE793B1013B264A32F8DD
:108C1000131019B31C4B254D1A4C224A19800026FB
:108C2000012326202E702370137000F04FFD15E0F5
:108C3000154C1E4922880B7004284FF6FF7002F174
:108C4000FF310CBF012202460A440E4E154D02F0C0
:108C50007F0201320121228031702B70FFF788FDE5
:108C60004FF001082FE70649064A0123002008704B
:108C700013702370A6E700BF348BFF1F789FFF1F80
:108C80007C9FFF1F319CFF1F0C9EFF1F8D9EFF1FAF
:108C90008E9EFF1F8F9EFF1F049FFF1FC830010085
:108CA000D03001007F9FFF1FB89DFF1FA89CFF1FB2
:108CB0002DE9F04F05468BB00F46AD480121164611
:108CC00003F034FFAA8812F0010440F0B080DFF80E
:108CD000CC8298F80030002B7DD1AB79A54AD15CCD
:108CE000A1B9DFF8BCA279781AF8039041B33978BA
:108CF0000139072900F2B780DFE811F0F1005401D3
:108D0000B5006C01B500B500B500E9007C78002C19
:108D100000F0CA800139EC68387854F82170FC689A
:108D2000411EB4F80080072900F2A780DFE811F0A7
:108D300074015901A5006C01A500A500A5009F00C4
:108D4000DFF854A2DAF80020B21AB2F5967F75D98E
:108D5000894A107801281ABF012010701170874AC3
:108D600018BF0146D05CC0EB0900C0B2FFF7F8F8AD
:108D70000124CAF80060AB889B0770D57B78002B74
:108D80006DD0F9F773F87E4B7E4A7F481B781278D6
:108D900039780078022515FB02330A2903EB80039A
:108DA00000F04E810C295AD1002B58D003F1190044
:108DB000764E774A013B0021400080B226F813101E
:108DC0000123157088F8003000F080FC714B0322FD
:108DD00020461A702FE0664802F0B4FF0121644873
:108DE00003F09EFE62482246214603F095FEAB88C2
:108DF000580725D42C68204608F002FD214602467B
:108E00005B4804F023F85A4804F036F8092201239D
:108E10008DE80C0000217F23554803F0EBFA002178
:108E20002846FFF707FB002388F8003055E7AB68BA
:108E30003146384698470BB0BDE8F08F0846FAE750
:108E40002B6804A8984704A808F0DAFC04A9024695
:108E5000474803F0FBFF464804F00EF8D6E72046EB
:108E60000BB0BDE8F08F00240AF8039083E70021DF
:108E7000D1543846FB699847FC68A4F80080002765
:108E800025223C238DE8840041211822384803F034
:108E90007FFAE968A879FFF7DFFB374A3E4B177086
:108EA0001E600BB0BDE8F08F3B490A68B21AB2F5FC
:108EB000967FD4D9304F0E603E78012E00F0B480FA
:108EC000E968184601233B70FFF7C6FBB3E7304A59
:108ED000E9791170012288F800200024C4E72A7A79
:108EE000013A4A45BFDD09F10104E4B2A145BAD017
:108EF000224E16F803B0CBEB0900C0B20021FFF7F9
:108F00002FF82B7A052BD9461BD9CBEB0402042A68
:108F100040F3AE80A4F1040BBBF1000FC0F2B080AF
:108F2000063B5B45A8BF5B465FFA83F9AA79134805
:108F3000B15C994205D000F8029001212846FFF764
:108F400079FAC9EB0400C0B201210B4EFFF708F813
:108F500000213423019100930548317040230B22F6
:108F60003F21A14603F014FA0124AB797CE700BF4E
:108F7000049FFF1F6C9FFF1F7D9FFF1FFC9EFF1F15
:108F80008D9EFF1F8E9EFF1F8F9EFF1FB89DFF1F90
:108F90007C9FFF1F7F9FFF1F689FFF1F348BFF1F5A
:108FA000E49EFF1F0FFA89F1E868604C50F82160D9
:108FB0002168049134785E4904980860002C71D0CF
:108FC000012C7FF450AF5B4A317A88F80040117071
:108FD000002449E7B9F1000F50D009F1FF34E4B2A1
:108FE00084E7B98A01F0040189B200293FF440AF57
:108FF0003B6A03929847039A00283FF43DAFAB7950
:10900000FC680021D15438E77B8A43453CD908F1FC
:1090100001081FFA88F830E73B8A43453BD208F144
:10902000FF381FFA88F828E725238DE81800424802
:109030003C703C231822412103F0AAF93046FAE69D
:10904000002B3FF40CAF3D4A3D4E1188394A03F1E5
:109050001900013B400080B226F81310012388F864
:109060000030157000F032FB364B20461D70E2E6F2
:10907000002A3FF755AF04F1FF3B4DE74C46F3E6BE
:109080004FF000094B4651E7BB8ADA077FF5F5AE92
:10909000B7F81080F1E6BB8AD9077FF5EEAEB7F8D6
:1090A0001280EAE62849C85CC0EB090009F1010E0C
:1090B000C0B201214FF0340B02F803E0FEF750FF7D
:1090C000B6681D48019440230B223F210124CDF8AE
:1090D00000B003F05DF940230B223F211648CDF884
:1090E00000B0019403F0D6F92146134803F018FDAF
:1090F000304608F085FBA0EB800000F15F0109B26B
:109100000F220D4803F008FD304608F079FB314688
:109110000246094803F09AFE074803F0ADFEE968ED
:10912000A879FFF799FAAB799EE600BFBC9FFF1FB5
:10913000689FFF1F7C9FFF1F049FFF1F0C9EFF1F48
:10914000B89DFF1F7F9FFF1FFC9EFF1F2DE9F0476B
:10915000DFF808926D4B99F800601B68DFF800A2F9
:1091600082B0003601934FF0030018BF0126019F23
:109170009AF8008004F03AFD0546042004F036FD1C
:109180000446052004F032FD800040EA4404062035
:1091900004F02CFD2C4364B25D4944EAC0000A7817
:1091A00080F00F03DBB29A425A4A3CD0176000228B
:1091B00059480B7003788DF800808DF8012053B367
:1091C000564A12684EF66021BA1A8A4219D8022B02
:1091D00059D0012B5FD0062B48D0032B63D0042B32
:1091E00069D0052B77D0072B7DD0082B00F083802A
:1091F000092B68D016B14A4802F0B0FE02B0BDE8B3
:10920000F087484A484C0023012123700370136003
:10921000938089F800103A4669464448FFF748FDB4
:109220003043C6B2E6E71268BA1A1E2A6BD99AF81A
:109230000020934222D0394C3D488AF80030012B5F
:10924000276082EA030207609846B1D0042BAFD1B1
:1092500037480068381AB0F5C87FA9D9354C20685E
:10926000381A3228A4D927601A46A1E73A46694637
:109270003148FFF71DFD3043C6B2BBE7012B4FF06D
:109280000002E3D1E4E73A4669462C48FFF710FDB7
:109290003043C6B2AEE73A4669462948FFF708FDB3
:1092A0003043C6B2A6E73A4669462648FFF700FDB6
:1092B0003043C6B29EE73A4669462348FFF7F8FCBA
:1092C0003043C6B296E73A4669462048FFF7F0FCBD
:1092D0003043C6B28EE73A4669461D48FFF7E8FCC0
:1092E0003043C6B286E73A4669461A48FFF7E0FCC3
:1092F0003043C6B27EE73A4669461748FFF7D8FCC6
:109300003043C6B276E7002252E700BFBC9FFF1F82
:10931000809FFF1FF09EFF1F7C9FFF1F749FFF1FFA
:10932000049FFF1F6C9FFF1F7E9FFF1FDC2A010011
:10933000849FFF1FF89EFF1F0C2F0100342A01009D
:1093400038290100D4280100BC3601002829010079
:1093500090290100182A0100AC90FF1F348BFF1FD9
:10936000F49EFF1F28B11028044BA8BF10201860DE
:109370007047024B01201860704700BF889FFF1F95
:1093800038B50F4D2B78013B01381B02C4B203F4F2
:109390007063200443F4404343F00C0300F4FE00E8
:1093A000184305F08BFD2868013860F03F00C0B21B
:1093B00004F0B2FD2046BDE8384004F0ADBD00BF6A
:1093C000889FFF1F70B5124D2B78013B1B0203F4E1
:1093D0007063064643F430430806320400F0FE4052
:1093E00043F00B03034302F4FE0018430C4605F060
:1093F00065FD2868013860F04F00C0B204F08CFDB4
:10940000304604F089FD2046BDE8704004F084BD7C
:10941000889FFF1F70B5124D2B78013B1B0203F490
:109420007063064643F410430806320400F0FE4021
:1094300043F00903034302F4FE0018430C4605F011
:109440003DFD2868013860F06F00C0B204F064FD93
:10945000304604F061FD2046BDE8704004F05CBD7C
:10946000889FFF1F38B5104D2B78013B1B0203F47A
:109470007063044643F41043000443F0090300F40E
:10948000FE00184305F01AFD2868013860F06F00EF
:10949000C0B204F041FD204604F03EFD0020BDE8CE
:1094A000384004F039BD00BF889FFF1F38B50E4D0E
:1094B0002B78013B1B0203F47063044643F45043D2
:1094C000000443F00D0300F4FE00184305F0F6FC21
:1094D0002868013860F02F00C0B204F01DFD20465E
:1094E000BDE8384004F018BD889FFF1F08B5002074
:1094F00005F0AEFD0028FAD108BD00BF08B5642113
:109500000720FFF75FFF7F210B20BDE80840FFF732
:1095100059BF00BF10B500217B20FFF753FF002487
:10952000E0B2FFF79FFF0134022004F095FB802C8E
:10953000F6D110BD10B504464FF4406004F09CFC19
:1095400004F0F4FC2CB1102C044BA8BF10241C60B8
:1095500010BD024B01241C6010BD00BF889FFF1F7F
:1095600010B5044641F0E00004F0D6FC04F07F00A2
:1095700004F0D2FCC4F3C610BDE8104004F0CCBC2B
:1095800038B5134D2B78044641F6FF72A0F5005014
:10959000824203F1FF33A8BF02461B0202F50052CC
:1095A00003F47063100443F4604343F00E0300F4CB
:1095B000FE005204184302F0FE42104305F07EFC08
:1095C000296801392046C9B2BDE83840FFF7C8BF55
:1095D000889FFF1F38B504460D46F02004F09CFC20
:1095E00035B1254414F8010B04F096FCAC42F9D1D6
:1095F000F720BDE8384004F08FBC00BF00B50B4B2E
:1096000083B00246998818680090032AADF80410C8
:1096100002D903B05DF804FB684606218DF80520E9
:10962000FFF7D8FF03B05DF804FB00BF2C37010043
:1096300000B50B4B024683B0186899880090131F41
:109640004C2BADF8041002D903B05DF804FB68465A
:1096500006218DF80520FFF7BDFF03B05DF804FB80
:1096600034370100030203F4FE43C0F3C61018436D
:10967000704700BF03784078DB0103F47E5300F0AD
:109680007F001843704700BF82B002AA114642F81B
:10969000040D002012F8013B03F07F03914243EADE
:1096A0000020F7D102B07047003210B403884FF0A9
:1096B000010404FA01F418BF012202FA01F123EABD
:1096C00004020A43028010BC704700BF70B5CEB2DE
:1096D0000C46054603F052FE864203D0314628462A
:1096E00003F066FE0135284603F048FE240A844252
:1096F00005D021462846BDE8704003F059BE70BD34
:1097000038B5054603F03AFE4FF0000460F3070455
:10971000681C03F033FE60F30F24A0B238BD00BF15
:10972000F8B504460020FFF7EBFF002C00F0698538
:109730004FF4AF610220FFF7C9FF4FF47A610420B4
:10974000FFF7C4FF4FF496610620FFF7BFFF4FF409
:10975000FA610820FFF7BAFF4FF4FA610A20FFF719
:10976000B5FF40F6B8310C20FFF7B0FF4FF42F6182
:109770002220FFF7ABFF40F6AC512420FFF7A6FFF5
:109780007D212A20FFF7A2FF0C210E20FFF79EFF6C
:1097900001211020FFF79AFF02211220FFF796FF08
:1097A00000211420FFF792FF00211620FFF78EFF03
:1097B00002211820FFF78AFF01211A20FFF786FFF8
:1097C00001211C20FFF782FF04211E20FFF77EFFEE
:1097D00014212020FFF77AFF01212620FFF776FFD2
:1097E00003212820FFF772FF04212C20FFF76EFFD2
:1097F00014212E20FFF76AFF00213020FFF766FFBB
:109800000C213220FFF762FF00213420FFF75EFFBA
:1098100000213620FFF75AFF00213820FFF756FFBE
:1098200000213A20FFF752FF00213C20FFF74EFFB6
:1098300000213E20FFF74AFF00214020FFF746FFAE
:1098400000214220FFF742FF1F214420FFF73EFF87
:1098500013214620FFF73AFF0E214820FFF736FF7D
:1098600011214A20FFF732FF0A214C20FFF72EFF7B
:1098700000214E20FFF72AFF06215020FFF726FF88
:1098800002215220FFF722FF0C215420FFF71EFF78
:1098900000215620FFF71AFF00215820FFF716FF7E
:1098A00001215A20FFF712FF08215C20FFF70EFF6D
:1098B0000A215E20FFF70AFF00216020FFF706FF64
:1098C00004216220FFF702FF01216420FFF7FEFE62
:1098D00000216620FFF7FAFE0B216820FFF7F6FE55
:1098E0007F216A20FFF7F2FE00216C20FFF7EEFED9
:1098F00000216E20FFF7EAFE00217020FFF7E6FE50
:1099000000217220FFF7E2FE00217420FFF7DEFE47
:109910001F217620FFF7DAFE13217820FFF7D6FE0D
:109920000E217A20FFF7D2FE11217C20FFF7CEFE18
:109930000A217E20FFF7CAFE1F218020FFF7C6FE06
:1099400013218220FFF7C2FE0E218420FFF7BEFE06
:1099500011218620FFF7BAFE0A218820FFF7B6FE04
:1099600000218A20FFF7B2FE00218C20FFF7AEFE17
:1099700000219620FFF7AAFE00219820FFF7A6FEFF
:1099800000219A20FFF7A2FE05219C20FFF79EFEF2
:1099900006219E20FFF79AFE0021A020FFF796FEE9
:1099A0007F21A220FFF792FE40F2A461A420FFF7DE
:1099B0008DFE4FF4E161A620FFF788FE0021A8206C
:1099C000FFF784FE0021AA20FFF780FE2921002056
:1099D000FFF77CFE0220FFF793FEB0F5805F0346A1
:1099E00080F0AC85D24A04201380FFF789FEB0F5E1
:1099F000805F034680F09985CE4A06201380FFF7EA
:109A00007FFEA0F52F739BB2B3F57A6F024606D99D
:109A100040F628210620FFF759FE40F62822C64BC3
:109A200008201A80FFF76CFEA0F52F739BB2B3F5E8
:109A30007A6F024606D940F6E4410820FFF746FE59
:109A400040F6E442BD4B0A201A80FFF759FEA0F50C
:109A5000FA739BB240F6AC518B42024606D94FF4E2
:109A6000FA610A20FFF732FE4FF4FA62B44B0C2081
:109A70001A80FFF745FEA0F5FA739BB240F6AC5191
:109A80008B42024606D940F6B8310C20FFF71EFE85
:109A900040F6B832AB4B0E201A80FFF731FE182883
:109AA000034600F23B85A84A10201380FFF728FEEA
:109AB000431E9BB20F2B024604D901211020FFF751
:109AC00005FE0122A14B12201A80FFF719FE0A2879
:109AD000034600F205859E4A14201380FFF710FE0E
:109AE0000128034604D900211420FFF7EFFD0023CD
:109AF000984A16201380FFF703FE7F28034600F2E2
:109B0000E884954A18201380FFF7FAFD05280346DC
:109B100000F2D884914A1A201380FFF7F1FD0C2837
:109B2000034600F2C8848E4A1C201380FFF7E8FD2C
:109B30000428034600F2B8848A4A1E201380FFF7E7
:109B4000DFFD0928034600F2A884874A20201380FD
:109B5000FFF7D6FD4628034600F29884834A222068
:109B60001380FFF7CDFDA0F5FA739BB240F6AC5120
:109B70008B42024606D94FF42F612220FFF7A6FD43
:109B80004FF42F627A4B24201A80FFF7B9FDA0F51D
:109B9000FA739BB240F6AC54A342024604D9214664
:109BA0002420FFF793FD2246724B26201A80FFF7F0
:109BB000A7FD7F28034600F262846F4A28201380A5
:109BC000FFF79EFD0628034600F252846B4A2A20C6
:109BD0001380FFF795FDA0F132039BB2B3F5967F9A
:109BE000024604D97D212A20FFF770FD7D22644BB7
:109BF0002C201A80FFF784FD0C28034600F23184E4
:109C0000604A2E201380FFF77BFD1E28034600F2DA
:109C100021845D4A30201380FFF772FD0928034636
:109C200000F21184594A32201380FFF769FD1E2883
:109C3000034600F20184564A34201380FFF760FD8A
:109C40007F28034600F2F283524C36202380FFF730
:109C500057FD7F28034600F2E38338206380FFF737
:109C60004FFD7F28034600F2D5833A20A380FFF7FB
:109C700047FD7F28034600F2C7833C20E380FFF7BF
:109C80003FFD7F28034600F2B9833E202381FFF782
:109C900037FD7F28034600F2AB8340206381FFF746
:109CA0002FFD7F28034600F29D834220A381FFF70A
:109CB00027FD394D28804420FFF722FD3028034638
:109CC00000F28A83354A46201380FFF719FD3028B9
:109CD000034600F27B83324C48202380FFF710FDBF
:109CE0003028034600F26C834A206380FFF708FDAA
:109CF0003028034600F25E834C20A380FFF700FD6E
:109D00003028034600F250834E20E380FFF7F8FC32
:109D10000128034604D900214E20FFF7D7FC002379
:109D2000204A50201380FFF7EBFC431E3CE000BFAD
:109D3000E09CFF1FA29EFF1F929CFF1F789EFF1FAB
:109D4000489EFF1F589CFF1F2A9CFF1FFC9DFF1F62
:109D5000349EFF1FD29CFF1F2E9CFF1FE69CFF1FFF
:109D60007A9CFF1F729CFF1F609CFF1F889EFF1F35
:109D7000F49DFF1FF09DFF1F0C9EFF1F549EFF1FB1
:109D80009C9EFF1F429CFF1FCC9CFF1FB09EFF1F8D
:109D90007A9EFF1FB89DFF1F509CFF1F529CFF1F04
:109DA000589EFF1F709CFF1F9BB20B2B024604D9CD
:109DB00006215020FFF78AFC0622CF4B52201A8042
:109DC000FFF79EFC0428034600F2E882CB4A5420A9
:109DD0001380FFF795FC431E9BB21D2B024604D94E
:109DE0000C215420FFF772FC0C22C54B56201A8020
:109DF000FFF786FC0128034604D900215620FFF70F
:109E000065FC0023BF4A58201380FFF779FC7F28A8
:109E1000034600F2BD82BC4A5A201380FFF770FC53
:109E2000431E9BB2092B024604D901215A20FFF799
:109E30004DFC0122B54B5C201A80FFF761FC431EEC
:109E40009BB2102B024604D908215C20FFF73EFC90
:109E50000822AF4B5E201A80FFF752FC431E9BB2D4
:109E60001D2B024604D90A215E20FFF72FFC0A228F
:109E7000A84B60201A80FFF743FC0228034600F23B
:109E80008182A54A64201380FFF73AFC012803462B
:109E900004D901216420FFF719FC01239F4A6220A5
:109EA0001380FFF72DFCC31E9BB2012B024604D981
:109EB00004216220FFF70AFC0422994B66201A80D5
:109EC000FFF71EFC7F28034600F25682954A682061
:109ED0001380FFF715FC7F28034600F24782924A61
:109EE0006A201380FFF70CFC7F28034600F23882BB
:109EF0008E4A6C201380FFF703FC0428034600F20F
:109F000029828B4A6E201380FFF7FAFB192803463B
:109F100000F21A82874A70201380FFF7F1FB0228B3
:109F2000034600F20B82844A72201380FFF7E8FB9D
:109F30000628034600F2FC81804A74201380FFF754
:109F4000DFFB0528034600F2ED817D4A8A2013805D
:109F5000FFF7D6FB0A28034600F2DE81794A8C20FF
:109F60001380FFF7CDFB0428034600F2CF81764A29
:109F700098201380FFF7C4FB0128034604D9002171
:109F80009820FFF7A3FB0023704A9A201380FFF765
:109F9000B7FB0128034604D900219A20FFF796FB5E
:109FA00000236B4A96201380FFF7AAFB0B28034679
:109FB00000F2A681674A9C201380FFF7A1FB831E55
:109FC0009BB2032B024604D905219C20FFF77EFBA0
:109FD0000522614B76201A80FFF792FB302803465A
:109FE00000F288815D4A78201380FFF789FB3028D2
:109FF000034600F279815A4C7A202380FFF780FBD8
:10A000003028034600F26A817C206380FFF778FBEA
:10A010003028034600F25C817E20A380FFF770FBAE
:10A020003028034600F24E818020E380FFF768FB72
:10A030003028034600F240814A4A82201380FFF70D
:10A040005FFB3028034600F23181474C8420238097
:10A05000FFF756FB3028034600F2228186206380FA
:10A06000FFF74EFB3028034600F214818820A380BE
:10A07000FFF746FB3028034600F20681A020E3806C
:10A08000FFF73EFB0128034604D90021A020FFF77B
:10A090001DFB0023354A9E201380FFF731FBC31EB2
:10A0A0009BB20C2B024604D906219E20FFF70EFB23
:10A0B00006222F4BA2201A80FFF722FB431E9BB2E1
:10A0C0007E2B024604D97F21A220FFF7FFFA7F22D0
:10A0D000284BA4201A80FFF713FBA0F5AF639BB2B7
:10A0E000B3F5167F024647D940F2A461A420FFF7DA
:10A0F000EDFA40F2A4623FE0108AFF1F5A89FF1F69
:10A10000128AFF1FBE9CFF1F429EFF1F249CFF1F41
:10A11000608AFF1F5889FF1FEC9DFF1F509EFF1F85
:10A12000809CFF1F8A9EFF1FB09CFF1F649CFF1F27
:10A13000189CFF1FD69EFF1FD89DFF1FAC9EFF1FC0
:10A14000709EFF1FFE9DFF1FE69DFF1F629CFF1F6D
:10A15000C49CFF1F3C9EFF1F469CFF1F5A9CFF1F75
:10A16000C89DFF1F5C9CFF1FD09DFF1FCC9EFF1F43
:10A17000BC89FF1F809EFF1FDD4BA6201A80FFF7C2
:10A18000BFFAA0F5AF639BB2B3F5167F024606D9BE
:10A190004FF4E161A620FFF799FA4FF4E162D54B45
:10A1A000A8201A80FFF7ACFA0628034666D8D24AE0
:10A1B000AA201380FFF7A4FA032859D82B88DFF8C8
:10A1C00058E3CE4FCE4ACF4DCF4ED04CD04903F0BE
:10A1D000010CAEF800C0C3F3400EA7F800E0C3F3D3
:10A1E00080071780C3F3C007CA4A2F70C3F3001754
:10A1F000C3F34015C3F38013378025800B80108094
:10A20000F8BD4FF6FF7398423FF492AA29283FF415
:10A21000E1AB17287FF68CAA19287FF6F5AA1B2830
:10A220007FF612AB1C283FF427AB1E287FF62CAB21
:10A230001F283FF431AB20283FF44AAB21283FF4DC
:10A2400053AB22283FF458AB23283FF461AB2428BA
:10A250003FF492AB25283FF497AB26283FF498AB08
:10A2600027283FF49DAB28287FF4B0ABFFF7A6BBAF
:10A27000AA200021FFF72AFA00209FE70021A8204A
:10A28000FFF724FA002392E70A218820FFF71EFA3D
:10A290000A23F3E611218620FFF718FA1123E5E6D9
:10A2A0000E218420FFF712FA0E23D7E61321822015
:10A2B000FFF70CFA1323C8E61F218020FFF706FAE8
:10A2C0001F23B9E60A217E20FFF700FA0A23ABE636
:10A2D00011217C20FFF7FAF911239DE60E217A2047
:10A2E000FFF7F4F90E238FE613217820FFF7EEF93C
:10A2F000132380E61F217620FFF7E8F91F2371E67C
:10A3000000219620FFF7E2F9002353E600218C207C
:10A31000FFF7DCF900232AE600218A20FFF7D6F9AF
:10A3200000231BE600217420FFF7D0F900230CE680
:10A3300000217220FFF7CAF90023FDE500217020FB
:10A34000FFF7C4F90023EEE500216E20FFF7BEF908
:10A350000023DFE500216C20FFF7B8F90023D0E5EA
:10A360007F216A20FFF7B2F97F23C1E50B21682026
:10A37000FFF7ACF90B23B2E500216620FFF7A6F941
:10A380000023A3E500216020FFF7A0F9002378E572
:10A3900000215820FFF79AF900233CE502215220C2
:10A3A000FFF794F9022311E50A214C20FFF78EF9FB
:10A3B0000A23A9E411214A20FFF788F911239BE41D
:10A3C0000E214820FFF782F90E238DE41321462049
:10A3D000FFF77CF913237EE41F214420FFF776F971
:10A3E0001F236FE400214020FFF770F900235CE495
:10A3F00000213E20FFF76AF900234EE400213C20B3
:10A40000FFF764F9002340E400213A20FFF75EF9EA
:10A41000002332E400213820FFF758F9002324E418
:10A4200000213620FFF752F9002316E400213420E2
:10A43000FFF74CF9002307E40C213220FFF746F91F
:10A440000C23FFF7F8BB00213020FFF73FF9002372
:10A45000FFF7E8BB14212E20FFF738F91423FFF78C
:10A46000D8BB04212C20FFF731F90423FFF7C8BB28
:10A4700003212820FFF72AF90323FFF7A7BB0121B7
:10A480002620FFF723F90123FFF797BB1421202093
:10A49000FFF71CF91423FFF761BB04211E20FFF70F
:10A4A00015F90423FFF751BB01211C20FFF70EF91A
:10A4B0000123FFF741BB01211A20FFF707F9012310
:10A4C000FFF731BB02211820FFF700F90223FFF745
:10A4D00021BB00211620FFF7F9F80023FFF711BB7D
:10A4E00002211220FFF7F2F80223FFF7F4BA00BFAF
:10A4F000E49CFF1F649EFF1F269CFF1F909CFF1F74
:10A50000CE9CFF1FDC9DFF1FEE9DFF1F529EFF1F75
:10A51000029EFF1F989CFF1F3E9EFF1F0C210E20D6
:10A52000FFF7D4F80C23FFF7BEBA4FF47A6104208A
:10A53000FFF7CCF84FF47A63FFF75EBA4FF4AF61E0
:10A540000220FFF7C3F84FF4AF63FFF74BBA00BF29
:10A55000F8B5BD2006F0C8FB204B214A054603CBC9
:10A560001368C5F803001A0CAC20C5F807102B803F
:10A57000AA70FFF777F82E46002426F80B0FA0B23A
:10A58000FFF7BEF8FFF76EF80234AC2C26F8020F86
:10A59000F5D16C1E05F1B8064FF0FF3014F8013FFD
:10A5A000082758400F4B40F300017A1E0B4012F071
:10A5B000FF0783EA5000F5D1B442EFD1C043FFF763
:10A5C00063F83A46C5F8B900BD21284604F0C4FC3A
:10A5D0002846BDE8F84006F08FBB00BF40370100B9
:10A5E0003C3701002083B8EDF0B50E4B0E4C05460C
:10A5F00093E8070085B024682E88AD7801AB83E826
:10A600000700270C184600220B21ADF804408DF8F6
:10A610000670ADF80C608DF80E5004F09DFC05B08E
:10A62000F0BD00BF4C3701003C370100F0B5124BC4
:10A63000124D1E68124F0FCD87B06C460FC495E8BF
:10A64000030044F8040B38683B79CDF80D00320C58
:10A65000292021808DF802208DF81130ADF800609E
:10A66000FFF700F80022ADF80B001221684604F055
:10A6700073FC07B0F0BD00BF3C3701005837010044
:10A680005C300100002004F0E3BC00BF02F02EBEED
:10A6900070B5124C82B0002540230646294620465C
:10A6A000009301958023202201F072FE202229468A
:10A6B000204602F031FA2046012102F037FA3046F6
:10A6C00007F09EF831460246204602F0BFFB2046C6
:10A6D00002B0BDE8704001F041BC00BF049FFF1F05
:10A6E000F0B5BC2983B075D90546441E00F1B80603
:10A6F0004FF0FF3014F8012F08275040404A40F334
:10A7000000017B1E0A4013F0FF0782EA5000F5D1DA
:10A71000B442EFD1C043FEF7B7FF0146D5F8B90008
:10A720000190019A914202D0B2F17F2F0BD105F135
:10A730000B00FEF79FFFAC280BD03248FFF7A8FFB5
:10A74000002003B0F0BD3048FFF7A2FF384603B049
:10A75000F0BD05F10D00FEF78DFF292840D1002442
:10A7600040F6AC5613E004281AD0062821D0082859
:10A770001FD00A2828D00C2822D1A1F5FA7292B253
:10A78000B24201D8FEF7A2FF0234AC2C0ED004F185
:10A790000D002844FEF76EFF022C0146A0B2E2D164
:10A7A000B1F5805FEED30234AC2CF0D1012003B0C0
:10A7B000F0BDA1F52F7292B2B2F57A6FE4D8E1E75D
:10A7C000222801D0242811D1A1F5FA7292B2B24206
:10A7D000DAD8D7E70D48FFF75BFF002003B0F0BDE4
:10A7E0000B48FFF755FF002003B0F0BD2A28C9D160
:10A7F000A1F1320292B2B2F5967FC5D8C2E700BF8E
:10A800002083B8ED9C3701008837010070370100C4
:10A81000B037010003290CD970B5461C82B005463B
:10A820000C46304603222A4907F058F810B102B00E
:10A8300070BD70470B2C05D905222649281D07F04D
:10A840004DF840B12448FFF723FF244802B0BDE88B
:10A850007040FFF7C9BE05F10901032201A807F006
:10A860008DF801A803221E4907F038F8D8B1032259
:10A870001C4901A807F032F808B301A803221A49BD
:10A8800007F02CF8B0B91948FFF702FFA11E89B2F2
:10A890003046FFF725FF0028C9D0154802B0BDE8B3
:10A8A0007040FFF7F5BE1348FFF7F2FEFFF750FECA
:10A8B0001148F3E71148FFF7EBFE1148C6E71148CE
:10A8C000FFF7E6FE02B0BDE87040FFF7AFBE00BF85
:10A8D0003C370100C8370100D0370100E4370100E0
:10A8E000E837010010380100283801002C38010039
:10A8F00040380100EC3701000038010054380100F5
:10A9000068380100143801002DE9F043174D2B6819
:10A9100083B081460F469046F3B1154E34880A192C
:10A9200092B218461146328006F05CFD28603A4625
:10A930004946204402F06CFDB8F1000F09D031887F
:10A940002868FFF767FF286806F0D6F900232B6018
:10A95000338003B0BDE8F083054E01930846318093
:10A9600006F0C2F9019B28601C46E0E7909FFF1F9C
:10A970008C9FFF1F10B51F4C4FF4FA70FBF7B6FF0A
:10A98000204601F0DFF900221146204602F0C4F80B
:10A990002046012102F0CAF82046002102F0C0F84A
:10A9A0000B221549204602F051FA204602F064FAC3
:10A9B0000F221249204602F049FA204602F05CFAC2
:10A9C0000F490722204602F041FA204602F054FACD
:10A9D000204601F0C3FA0B4B0B4A1A604FF4FA7091
:10A9E000FBF784FFFFF722FE0848BDE81040FFF7A1
:10A9F0004FBE00BF049FFF1F6C3801007838010074
:10AA00008838010048A1FF1F09A900009038010003
:10AA10000020704790F8392090F83800101A7047DD
:10AA200090F8383090F839209A4205D95A1C0344DE
:10AA300080F83820187E70474FF0FF30704700BF15
:10AA400090F8383090F839209A4286BF1B18187E4B
:10AA50004FF0FF30704700BF704700BF38B5054664
:10AA6000B0F85E0090B195F85D301446C3F1210254
:10AA700094420CD805F13B001844224602F0C8FC71
:10AA800095F85D30234485F85D30204638BD0120BF
:10AA900014462871EEE700BFB0F85E306BB190F855
:10AAA0005D30202B07D8C218013380F85D300120BB
:10AAB00082F83B107047012303710020704700BFEC
:10AAC0000023426980F8383080F8393080F85C30F3
:10AAD00080F85D3080F85E3080F85F3006CA30B4B0
:10AAE0000D68046943662A4383660A60A37042695D
:10AAF00090F861301649146813441D7A5B7B01EBB2
:10AB0000C5051B026D6803F4E06343F064032B602A
:10AB100090F8623013449D7CDB7D01EBC5011B0284
:10AB2000496803F4E06343F064030B6021685368F1
:10AB3000194205D0036927225A70036904229A71C9
:10AB4000036920225A71036980229A7030BC7047D1
:10AB5000C443010043690CCB12681A420CD0094B64
:10AB600099420AD9084B9942036994BF1A220D22CF
:10AB70005A70036904229A717047036927225A7038
:10AB8000F7E700BF7F1A06003F420F0010B50269C9
:10AB9000D378DBB2D90604463DD510215806D170D2
:10ABA00038D503F0040303F0FF02002B51D03D49D8
:10ABB000626E00230B7084F85D30002A5BD09047F2
:10ABC00094F85D30002B56D02369D0229A70236907
:10ABD00094F83B201A712369012284F85C20022238
:10ABE000DA7010BD304B84F860009C424AD02F4B85
:10ABF0009C4252D094F8391013791F29DBB207D840
:10AC00002848007820B16018013184F839100376A3
:10AC10000223D37010BD5906C3D4917801F01001FE
:10AC200001F0FF000029DDD013F001031ED194F8DC
:10AC30005C1094F85D00884281BF4B1C091984F8B0
:10AC40005C3091F83B3013712369D0229A702269ED
:10AC5000DEE7236984F83920C0229A702369114AFB
:10AC60001979012111700222DA7010BDC02393708E
:10AC700022691379CCE70122002384F85D2084F84F
:10AC80003B30A1E7626994F861300949134403221B
:10AC9000187A02F043FD2269ACE7626994F86130EA
:10ACA0000449F3E7949FFF1FF890FF1F6491FF1F73
:10ACB00015AD000021AD00000369DB7803F020032F
:10ACC00073B190F860300133DBB2012B80F8603053
:10ACD0001AD9426990F861301344187A02F09ABD8B
:10ACE00070B5426903F0FF0590F8613013440446E3
:10ACF000187A02F08FFDA36E5BB184F8385094F897
:10AD00003900BDE87040184790F85F30002BE0D064
:10AD1000704770BD0148FFF7CFBF00BFF890FF1F1D
:10AD20000148FFF7C9BF00BF6491FF1F2DE9F0473D
:10AD3000374FDFF8E0903B68026982B00646009327
:10AD4000DDF800800021A025D3789B065BD53B6809
:10AD50000193019BC8EB03030F2BF5D949B1102BCD
:10AD6000F2D000209070336980229A7002B0BDE862
:10AD7000F087726996F8613013440521187A02F061
:10AD800043FF726996F861301344012193F812A0D1
:10AD9000504602F039FF09240021504602F020FFFE
:10ADA0002B46013BFDD10121504602F019FF2B46F5
:10ADB000013BFDD1013CEFD1706996F8611001446F
:10ADC0004FF4A0720C7A4B7B09EBC4011B0249685B
:10ADD00003F4E06343F064030B6096F862300344CD
:10ADE000997CDB7D09EBC1011B02496803F4E06338
:10ADF00043F064030B60013AFDD13269D3789B06BE
:10AE00004FF00101A3D4012002B0BDE8F08700BFDC
:10AE1000BC9FFF1FC4430100F0B503691222DA7022
:10AE20000269937803F0200385B004460D46002B99
:10AE30005ED0B42393703C4922690B680093009E56
:10AE400005E00B680193019B9B1B042B42D8D37830
:10AE500003F0200303F0FF00002BF2D094F85D30E4
:10AE6000002B31D04FF0000E4FF0020C04EB0E031C
:10AE700093F83B3013710B680393039F206907E03D
:10AE80009B060DD50B680293029BDB1B052B28D874
:10AE9000C378DBB203F0020202F0FF06002AEFD013
:10AEA00080F803C02669F378DBB2DF0632462DD482
:10AEB0009F062BD5DB0731D40EF1010E94F85D30DF
:10AEC0005FFA8EFE7345D1D800201DBB002384F8A5
:10AED0005E3004E09070236980229A70042005B0EF
:10AEE000F0BD86702369802204209A7005B0F0BD01
:10AEF00003F0FF06FFF71AFF10B9042005B0F0BDFC
:10AF0000236984F85F60B0229A7094E78023B3705D
:10AF10000420DAE726698023B370D7E7BEF1000F7B
:10AF20000CBF02200320F6E7BC9FFF1F2DE9F04174
:10AF300006690025122780F8385080F83950F770DC
:10AF4000D0F810C09CF802E00EF0200E88B0044645
:10AF5000884615461E46BEF1000F49D0B4238CF832
:10AF60000230784B21691A680092DDF800E006E0B3
:10AF70001A6801920198CEEB0000042830D8C878F6
:10AF800000F0200000F0FF070028F1D04FEA48024F
:10AF900042F00102D2B20A711A680292DDF808E0AA
:10AFA000206906E01A6803920399CEEB0101052996
:10AFB0002AD8C17801F0020101F0FF070029F1D081
:10AFC0004FF0020C80F803C02269D17811F011070C
:10AFD00022D12DBB002E0CBFA0238023937003E051
:10AFE0008F70236980229A70384608B0BDE8F081DE
:10AFF0000EF0FF07FFF79AFE0028F5D0236984F8CA
:10B000005F70B0229A70ACE787702369802238465F
:10B010009A7008B0BDE8F081802393700027E3E7C1
:10B02000012D75D0A021917021690A79BE4667462D
:10B030004FF0A80C1A680492049805E01A6805926B
:10B04000059A121A052A4AD8CA7802F0020202F0BA
:10B05000FF08002AF2D0CF702169CA78D2B212F06C
:10B06000100F08465AD1920658D5013DEDB2012D78
:10B0700049D0BEF11F0F3BD90A79012DDAD11A68E8
:10B080000692069D05E01A680792079A521B052A48
:10B0900046D8C27802F0020202F0FF01002AF2D084
:10B0A0000223C3702269D378DBB2D9063AD49B0657
:10B0B00034D5B023BEF11F0F93703FD8226904EB43
:10B0C0000E0312791A760EF1010E5FFA8EFE16B19A
:10B0D000236980229A7084F839E0774684E781F802
:10B0E0000280236980229A70774684F839E07BE7F2
:10B0F00004EB0E0291F8048082F818800EF1010E24
:10B100005FFA8EFEB9E781F802C021690846B0E710
:10B11000A82191702069BE460279B0E7774663E7BF
:10B120008170DEE71021A023D170013BFDD122699F
:10B13000937803F0F7037746937055E723691B79FB
:10B14000C5E700BFBC9FFF1F0148FFF71FBD00BF41
:10B15000F890FF1F0148FFF719BD00BF6491FF1F62
:10B16000704700BF38B5144C037801225B000546D8
:10B17000204684F83B3084F85E2084F85D20FFF799
:10B180008BFC20460021FFF747FE0B4C297801235A
:10B1900020461A46FFF7CAFE0128F6D194F8383047
:10B1A00094F839209A4205D9E218013384F83830EE
:10B1B000107E38BDFF2038BDF890FF1F38B51B4CFE
:10B1C000037801225B000546204684F83B3084F872
:10B1D0005E2084F85D20FFF75FFC20460021FFF72A
:10B1E0001BFE124C2978204601230222FFF79EFE07
:10B1F0000228F6D194F8382094F839108A420FD2F8
:10B20000531CDBB2A018994284F83830007E0AD96A
:10B21000234402321B7E84F8382040EA032038BDE4
:10B220004FF6FF7038BD40F47F4038BDF890FF1FE7
:10B230000C2901D9002070470231490001F0FE01BC
:10B24000FFF7BCBF70B50C4C0378164601255B00B8
:10B25000204684F83B3084F85E5084F85D50FFF758
:10B260001BFC31462046FFF717FC29462046BDE867
:10B270007040FFF7D1BD00BFF890FF1FF8B505463D
:10B280000F461646412421463A462846FFF7DAFF84
:10B29000611C0234C9B232462846E4B2FFF7D2FF3D
:10B2A000592CF0D1F8BD00BF38B504460D463548DD
:10B2B000FFF706FC6322802120462570FFF7C2FFBE
:10B2C000012002F0C9FC204600225E21FFF7BAFFF0
:10B2D00020465D21FFF746FF242801D0002038BD1D
:10B2E000204606220C21FFF7C9FF204601222B2110
:10B2F000FFF7A8FF204601222C21FFF7A3FF2046DD
:10B300000E222D21FFF79EFF204600222E21FFF75F
:10B3100099FF204601222F21FFF794FF20460522A6
:10B320003021FFF78FFF204601223121FFF78AFFEE
:10B33000204600223221FFF785FF204600223321DC
:10B34000FFF780FF204600223421FFF77BFF2046D5
:10B3500000223521FFF776FF204600225B21FFF710
:10B3600071FF204610225C21FFF76CFF204620224F
:10B370005D21FFF767FF20468F225E21FFF762FF06
:10B38000012038BDF890FF1F10B4047F4160022CEB
:10B39000C26002D010BC01F0D7BB836810BC184754
:10B3A00090E80C00F0B41C6859682568164F174ED9
:10B3B00029432160164D17491760D6601561116049
:10B3C000417A154A5C180A3194F8244053F8215008
:10B3D00002EBC40149680D60017A5C1803EB81013E
:10B3E000247ECD6902EBC40149680D60817A58184A
:10B3F00003EB810390F83000596B02EBC002F0BC04
:10B4000053681960704700BF01401F0001100038E9
:10B410000110007800001F80C4430100704700BF86
:10B42000F0B50C1EBDF8146034DBB0F906701919C4
:10B43000B942C4BF3B1B1BB2002BA6461CDD002A31
:10B440001146B8BFD11D02F00705CC10826A012059
:10B4500007FB04E1A840012E0A44C0B21ED00CD361
:10B46000022E09D1013B12FA83F3013A12F8011FAF
:10B4700041409A421170F9D1F0BDC043013B12FA2C
:10B4800083F3C0B2013A12F8011F014093421170D8
:10B49000F9D1F0BD23441BB20024C6E7013B12FAE8
:10B4A00083F3013A12F8011F01439A421170F9D156
:10B4B000F0BD00BFF8B50D1E0EDB14461F46064654
:10B4C00001F03AFBA84207DD002C05DB304601F015
:10B4D00037FBA04201DCF8BDF8BD304601F02AFB85
:10B4E000022853D003284BD0012806D16540F388A9
:10B4F0006C406540013B5D1B2DB2012F03D02AD368
:10B50000022F14D0F8BD002C2246B6F90630B06ADE
:10B51000B8BFE21D42F3CF0202FB035504F007045B
:10B52000435D012101FA04F41C434455F8BD002C8D
:10B530002246B6F90630B06AB8BFE21D42F3CF0228
:10B5400002FB035504F00704435D012101FA04F4F2
:10B550005C404455F8BD002C2246B6F90630B06A6E
:10B56000B8BFE21D42F3CF0202FB035504F007040B
:10B57000435D012101FA04F423EA04044455F8BDB3
:10B580003389013B591B25460CB2B6E7F188328955
:10B590000139013A4D1B141B2DB224B2ADE700BF97
:10B5A0002DE9F041079E9DF91880089D04461F462D
:10B5B00000F0C0FF0D4B0E480E4984F83380FF2287
:10B5C000002F08BF1F4684F82F20002384F8302066
:10B5D00084F8312084F832202060A665E565676232
:10B5E00061652362A3622046BDE8F081F890FF1FE9
:10B5F0001C3901000110013810B50446806A034B64
:10B60000236008B105F078FB204610BD1C3901000D
:10B61000F8B5436ADBB190F82C200125AA4083F8E5
:10B620003B2083F85E5083F85D500446406A03680F
:10B630000E461B6800219847606A036831461B6804
:10B6400098472946606ABDE8F840FFF7E5BBC26B42
:10B65000C56C1368046A23EA050313604CB12268C1
:10B660004FF00043D3625163D36A002BFCDA936B33
:10B67000F8BD836B466B0825802410E03768426C68
:10B680003A4332601F68826C3A431A601A68876CCA
:10B69000013D22EA07024FEA54041A6007D0214212
:10B6A000ECD13268476C22EA07023260EAE7F8BD63
:10B6B00070B50446406A0D4600282BD0A16DFFF7F7
:10B6C00049FA002D20460CBFA621A721FFF7A0FFB5
:10B6D000606A20B1E16DBDE87040FFF73BBA216CB4
:10B6E000226D0868236A02430A6093B1DA7A82B154
:10B6F000D00703D5224A99691160DA7A910703D5F8
:10B70000204AD9691160DA7A520702D51E4A1B6AAB
:10B71000136070BD236A002B2BD0D97A626DE1B122
:10B7200072B6D97ACE0706D51848D968066831406E
:10B7300099610160D97A880706D5154819690668A4
:10B740003140D9610160D97A4E0705D51148596950
:10B75000066831401962016062B61B68D96891427F
:10B7600007D00D4818600D49DA6042F0804018613A
:10B770001960226C216D136823EA01031360A0E7AE
:10B7800000E100E004E100E008E100E080E100E029
:10B7900084E100E088E100E001403F0000003F80DC
:10B7A000436A2DE9F04105460E469046002B3ED0F7
:10B7B00090F82C100124A14083F83B1083F85E40E0
:10B7C00083F85D40406A036800211B6808F1FF3779
:10B7D0009847FFB2B8F1000F23D03744A046013E8E
:10B7E000686A16F8011F03681B6898470134B7425E
:10B7F000E4B216D0202CF3D10121686AFFF70CFBCC
:10B8000095F82C206B6A520083F83B2083F85E8009
:10B8100083F85D80686A036800211B6898470124EB
:10B82000DEE7686A0121BDE8F041FFF7F5BAC26BB7
:10B83000C16C136823EA010306EB080413604FF0A0
:10B840000048A6420ED02B6A16F801EB63B11A68C5
:10B85000C2F82C80C2F834E0D36A002BFCDAA6428E
:10B86000936BF0D1BDE8F081AB6BD5F834C0082004
:10B870008021DCF800206F6C1EEA010F14BF3A43F0
:10B88000BA43CCF800201A68AF6C3A431A601A68C1
:10B89000AF6C013822EA07024FEA51011A60E8D181
:10B8A000CFE700BF70B50446406A0D46002828D097
:10B8B000A16DFFF74FF920462946FFF7A9FE606A00
:10B8C00020B1E16DBDE87040FFF744B9216C226DF5
:10B8D0000868236A02430A6093B1DA7A82B1D0071A
:10B8E00003D5234A99691160DA7A910703D5214A71
:10B8F000D9691160DA7A520702D51F4A1B6A1360B0
:10B9000070BD236A002B2BD0D97A626DE1B172B67B
:10B91000D97ACE0706D51948D968066831409961A9
:10B920000160D97A880706D515481969066831403B
:10B93000D9610160D97A4E0705D512485969066860
:10B9400031401962016062B61B68D968914207D024
:10B950000D4818600D49DA6042F0804018611960A6
:10B96000226C216D136823EA01031360A3E700BF73
:10B9700000E100E004E100E008E100E080E100E037
:10B9800084E100E088E100E001403F0000003F80EA
:10B990002DE9F041044686B0806A9DF830801E464D
:10B9A0000F461546B4F90830002800F04281DA1D30
:10B9B00048BF03F10E02B4F90630D21003FB02F2C5
:10B9C000002105F0BDFCB4F90820202A00F3928084
:10B9D000B4F90610A34B0120203A733902EBD2725E
:10B9E00001EBD1714FF0200E029073208DE80140E1
:10B9F00042F34F0241F34F01204600F051FE606ACE
:10BA000084F82D70002800F04D81002D40F08A80D0
:10BA1000B4F90830202B14BF3D253C2584F82C5068
:10BA2000B8F1000F40F0858006B394F93300002888
:10BA300018DBC0B2012102F0E7F8012194F83300CD
:10BA400002F0CEF8012002F007F9002194F833004B
:10BA500002F0C6F80A2002F0FFF8012194F8330042
:10BA600002F0BEF8606A002800F08280A16DFFF746
:10BA700071F804227C492046FFF792FE217A0139B1
:10BA8000C9B22046FFF7C4FD784904222046FFF7DB
:10BA900087FE94F92D30012B14BF1421102120466C
:10BAA000FFF7B6FD042272492046FFF779FEB4F98C
:10BAB0000630802B00F09280602B00F0A680D92108
:10BAC0002046FFF7A5FD94F92D30012B14BFF1217D
:10BAD00022212046FFF79CFD204606226549FFF7FC
:10BAE0005FFE606A50B3E16DFFF734F8012006B0E5
:10BAF000BDE8F081B4F906105F4B0120403A52399D
:10BB00004FF0400E029002EBD272522001EBD17145
:10BB10008DE8014042F34F0241F34F01204600F00F
:10BB2000BFFD6CE76DB284F82C50B8F1000F3FF404
:10BB30007BAFFEF7C5FF002E94D076E7216C226D17
:10BB40000868236A02430A6073B1DA7A62B1D007E7
:10BB500003D54A4A99691160DA7A91077CD4520771
:10BB600002D5474A1B6A1360012006B0BDE8F08188
:10BB7000236A002B2BD0D97A626DE1B172B6D97AE3
:10BB8000CF0706D53F48D96805682940996101600B
:10BB9000D97A8E0706D53C48196905682940D961CC
:10BBA0000160D97A4D0705D538485969056829409B
:10BBB0001962016062B61B68D968914207D03448A7
:10BBC00018603449DA6042F0804018611960226CD4
:10BBD000216D136823EA010313604AE7B4F90830C2
:10BBE000202B00F08680402B7FF469AF2A49204645
:10BBF0000322FFF7D5FD94F92D30012B14BFCF217F
:10BC00009F212046FFF704FD59E7B4F90830102BB7
:10BC10007FF455AF214920460322FFF7C1FD94F977
:10BC20002D30012B14BFAF2110212046FFF7F0FC6F
:10BC300045E7DA1D48BF03F10E02B4F90630D21011
:10BC400003FB02F21046059205F04EF8A0620028B0
:10BC50003FF44DAF059AB3E6114AD9691160DA7A1B
:10BC60007DE700BF74390100543B0100583B0100DF
:10BC70005C3B0100603B0100683B010000E100E02B
:10BC800008E100E080E100E084E100E088E100E01C
:10BC900001403F0000003F8070390100283E010054
:10BCA00004E100E0012194F83100244F01F0ACFFE1
:10BCB00094F83200012101F0A7FF94F9312094F9A2
:10BCC000323057F83220E26357F83330206A236469
:10BCD0000125E56425651A682A431A6078B1B8F130
:10BCE000000F3FF428AFFFF75BFB002E3FF4BAAE26
:10BCF0009BE6042212492046FFF752FDDFE6294663
:10BD000094F82F0001F080FF294694F8300001F0EC
:10BD10007BFF94F92F2094F9303057F8322062637A
:10BD200057F833306564A5641A68A36322F00102F2
:10BD30001A60002E3FF496AE77E600BFC4430100C0
:10BD40006C390100B0F90820D31D48BF02F10E0381
:10BD5000B0F90620806ADB1002FB03F2002105F037
:10BD6000EFBA00BFF0B50029BDF814502EDBB0F9D2
:10BD70000660B1422ADA002A59DBB0F9087014468D
:10BD80001C44BC42C4BFBB1A1BB2002B1EDDD2B286
:10BD9000D408D0F828E016FB041112F00702DBB239
:10BDA0000EEB010421D0C2F10807FAB2374F9342DB
:10BDB000BF5C0CD2C3EB020CFF2646FA0CF6012D39
:10BDC00007EA06073FD005D3022D36D0F0BD012D7E
:10BDD00039D030D21EF8016026EA07070EF801704C
:10BDE0009342F3D3B0F906100C449A1AD2B2072A40
:10BDF00010D9022D36D0002D14BFFF260026134681
:10BE00002670083BB0F90610DBB2072B0C44F7D8BC
:10BE100002F00702002AD9D01D4B012D9B5C1DD0DA
:10BE200017D3022DD2D1227853402370F0BD134492
:10BE30001BB20022A1E7022D25D11EF80160774038
:10BE40000EF80170CCE71EF8016037430EF8017060
:10BE5000C6E7227822EA03032370F0BD2278134359
:10BE60002370F0BD11462378DB4323700839B0F905
:10BE70000630C9B207291C44F5D812F00702A5D034
:10BE8000034B9B5CCFE73444AFE700BF0C390100A4
:10BE9000FC38010070B4C47DBDF80C50022C18D0E1
:10BEA000032C1FD0012C0BD0002A03DBB0F9084073
:10BEB000944201DC70BC7047039570BCFFF7B0BAC8
:10BEC000C4880395013CA41A0A4621B270BCFFF74E
:10BED00049BF0689C488013E641AB21AE41A12B234
:10BEE00021B2E1E704890395E41A641A114622B2EB
:10BEF00070BCFFF737BF00BF70B4C57DBDF80C60E4
:10BF0000022D1AD0032D12D0012D03D0039670BC40
:10BF1000FFF728BFC488E41AA41A0A4621B2002AEF
:10BF200003DBB0F90840944213DC70BC704704890D
:10BF3000013C641A114622B2F1E7C48805890396D0
:10BF4000013CAD1AED1A621A11B22AB270BCFFF7A9
:10BF500009BF039670BCFFF763BA00BF2DE9F84331
:10BF60000446406A002863D0A16DFEF7F3FD052268
:10BF700074492046FFF714FCA1790139C9B2204663
:10BF8000FFF746FBB4F90820E588A66AD31D48BF31
:10BF900002F10E03DB10626A15FB03F51FFA85F848
:10BFA000002A7BD094F82C300125AB4082F83B303E
:10BFB00082F85E5082F85D50606A036840211B6819
:10BFC00008F1FF379847BFB2B8F1000F23D03744CC
:10BFD000A846013E606A16F8011F03681B6898476F
:10BFE0000135B742EDB216D0202DF3D10121606AA0
:10BFF000FEF712FF94F82C20636A520083F83B206E
:10C0000083F85E8083F85D80606A036840211B6866
:10C0100098470125DEE70121606AFEF7FDFE606AB0
:10C02000002800F08D80E16DBDE8F843FEF792BD79
:10C03000236A002B2BD0D97A626DE1B172B6D97A1E
:10C04000CE0706D54048D968056829409961016046
:10C05000D97A8D0706D53D48196905682940D96107
:10C060000160D97A480705D53948596905682940DA
:10C070001962016062B61B68D968914207D03548E1
:10C0800018603549DA6042F0804018611960226C0E
:10C09000216D136823EA0103136068E7E26BE36C28
:10C0A0001168276A0B4306EB080913604FF0004E36
:10C0B0004E450DD016F801CB2FB33A68C2F82CE0EC
:10C0C000C2F834C0D36A002BFCDA4E45936BF1D131
:10C0D000226C236D11680B43136097B1FB7A83B117
:10C0E000D90703D51D4BBA691A60FB7A9A0703D5A5
:10C0F0001B4BFA691A60FB7A5B0702D5194B3A6A47
:10C100001A60BDE8F883A36BD4F83480082080213E
:10C11000D8F80020656C1CEA010F14BF2A43AA431B
:10C12000C8F800201A68A56C2A431A601A68A56C22
:10C13000013822EA05024FEA51011A60E8D1B7E757
:10C14000276AC5E70439010080E100E084E100E0EE
:10C1500088E100E001403F0000003F8000E100E096
:10C1600004E100E008E100E02DE9F04F85B09946D8
:10C17000BDF93870BDF83CA0BB1AC1EB090B002B10
:10C18000B8BF5B42BBF1000FB8BFCBF1000B5B4502
:10C190000D4616460093804648DC4D453A463346E8
:10C1A0004CDC194613460A46C5EB09019B1A89B2B5
:10C1B000002B0CB2B8BF5B4204EBD474BE42ACBFE0
:10C1C0004FF0FF3201224D45039102924FEA640481
:10C1D00029DC9BB201930DE0D8F80070BF69B84725
:10C1E000019BE41AA3B21CB20135002C2DB211DB65
:10C1F000A94518DB009B5B452A465346314640461D
:10C20000EADCD8F800205346976929463246404672
:10C21000B847E5E7029A1644039AA94502EB0304DE
:10C2200036B224B2E6DA05B0BDE8F08F4A462B46B6
:10C23000B94635464D4517461E46B2DD30462946BD
:10C240003E464D4607468946AEE700BF10B4046837
:10C250002469A44610BC604730B40468BDF8085097
:10C260000295A46BA44630BC604700BF30B404689C
:10C27000BDF808500295E46BA44630BC604700BF8F
:10C2800070B40468BDF90C60BDF8105003960495B5
:10C29000246CA44670BC6047704700BF10B582B0E4
:10C2A000B0F90C2001910168009200220C6CB0F9E9
:10C2B0000A301146A04702B010BD00BF704700BF52
:10C2C00001F003010129C17506D0032904D0C288F9
:10C2D00003894281838170470289C38842818381B7
:10C2E000704700BF2DE9F0410568134E6F6986B0B5
:10C2F000B7420446BDF8308010D1013B13441BB255
:10C300000093CDF804800B46AD6A2046A847236809
:10C31000DB6AB3420AD106B0BDE8F081059304920E
:10C320000391B84703A925680EC9E6E7204606B081
:10C33000BDE8F041184700BF99C200002DE9F04167
:10C340000568124E6F6986B0B7420446BDF830806A
:10C350000FD1013BCDF804800B4400921BB2AD6AB3
:10C360002046A8472368DB6AB3420AD106B0BDE87D
:10C37000F081059304920391B84703A925680EC97B
:10C38000E7E7204606B0BDE8F041184799C2000033
:10C390002DE9F04F0568DFF858B06F6985B05F454B
:10C3A0000646BDF93890BDF83CA00C46904615D124
:10C3B0001F19BC420CDACDF800A0214601342D6AC9
:10C3C0004B464246304624B2A847BC423568F2DBB1
:10C3D000EB6A5B4507D105B0BDE8F08F0393B84722
:10C3E0003568039BE4E7304605B0BDE8F04F1847D9
:10C3F00099C200002DE9F04387B099420546BDF986
:10C400003840BDF83C6025D0A24212D00768DFF862
:10C410008080D7F81490C14532D18DE8500028466D
:10C42000BC6AA0472B68DB6A434524D107B0BDE84E
:10C43000F083994202DD08461946034628680E96A5
:10C44000C46B01335B1A1BB22846A44607B0BDE893
:10C45000F0436047A24202DD134622461C4628688C
:10C460000E96631C846B9B1A1BB22846A44607B029
:10C47000BDE8F0436047284607B0BDE8F0431847E1
:10C48000059304920391C84703A92F680EC9C4E716
:10C4900099C200002DE9F04FD0F800E0DFF890904D
:10C4A000DEF814B083B0CB450446BDF93080BDF84A
:10C4B00034A00D4617461E4631D1CDF800A0DEF857
:10C4C00024B0294633463A462046D8472368CDF85B
:10C4D00000A008F1FF323A44D3F824B0294612B242
:10C4E00033462046D8472368CDF800A02946D3F824
:10C4F00020B03A4643462046D8472068CDF800A0F1
:10C50000711E29444346056A09B23A462046A847A7
:10C510002368DB6A4B4506D103B0BDE8F08FD847EE
:10C52000D4F800E0C9E7204603B0BDE8F04F184753
:10C5300099C20000F0B4002401264FF6FF75094FA0
:10C5400007600471C475C48104824476C461867531
:10C55000067685824582C180028141818281F0BC5C
:10C56000704700BF343E01002DE9F04F85B00668EA
:10C57000BDF84450BDF93880CDF8008004460195DF
:10C58000D6F848B00392BDF93C60BDF940708946C9
:10C590009A46D84723680195009742465146D3F8FA
:10C5A000488020463346C0472068039B0E930F9572
:10C5B000856C4B463A4631462046AC4605B0BDE850
:10C5C000F04F60472DE9F04F87B01746BDF9404066
:10C5D00000912546E91D059344BF2B4603F10E014A
:10C5E0000268BDF8486053690294C91003912B4951
:10C5F000BDF9444001968B42824645D1002C3CDD7A
:10C60000029B3C445E1EB6B24FF0000923B2049375
:10C6100001364D46029B002B28DD059B002403EBD1
:10C62000090806E0EDB22B0604F1010411D4A6427C
:10C630001CD0A1B211F0070F23B24FEA4505F1D18A
:10C64000002BB8BF0733DB10013418F803502B065A
:10C65000EDD5009BD2F818B019443A4609B2019BB7
:10C660005046D847A642DAF80020E2D1039B0137B2
:10C670009944049B3FB2BB42CCD1D36A074A934250
:10C6800006D107B0BDE8F08F9847DAF80020B5E78B
:10C69000504607B0BDE8F04F184700BF99C20000F0
:10C6A00070B4BDF90C60BDF91050BDF8144003968C
:10C6B0000495059470BCFFF785BF00BF2DE9F04FCE
:10C6C00093B090460591C1691090BDF87000079035
:10C6D000BDF874909DF878A00493002900F0CD80F7
:10C6E0000A7A0AC9894604998A1AD2B203EBC203AC
:10C6F000BAF1010FDA780B9293F905201E8893F8AE
:10C7000002B00F9293F9064079D913B2099323B27C
:10C710000C93109B1A68A94B1193194653698B42CD
:10C7200040F0A6800B9B002B55D01FFA88F3002108
:10C730000D93C8462344DDF8409006910E930F46B2
:10C740000C46BBF1000F3FD0BDF818100C9B0397AF
:10C750001FFA8AF0CB1813FB00F304900E980144E3
:10C760000D98034409B21BB20A910893002505E015
:10C770000135EBB264009B45E4B222D9039B2B4404
:10C78000590703D1731C18F806409EB22306EFD553
:10C79000099BBDF81000E91811FB00F10598BAF1EA
:10C7A000010F0FFA8AF301441CD0079801900093FF
:10C7B000D26909B217464846089AB847D9F8002006
:10C7C000D6E7039F5F44FFB2069B0B9901330693A4
:10C7D000DBB29942B5D8D36A119A934243D113B0D0
:10C7E000BDE8F08F0F9B191893690A9A29441F46D8
:10C7F00009B2079B4846B847D9F80020B8E700239C
:10C800000C93099385E70A9A0D9B0132013B52B2C2
:10C8100013F0FF030A920D936FD1DDF81890079B78
:10C82000DDF83C80DDF820A04B4517D0BAF1010FB0
:10C8300000F0C8800B9A109DCDF804900BEB8B0193
:10C840004FEACB030A4400931146DEF81C405346DE
:10C85000424609B22846A047D5F800E0DEF82C3061
:10C86000119A9342BBD0109813B0BDE8F04F18470F
:10C87000109D284698472A6854E7109A0598B2F9FF
:10C880000A308342ABDDB2F90C304345A7DD062305
:10C8900013FB0A03002BA2DD08EBCA03002B9EDD6D
:10C8A000537E2BB9049BAF2B02D90133DBB2049327
:10C8B000109BD3F800E0414B11931A46DEF8143078
:10C8C000934240F08E801FFA88F30E9308339BB298
:10C8D000BDF81420059305230D9300230A93CDF88A
:10C8E0003C800FFA8AF3DDF84080CDF818900B9267
:10C8F0001FFA8AFBCDF820A099460A9ABDF81000CD
:10C900000B9C0E9D0523194611FB00232C48114654
:10C91000C75C039702FB0B4214FA81F312B21BB2FD
:10C9200009920C932C462E461CE0089B0999012B7A
:10C930002AB24B4640462DD0079F0197CDF8009074
:10C94000DEF81CA0D047D8F800E0039B5B08013458
:10C950000393059BA4B25D445E44A342ADB2B6B25C
:10C960003FF451AF039BD807DFD4079B069A93424D
:10C97000EBD0089B012B16D0069B0193CDF80090BD
:10C98000DEF81CA009994B4632B24046D047D8F891
:10C9900000E0DAE7DEF818A0079B0C9922B2D04736
:10C9A000D8F800E0D1E7DEF818A00C99134640460D
:10C9B00022B2D047D8F800E0C7E700BF99C2000014
:10C9C000843E01000B99109DCDF800900531DEF8F2
:10C9D000204009B2424608232846A047D5F800E087
:10C9E0003CE7109C20469847D4F800E06BE700BF76
:10C9F000F0B5C36985B004462BB30A2968D00D2968
:10CA00004AD01A7A914247D3587A884244D35D6813
:10CA10008A1A05EBC205AA78002A50D0E8780028C7
:10CA20004DD0207E00283AD095F905E0B4F90E00EB
:10CA3000A67DB4F90A70724406FB0202BA4262DCB7
:10CA4000B4F9102030E00A2956D00D2924D0027EF6
:10CA5000002A4BD0B0F90E00A57DB4F90A60062279
:10CA600012FB0502B2423EDD228AE38102EBC502DF
:10CA700012B218462282A78A668A02950B468DE872
:10CA8000C00001462046FFF719FEA37DE28903EBB3
:10CA9000430302EB4303E381012005B0F0BDA67D13
:10CAA000B4F90E00B4F91020B4F814E0678A0296C5
:10CAB0000B468DE8804001462046FFF7FFFD2979AF
:10CAC000E389A27D012001FB0233E38105B0F0BDC3
:10CAD0000022C2819A7A817D038A01FB023303829C
:10CAE000012005B0F0BDB4F91020C4E7857DB4F98C
:10CAF0001020B0F90E00BEE7028A817DC38102EBEF
:10CB0000C1030382C8E70020E0819B7A228A03FBED
:10CB1000062212B22282C7E7C1810282704700BF9B
:10CB2000002908BF01218175704700BF81824182C1
:10CB3000704700BFC07D7047B0F90A00704700BF62
:10CB4000B0F90C00704700BF10B4EFF3108272B65A
:10CB5000437F33B9017F012907D003290FD0012377
:10CB6000437702B962B610BC7047124C2168A1B17C
:10CB7000114943610B68836108605861EFE70F4C0E
:10CB8000216881B10E4943610B6883610860586177
:10CB90000C4B4FF080511960E1E7074B4161816117
:10CBA00020601860DBE7064B4161816120601860FE
:10CBB000EEE700BFA89FFF1FA49FFF1F989FFF1FC6
:10CBC0009C9FFF1F04ED00E070B5EFF3108272B67A
:10CBD0000C4C206880B10C4E00254369236073B172
:10CBE0009D6102B962B6457783689847EFF310827A
:10CBF00072B620680028F0D102B962B670BD336009
:10CC0000EFE700BF989FFF1F9C9FFF1FFFF7DCBF50
:10CC1000184A30B41468002C27D0036821688B426E
:10CC20000ED2CB1A00218460C1602360E0601060E6
:10CC30000223037530BC704711688B42144608D339
:10CC4000A2685B1A0360002AF6D18260C460A0600B
:10CC5000EEE7D268C2608460E060C568CB1A022249
:10CC6000A8602360027530BC70478460C4601060A7
:10CC7000DEE700BFA09FFF1FF8B5224E34682CB33B
:10CC80002368002B3AD1204F1D4604E03468ECB1F4
:10CC90002368002B32D1A36803B1DD6020693360C3
:10CCA000036825751B68BB4221D1037F4560022BB9
:10CCB000C46020D0FFF748FF6368002BE6D02360F4
:10CCC0002046FFF7A5FF3468002CE1D1EFF3108375
:10CCD00072B60E4A00211068116003B962B628B11D
:10CCE0008468FFF795FF20460028F9D1F8BD224659
:10CCF00000219847E0E783689847DDE7013B236020
:10CD0000E4E700BFA09FFF1F89B30000B09FFF1F93
:10CD1000024A136801331360FFF7AEBFBC9FFF1FC9
:10CD2000704700BF0368F0B4FBB1002501249D608B
:10CD3000DC601B4C1A601C44241104F144056A1188
:10CD4000032692009E60174F0679174B47F8241070
:10CD500002F1604202F5614205F01F05012000FA70
:10CD600005F5E6541560F0BC7047104C236843F499
:10CD70000003236000BF0E4B0E4DA4F58734A4F5CD
:10CD80009E7401261E60234604609C68002CD0D04F
:10CD90001033AB420360F8D1002303601846E2E78A
:10CDA000008FFCBFD091FF1F44E400E03C800440B2
:10CDB00000700340407103400168A9B10B4BF0B40F
:10CDC0000B441B110A4E0B4F0B4D46F8237003F119
:10CDD000440202F01F0401235211A340002445F82D
:10CDE00022308C600460F0BC704700BF008FFCBF35
:10CDF000D091FF1F21CD000080E100E0024A034BEB
:10CE0000012111601B6818470C710340D091FF1F6E
:10CE1000024A034B012111605B6818471C710340F3
:10CE2000D091FF1F024A034B012111609B681847F4
:10CE30002C710340D091FF1F024A034B0121116066
:10CE4000DB6818473C710340D091FF1FF8B50E46D0
:10CE500071B17AB10746144600253B6816F8011BEC
:10CE60001B6838469847013C0544F6D12846F8BD72
:10CE70000846F8BD1046F8BD00B5064A036812889A
:10CE80005B6883B001A9ADF804200222984703B083
:10CE90005DF804FB84430100F0B507468BB0002A1F
:10CEA00033D0012A08BF0A2251B3212400E0F4B292
:10CEB000B1FBF2F502FB1511C8B2092900F13001EE
:10CEC00098BFC8B20AA988BF3730214488BFC0B212
:10CED00001F8240C661E2946002DE8D133B1013C2F
:10CEE000E4B20AAB23442D2203F8242C3B6801AAA8
:10CEF00011195B683846C4F1220298470BB0F0BDA7
:10CF000030228DF825202124E8E70368C9B21B6888
:10CF100098470BB0F0BD00BF0029BABF49422D238E
:10CF200000230A22FFF7B8BF374A384913681B06A7
:10CF3000FCD40B6813F08003F8D172B634490A7838
:10CF4000002A5FD0334A3448F0B4344C176806687E
:10CF50002568D4680C303E44143200681268304FA3
:10CF600035442C4420440244C2F34E022D4E2E4838
:10CF70002E4D2F4C42F400423A60376806682D6807
:10CF80002C4A24680C303E44006812682A4F35440D
:10CF90002C4420440244C2F34E02284E2848294D16
:10CFA000294C42F400423A60376806682D68274AE7
:10CFB00024680C303E4400681268254F35442C44E8
:10CFC00020440244C2F34E02224E2348234D244CF7
:10CFD00042F400423A60376806682D68214A2468A6
:10CFE0000C303E440068126835442C44204402440E
:10CFF000C2F34E021C4842F4004202600B7062B65B
:10D00000F0BC704762B6704724B0034024B00B40B8
:10D01000B59FFF1F38B003403CB0034040B0034011
:10D020002CB0034058B003405CB0034060B00340F4
:10D0300064B003406CB0034030B0034038B00B40E4
:10D040003CB00B4040B00B4044B00B404CB00B40E8
:10D050002CB00B4058B00B405CB00B4060B00B40A4
:10D0600064B00B406CB00B4030B00B4030B429487A
:10D07000294A2A4B2A4D6024E121047011701B7843
:10D08000284C082B30D00A2B2748284937D00C2BA6
:10D090000CBF35223D2212232A60236002600B6000
:10D0A000234B24491B78244ABBB101230B60136036
:10D0B000224B23491B78234A012B26D9042B0FD955
:10D0C000082B1ED9102B94BF862387230B60136077
:10D0D0001D4B01221A7030BC70470B601360E7E7EC
:10D0E00084230B601360F3E700F58E200F490830AE
:10D0F000012213232A60236002600B60D0E73922EB
:10D10000F7E785230B601360E2E780230B60136071
:10D11000DEE700BF0040074001400740E091FF1FED
:10D1200008B003400CB0034008B00B400CB00B40FB
:10D13000B89FFF1F20B0034020B00B40E191FF1FBC
:10D1400024B0034024B00B40B59FFF1F0C2830B41F
:10D1500017D91023984228BF18461C46104A114D73
:10D160001178181A8C42287018D00F4913700B7858
:10D1700023B10E490E4A00230B60136030BCFFF749
:10D1800075BF0A2802D90C231C46E7E7082802D9F4
:10D190000A231C46E2E708231C46DFE730BC704741
:10D1A000E091FF1FB49FFF1FB59FFF1F24B00340F6
:10D1B00024B00B4028282FD8334B2DE9F0411E5CBA
:10D1C000FF2E2BD0314B1B78002B2AD132062CD4CA
:10D1D00072B62F4D2F4C2F46012326602B7062B65E
:10D1E00072B623681B060CD43B781BB9F4E72B7886
:10D1F000002BF1D062B602F09BF972B623681806D4
:10D20000F5D5254B1B6800222A7062B6234A107898
:10D2100043FA00F0BDE8F081002070470020BDE82F
:10D22000F081FFF781FE3206D2D572B61C4DDFF8D1
:10D230007C801C4C06F04007FFB206F03F06D8F891
:10D240000030DFB123F01003C8F80030012326605E
:10D25000134A2B7062B672B6236819060CD4137881
:10D260001BB9ECE72B78002BE9D062B602F060F92D
:10D2700072B623681B06F5D50B4BC3E743F01003CA
:10D28000C8F80030E2E700BF88430100B59FFF1FE8
:10D29000B79FFF1F00B0034010B00340B49FFF1FB3
:10D2A000B69FFF1F00B00B4010B00B400CB00B40FE
:10D2B0000A4A0B49136843F4805313600B7843B94F
:10D2C000084BC0221A70084B80F30C0000B2188083
:10D2D0007047044B80221A70F5E700BF2C80044091
:10D2E000B89FFF1F21C00C4000C00C40F0B51B4B85
:10D2F0001B4E596818689A68DB6885B06C460FC485
:10D30000337899071DD5174A174C1378174913F02E
:10D31000700318BF1370164A164B8027177000262B
:10D320003320032226706D4608701A7072B6043CD2
:10D3300045F001052046A84762B6237813F0700334
:10D3400009D10D4B064901E0013B02D00A78D20712
:10D35000FAD505B0F0BD237005B0F0BDB4430100AF
:10D360000100024000000240040002400B000240A5
:10D37000070002400A000240410D0300B0F5006FB3
:10D380000AD210B5094B1B78DB07044606D504F119
:10D39000A0500078C0B210BD00207047FFF7A6FF74
:10D3A00004F1A0500078C0B210BD00BF01000240DF
:10D3B000B0F5006F17D238B50F4B1B78DA070D4662
:10D3C000044611D504F1A0500378AB420AD00B4AB1
:10D3D000137813F0700318BF1370074A05701378A1
:10D3E000DB07FCD538BD7047FFF780FF04F1A05084
:10D3F0000378AB42EBD1F5E70100024000000240A8
:10D4000008B5F4F763FBF5F71DFA02F091F8FAE7B7
:10D41000844641EA000313F003036DD1403A41D33F
:10D4200051F8043B40F8043B51F8043B40F8043BFE
:10D4300051F8043B40F8043B51F8043B40F8043BEE
:10D4400051F8043B40F8043B51F8043B40F8043BDE
:10D4500051F8043B40F8043B51F8043B40F8043BCE
:10D4600051F8043B40F8043B51F8043B40F8043BBE
:10D4700051F8043B40F8043B51F8043B40F8043BAE
:10D4800051F8043B40F8043B51F8043B40F8043B9E
:10D4900051F8043B40F8043B51F8043B40F8043B8E
:10D4A000403ABDD2303211D351F8043B40F8043B2E
:10D4B00051F8043B40F8043B51F8043B40F8043B6E
:10D4C00051F8043B40F8043B103AEDD20C3205D33E
:10D4D00051F8043B40F8043B043AF9D2043208D036
:10D4E000D2071CBF11F8013B00F8013B01D30B88A8
:10D4F00003806046704700BF082A13D38B078DD086
:10D5000010F003038AD0C3F10403D21ADB071CBF57
:10D5100011F8013B00F8013B80D331F8023B20F8C1
:10D52000023B7BE7043AD9D3013A11F8013B00F8FA
:10D53000013BF9D20B7803704B7843708B78837082
:10D540006046704708B5104C08E0236859050DD4B3
:10D5500023681A050FD42368DB0411D42368580309
:10D56000F3D500F08DFE23685905F1D502F044F89B
:10D5700023681A05EFD502F0D5F82368DB04EDD552
:10D5800000F0F0FCEAE700BF3480044008B5FFF784
:10D59000D9FF00BF014B10221A80704700200540C0
:10D5A000704700BF094908B50B6830B16A46184496
:10D5B000A2F58052904202D20860184608BD03F0DE
:10D5C00065FB0C2303604FF0FF3008BDE491FF1FA3
:10D5D000FEE700BFEFF3138070B9EFF310836BB970
:10D5E000EFF305825AB94FF48070EFF311832BB13A
:10D5F000984228BF184670474FF0FF3070470F2AF7
:10D6000001D81846F1E7014BD05CEEE7F0E300E00B
:10D61000F0B44D1E2E46002400E00134B0FBF2F3BE
:10D6200002FB1300092800F130078ABF3730F8B237
:10D63000C0B206F8010F1846002BEED10A1953703C
:10D640004CB1107815F8016F28700133E01A83424D
:10D6500002F80169F5DB0846F0BC7047704700BF6F
:10D6600010B40F4B53F8302092F880422CB10123B4
:10D6700069B182F8803010BC704703EBC0035B686F
:10D680001A6841B922F002021A6010BC704782F891
:10D69000003110BC704742F003021A6010BC7047A2
:10D6A000C44301001C4A02EBC00301295B6811D08E
:10D6B00004291BD052F83000002280F8802229B1C2
:10D6C000022920D0032922D01A6070474FF48072BB
:10D6D0001A60704752F830004FF4A27280F880123E
:10D6E0001A601A6822F020021A60704752F830104F
:10D6F0004FF4A272012081F880021A601A6842F089
:10D7000020021A60704740F203121A6070474FF40B
:10D7100081721A60704700BFC4430100212848D8B5
:10D72000F8B5042A44D8DFE802F0484B4E03450020
:10D730004FF410262B4B03EBC0030D465C682168A9
:10D7400011F4E06148D0284B284A2949C3F89C21AC
:10D7500004F140422748C3F8A411A2F59221264FB4
:10D76000C3F8A0017C292548C3F8A871C3F8AC010F
:10D770002CD9A2F594237C2B2AD9A2F596237C2BB5
:10D7800028D9A2F598237C2B29D9A2F59A227C2AA4
:10D7900027D81B4872B6236823F4702343F08072A5
:10D7A000C4F384011643236040F82150266062B61A
:10D7B000F8BD70474FF43026BCE74FF40026B9E7B8
:10D7C0004FF44026B6E74FF42026B3E70D48E1E7D3
:10D7D0000D48DFE70D48DDE7FFF764FFB3E70C48CE
:10D7E000D8E7F8BDC44301000082FF1FF188FF1F86
:10D7F0009988FF1FC588FF1F6D88FF1F4188FF1F85
:10D80000C092FF1FE891FF1F2092FF1F7092FF1F21
:10D81000A092FF1F1A4B03EBC00010B4426802F144
:10D820004043A3F592217C2923D9A3F594217C2997
:10D830000DD9A3F596217C291FD9A3F598217C2920
:10D8400019D9A3F59A237C2B11D80E4C00E00E4C6D
:10D8500072B613680D4823F08773C2F3840123F472
:10D86000803343F08073136044F8210062B610BC2B
:10D870007047074CECE7074CEAE7074CE8E700BFC6
:10D88000C4430100C092FF1F2092FF1F5DD600001D
:10D89000E891FF1FA092FF1F7092FF1F30B4054B4D
:10D8A000054D064C002210211A602A602060196084
:10D8B00030BC704714D0034004D0034000D0034074
:10D8C000282838B52ED0002904464FDD5F4B1B7841
:10D8D000012505FA03F28A4202D8212837D938BD3A
:10D8E0000338C2B2012A3AD9202C4AD0192C48D088
:10D8F000574A126802FB011222FA03F31D2800F2B4
:10D900009B80DFE800F0928B847D9999766F9999DE
:10D910009999999999999968615A53994C999999B2
:10D9200099999945494B1B780B2B08D90C2B1CBF97
:10D930000C3B19410846BDE83840FFF7B9BCC3F1BC
:10D940000C0399400846BDE83840FFF7B1BC2946B2
:10D95000FFF786FE2946BDE83840FFF7A3BE3D4AE3
:10D96000126802FB011222FA03F3C7E72128B6D896
:10D970000021FFF775FE20460121BDE83840FFF782
:10D9800091BE354A126802FB011222FA03F3B5E791
:10D990003249334A0B604FF45173136038BD31493B
:10D9A000314A0B604FF45173136038BD2F49304A30
:10D9B0000B6040F24443136038BD2E492E4A0B6081
:10D9C00040F24443136038BD2C492D4A0B6040F2AD
:10D9D0004443136038BD2B492B4A0B6040F244434B
:10D9E000136038BD29492A4A0B6040F24443136052
:10D9F00038BD2849284A0B6040F24443136038BDC3
:10DA00002649274A0B6040F24443136038BD25493C
:10DA1000254A0B6040F24443136038BD2349244A31
:10DA20000B604FF45173136038BD2249224A0B60DA
:10DA30004FF45173136038BD212C3FF650AF7F294E
:10DA4000D4BF00210121204693E700BFC892FF1FE9
:10DA5000088003400890034008800B4010800B4072
:10DA600048A0044018800B404CA00440188003409C
:10DA700008B004401080034004B0044040800340DC
:10DA800018C004403880034014C00440288003407C
:10DA900010B00440208003400CB0044030800340AC
:10DAA00010C00440488003401CC00440189003404C
:10DAB00034900440109003403090044038B1102856
:10DAC00028BF1020044AC3B2107813707047024A6E
:10DAD0000123107813707047C892FF1F2DE9F84397
:10DAE0000E4680463249334D304603F055F847F62E
:10DAF000122300281ABF1D464FF002094FF00109FA
:10DB0000002425FA04F002F051FE4FF05E51074662
:10DB100002F0A4FE0146304603F052F830B9013459
:10DB2000072CEED1E80902F041FE0746314638469F
:10DB300002F048FF4FF07C5102F086FD03F07AF8C6
:10DB40004FF6FF729042A8F1030328BF1046012B45
:10DB500029D9B8F1170F17D8174B23FA08F303F098
:10DB6000010383F0010223B9B8F1190F0FD0BDE80A
:10DB7000F883124B124D13491A6044EAC9042A6013
:10DB800008601C60BDE8F883B8F1200FECD10E4BA3
:10DB90000E4D0F49002244EAC9041A602A60086049
:10DBA0001C60BDE8F8830B4B0B4D0C49F2E700BF3E
:10DBB000001BB740006CDC026006F00000800340F0
:10DBC000048003400880034000800B4004800B4029
:10DBD00008800B40009003400490034008900340ED
:10DBE000212801D8FFF73CBD704700BF212806D887
:10DBF000044B53F8303093F80002C0B27047002055
:10DC0000704700BFC4430100212801D8FFF74ABD77
:10DC1000704700BF72B60C490C4B0D4A1B68086870
:10DC2000126862B6520102D5322B88BF0130094911
:10DC3000C3F5BB334FF47A72FF33A1FB031302FB2E
:10DC400000F000EB93107047BC9FFF1F18E000E04E
:10DC500004ED00E0ABAAAAAA2DE9F843054672B686
:10DC6000204F214B214A1B683C68126862B6520162
:10DC700002D5322B88BF013495B3C3F5BB331C4E9C
:10DC8000DFF86490DFF86480FF334FF47A72A6FB0C
:10DC9000031302FB04F404EB931472B6D9F80010DA
:10DCA0003A68D8F800E062B6C1F5BB33FF33A6FB93
:10DCB00003031EF0806FC4EB93134FF47A7002D00D
:10DCC000322988BF013200FB0233B3F57A7F04D3D7
:10DCD000013D05D004F57A74DFE701F029FCDCE7AB
:10DCE000BDE8F883BC9FFF1F18E000E004ED00E0F2
:10DCF000ABAAAAAAF8B52D4B2D49DFF8D0E0DFF882
:10DD0000D0C02C4E2C4D2D4C2D4A2E4F4FF40000E0
:10DD100018604FF0807018604FF0007018604FF07E
:10DD2000806018604FF000601860002008602823B1
:10DD30004BF6FF71CCF80010CEF800303360136062
:10DD40002B6023603B60B3629362092245F8242C68
:10DD5000C4F8D80F05F57F65C7F8D41F07F5FF276E
:10DD600007F5FA67C6F8F83F2B6006F5FF26C4F8FA
:10DD7000D42F05F5FD2504F5FF24386006F2F4766E
:10DD80001148316005F5FF6504F5FD642B602360E3
:10DD90000260FFF76BF91920FFF75EFF00F0B6FF96
:10DDA00040F21310BDE8F840FFF756BF08E100E06D
:10DDB0000480034014800340248003402C800340EF
:10DDC0001C8003403480034000800B400C800340E3
:10DDD000088003402DE9F84F214B1B6807460BB123
:10DDE00001221A70DFF888901E4D99F80040DFF884
:10DDF00084801D4E0134272C8ABF4FF0000A5FFA41
:10DE000084FA5446AB462B78A34216D1FFF7E2FBC7
:10DE100040281FDC33791B06F5D59BF80030013311
:10DE2000272B86BF00221346DAB218F80330DBB284
:10DE3000F3712A702B78A342E8D00C490A4BFFB249
:10DE400008F804700120AC22087089F800A0DA708C
:10DE5000BDE8F88FFF28D6DD01F06AFBD3E700BFED
:10DE600034A0FF1F31A0FF1F00C0064030A0FF1FDD
:10DE700038A0FF1FC89FFF1F1C4BDFF894C01A6813
:10DE80001B49F0B542F480521A4D1A60DFF884E065
:10DE9000194F1A4E1A4C00238CF800304FF451726F
:10DEA0002B701F2840F213358EF800303B70337012
:10DEB00025600A6012D819460124124A124D1170C9
:10DEC0001248547000212C27402693724FF40034DE
:10DED00091701174D7702E700460F0BDC0F344319E
:10DEE000C0F3471400F01F03E7E700BF348004408D
:10DEF0000CC00440C59FFF1F31A0FF1F30A0FF1FB3
:10DF000008C0044000C0064031E400E004E100E045
:10DF1000C49FFF1F38A0FF1F034B1B68DB0401D504
:10DF2000FFF758BF704700BF3480044010B5044C61
:10DF3000237823B101F0FCFA2378002BFAD110BD2D
:10DF400030A0FF1F054A064B10781B78C0B2DBB229
:10DF5000984238BF4030C01A704700BFC49FFF1FAF
:10DF6000C59FFF1F30B42B4B1A7994061FD52A4842
:10DF7000DA790378294901333F2B0978C8BF002398
:10DF80008B42D2B203D0264CD9B2E2540170254A5A
:10DF9000116861B1244A1278D2B2934236BFC2F1FD
:10DFA00040029B1A9B18272BC4BF01230B70194AF0
:10DFB000D378DBB2180611D45A060DD5154B1B7950
:10DFC0005B0609D5194B1A491B6800220A7003B178
:10DFD0001A70104B2C22DA7030BC70471179090688
:10DFE000EAD5144910480C780178C9B28C420DD09A
:10DFF0004A1C272A84BF00210A460F4D054C98BFB2
:10E00000D1B2AA5CD2B2E2710170D5E76C21D170B5
:10E01000D2E700BF00C00640C49FFF1FC59FFF1F7F
:10E02000F09FFF1FC09FFF1F31A0FF1F34A0FF1FE5
:10E0300030A0FF1F38A0FF1FC89FFF1F21282FD827
:10E04000184B195CFF292BD0174B184ADFF870C00A
:10E0500003EBC000F0B54368DFF868E0144F154DDE
:10E06000154E00241C60DEF80030012043F0200330
:10E070008840CEF8003014604FF4A07338602E60F2
:10E08000C2F800C0013BFDD113689B05FCD42023DE
:10E09000013BFDD1094B09B233F8110080B2F0BD4C
:10E0A00000207047D4440100C443010000500440E4
:10E0B0000850044004500440000002030051044092
:10E0C00080014A0038800440431E032B14D872B6E6
:10E0D0000A4951F8230068B170B4094C058834F836
:10E0E0001320466841F82360521B24F8132062B6BF
:10E0F00070BC704762B670470020704794A0FF1F45
:10E10000D8A2FF1F013803280BD872B6074B53F86B
:10E11000203043B100205B680130002BFBD162B698
:10E120007047002070471846F9E700BFE8A0FF1FBE
:10E1300030B472B62B4A13781D0706D52A4B196ADC
:10E14000002936D0996A002941D053781C0706D59A
:10E15000254B196C00293ED0996C002939D0937851
:10E16000190705D5204B196E002936D0996E89B153
:10E17000D3781B0707D51C4BD3F880207AB3D3F88C
:10E18000882011213AB162B6184B00221A7030BCB7
:10E1900000F04ABE0D21154C154D227843F8315040
:10E1A00003EBC1030830013A5860227062B630BCFC
:10E1B000704704220D4C0F4D217843F8325003EB89
:10E1C000C20308304A1E5860227062B6EFE705218C
:10E1D000E1E70921DFE70822ECE70C22EAE7102259
:10E1E000E8E700BFF84401000080FF1F11A1FF1FF6
:10E1F000C800400088004000431E032B1DD81B4A66
:10E20000400140F0100030B4104472B6184CE25C8B
:10E21000032A1BD8DFE802F00212151703220D882B
:10E22000E25410F0080F14BFC823882343EA0543C3
:10E2300008310360416062B630BC7047083002228A
:10E24000EDE70522EBE708300422E8E7094A52F837
:10E25000230038B1084A52F82300416042F82310E5
:10E2600062B6E9E742F82310034AF7E70080FF1F90
:10E2700020A1FF1FE8A0FF1FF8A0FF1F00BE7047EE
:10E280002DE9F04FDFF818B3DFF818A387B044E0AA
:10E29000AD4F4FEA930807EBC809013ED9F80420B7
:10E2A00003F00803F6B2A2F1080003F0FF04002B0C
:10E2B00040F0018157F838301B0C99B222F8081C45
:10E2C000002B00F0EF80A14B22F8064C42F8044CE2
:10E2D00053F82620002A00F0CF819D4D55F82630B6
:10E2E00058609C4C45F8260034F81630194424F840
:10E2F000161000F079FD002800F0C281964A974B75
:10E3000019F0080F00F1080018BF1346C9F80400FF
:10E3100047F8383008238BF800309BF80040E4B20F
:10E3200065071CD58E4B1B78B3B18E490A7802F075
:10E33000FF0322B1013BDBB20B7003B900BE8A4977
:10E340000A7802F0FF032AB1013BDBB20B70002B0D
:10E3500000F0688100F066FE04238BF8003004F0C2
:10E36000080303F0FF02002B00F0C9809AF8003088
:10E37000DBB21E098CD19A08DFF8CC9159F8321023
:10E3800009EBC200C1F38301013940680C2900F296
:10E390008580DFE801F07A7A8383838383834683F1
:10E3A000838307000168714D4068714F714E68604A
:10E3B000296088B240F281610024674B49F832300D
:10E3C0004FF0010E88423C60C9F81040C9F818406F
:10E3D00086F800E05C4A00F2E780B0F5D06F80F08C
:10E3E0001B82B0F5817F00F0D98100F2698180281D
:10E3F00000F02A82822840F0D781A98801F07F01AD
:10E40000042900F2D1815C485C4A890008441470F8
:10E41000547001788C0740F1608382F800E002219B
:10E4200073E1534F3A682AB3554B524E55481988F9
:10E430003478057840298E4645F0020828BF4FF011
:10E44000400E002C84F001043470CEEB01010CBFAF
:10E450008824C82409EBC80689B285F0010544EA7E
:10E460000E447260198049F83840724405700029E2
:10E4700065D03A603D4B1A88B2F5A06F0ED10021ED
:10E480009A785970404B1A7008E038493F4C0D6833
:10E49000A54200F09880304949F832103C4A0123E7
:10E4A000137037E72C4A2D4B19F0080F18BF13468D
:10E4B00047F838302EE700F0B7FC364A364952F8B4
:10E4C0002630002B00F0E38058688C5D42F826006F
:10E4D00003F10802C9F80420032C05D8DFE804F092
:10E4E0002C02292602228A551A8819F0080F0CBF1F
:10E4F0008823C82343EA024347F838300AE7E00795
:10E5000000F19380210600F1D180A20706D5234AAD
:10E51000234913780220DBB213700870E30602D59A
:10E520001F4B10221A7007B0BDE8F08F04228A55E5
:10E53000DAE705228A55D7E703228A55D4E7BEF1E8
:10E54000400F18BF002294E70080FF1F94A0FF1F18
:10E5500040A0FF1FD8A2FF1FC80040008800400055
:10E560001CA1FF1FA5A0FF1F90A1FF1F08A1FF1F57
:10E570003CA0FF1FA4A0FF1FC020074014A1FF1F45
:10E5800050A0FF1F10A1FF1F982007402109000382
:10E5900094200740E8A0FF1F20A1FF1F882007400C
:10E5A0008020074090200740B0F5106F00F07C817C
:10E5B00040F2A38040F62112904240F07B82A54AAF
:10E5C000012313706AE74C68A3498C427FF463AF60
:10E5D0000178A9297FF45FAF417845297FF45BAFCB
:10E5E0008178C2297FF457AFC1786B297FF453AF8C
:10E5F0009A489B4E0178347881F00105002C41F057
:10E60000020105700CBF8820C82084F0010449F87D
:10E61000310009EBC10193483470002505244D6099
:10E62000047038E700F064FF94E68F4B89488B490B
:10E630001A614FF0020E80F800E08C4F0A708C498E
:10E64000196099608B4E8C4D8C4C9A610D213970FC
:10E65000FF213170DFF84CE229702270884D894A21
:10E660008EF800109F27012406F8047C5D6004707A
:10E67000DA6007B0BDE8F08F43F82600824D30E63F
:10E68000824A47F8380013780133137042E68B5DF5
:10E69000032B00F2BA8001A252F823F015E3000028
:10E6A00015E30000F5E60000EFE600006F49724B4D
:10E6B00080220D2008701A70A2077FF52FAF26E781
:10E6C00040F20232904240F0ED81AA8802F07F02CF
:10E6D000042A69D86D88002D66D16449CDF804E01C
:10E6E000920011440A7842F002020A70C1E101234B
:10E6F0008B550FE600238B550CE6B0F5086F53D110
:10E700006349644A097811707146ED888D4280F042
:10E71000E88252480478402DAE4644F0020C28BFEF
:10E720004FF0400E02EB0E0309EBCC0102930123E4
:10E730004A604FEA0E48CEEB050101930025C8223E
:10E7400042EA080384F0010249F83C303570027057
:10E75000DFF814C1424BDFF8048149BBBEF1400F22
:10E760007FF42DAF42F0020C09EBCC03029ADFF8E4
:10E77000F8E05A608DBB0D0445F088059DF8043023
:10E780004EF83C500A4433700470134640297FF41D
:10E7900016AF0021404A3B60118010E7AA8802F0C2
:10E7A0007F02042A40F28B81304A0F23137006E760
:10E7B0004029D7D942F002020CEBC200029E46600B
:10E7C000BDB19DF8045035481D703346403988F876
:10E7D000004040334CF83200DCE79DF804303370E1
:10E7E0000D04029B047045F0C8050B444EF83C50E4
:10E7F000CCE79DF804501D70029B1D4888F800402E
:10E80000403940334CF83200C4E719F0080F0CBF10
:10E81000022303238B557DE521494A68002AC3D092
:10E820006C88B5F804E003E00C314A68002ABBD0DC
:10E830000B88A342F8D14B887345F5D1240A032CE9
:10E840000CBF1178098960E7124A022114705470D4
:10E850005BE700BF942007400100040010A1FF1FE8
:10E86000A4A0FF1FA5A0FF1F0080FF1FC02007401E
:10E8700088004000882007408020074098200740FB
:10E8800054A0FF1FA8A0FF1F40A0FF1F11A1FF1F42
:10E890001CA1FF1F14A1FF1F50A0FF1FC8004000B4
:10E8A000FC4401008C200740B248116AAC78047027
:10E8B0000C0600F19881D9F82820AF49100600F124
:10E8C000DB81D9F83020AC49120600F1D081D9F8AB
:10E8D0003820A949130600F1C581D9F84020A6497E
:10E8E000150600F1BA81D9F84820A349140600F1B1
:10E8F000AF81D9F85020A049100600F1A481D9F8C1
:10E9000058209D49120600F19981D9F860209A4952
:10E91000130600F18E81D9F868209749150600F199
:10E920008381D9F870209449140600F17881D9F8D0
:10E9300078209149100600F16D81D9F880208E4928
:10E94000120600F16181D9F888208B49130600F185
:10E950005581D9F890208849150600F14981D9F8E8
:10E9600098208549140600F1FF808448844A85492F
:10E9700001908548854D864C0497002305960295A5
:10E9800080460F4616461D460394306828B14468F9
:10E9900000F04AFA2046002CF9D100233360029B94
:10E9A00038681A46002342F8253028B1446800F040
:10E9B0003BFA2046002CF9D100223A60019A98F8DF
:10E9C00000301146002241F8042B039A0191023BCA
:10E9D0004FF0000122F81510032B07D8DFE803F0F1
:10E9E0005D025D024FF0010388F800300135042D0F
:10E9F00006F1040607F1040708F10108C5D1654CCA
:10EA0000654D2278654B049F059E002110072970F3
:10EA10001A7000F19280624962780A700021C9F888
:10EA20003010C9F838101107DFF84C816ED4A27885
:10EA30005C49DFF844810A7000211207C9F85010C0
:10EA4000C9F858104BD4E27857494B4C0A70130759
:10EA50004FF00001C9F87010C9F8781000F1AE80CD
:10EA600033780193002283F00105C9F89020C9F89A
:10EA700098200021029188468E460A464B48047829
:10EA800044F0020C09EBCC030393019B002B039B86
:10EA90005A600CBF8822C82252E64FF0000388F863
:10EAA0000030A3E7B0F5A06F7FF47EAE0123002510
:10EAB0000193DEE740F621229042F7D074E66D889C
:10EAC000002D7FF471AE3A49CDF804E09200114474
:10EAD0000A7822F002020A70CBE7022115E600F064
:10EAE00083F9002800F0EB800830324AC8F864004F
:10EAF000C8F8602000F078F9002800F0DA800830CB
:10EB00002D4AC9F86C00C9F868209CE700F06CF940
:10EB1000002800F0E0800830264AC8F84400C8F811
:10EB2000402000F061F9002800F0CF800830224A30
:10EB3000C9F84C00C9F8482079E700F055F90028D9
:10EB400000F0A58008301B4AC9F82400C9F820202D
:10EB500000F04AF9002800F094800830164AC9F8FD
:10EB60002C00C9F8282056E7D1F89C00083800F09E
:10EB70005BF9FAE61CA1FF1F0080FF1FF8A0FF1F32
:10EB800094A0FF1FE8A0FF1F20A1FF1F40A0FF1FB0
:10EB9000D8A2FF1FF844010011A1FF1FC4200740A5
:10EBA000C8200740CC200740D020074010A1FF1FFD
:10EBB000C020074088004000C800400000F014F961
:10EBC000002870D008304F4AC4F88400C4F8802070
:10EBD00000F00AF9002860D008304B4AC9F88C00D0
:10EBE000C9F888203CE7506A083800F01DF962E651
:10EBF000D1F89400083800F017F9B0E6D1F88C008D
:10EC0000083800F011F9A4E6D1F88400083800F0C3
:10EC10000BF998E6C86F083800F006F98DE6486FE2
:10EC2000083800F001F982E6C86E083800F0FCF8F8
:10EC300077E6486E083800F0F7F86CE6C86D0838DB
:10EC400000F0F2F861E6486D083800F0EDF856E69D
:10EC5000C86C083800F0E8F84BE6486C083800F05B
:10EC6000E3F840E6C86B083800F0DEF835E6486B9C
:10EC7000083800F0D9F82AE6C86A083800F0D4F855
:10EC80001FE62A78C9F8280001322A70C3E62A78DC
:10EC9000C9F8200001322A705AE72A78C9F888009A
:10ECA00001322A70DCE62A78C4F8800001322A702A
:10ECB0008EE72A78C9F8680001322A70C3E62A78FC
:10ECC000C8F8600001322A7014E72A78C9F84800B1
:10ECD00001322A70ABE62A78C8F8400001322A7067
:10ECE0001FE740298E4628BF4FF0400E02EB0E036F
:10ECF00002930123CEEB01014FEA0E480025019358
:10ED0000BCE600BF88004000C8004000F8B500F035
:10ED10008FFD294B29482A4C2A4F2B4DDFF8BCC0C8
:10ED2000DFF8BCE0294E00221A605A609A60DA606F
:10ED30001A615A619A61DA611A625A629A62DA62F7
:10ED40001A635A639A63DA631A645A649A64DA64D7
:10ED50001A655A659A65DA651A665A669A66DA66B7
:10ED60001A675A679A67DA67C3F880200168C3F8A0
:10ED7000842041F480210160C3F307212170C3F393
:10ED80000740134938701B0E2B70FF238CF800309E
:10ED9000104D8EF8003010480B700123337084F84A
:10EDA000642070264FF40074102207F82C3C2E705B
:10EDB000046081F8F820F8BD0080FF1F3480044013
:10EDC0009C200740B0200740B42007409420074013
:10EDD0001020074049E400E008E100E080200740FF
:10EDE00088200740704700BF72B60D480268B2FA2B
:10EDF00082F30F2B10DC4FF00041D94022EA0102D0
:10EE0000026062B6074803EBC303DB00C2180021AF
:10EE1000C15010465160704762B60020704700BF75
:10EE2000CC92FF1FBC83FF1F0D4B0E4AC31AA2FBDF
:10EE300003231B090F2B0CD80B4A127852B972B658
:10EE40000A484FF00041026821FA03F31A430260B6
:10EE500062B67047064A1278002AF0D0FFF768B908
:10EE6000BC83FF1F398EE33811A1FF1FCC92FF1F17
:10EE70001CA1FF1F38B50E4B0E4C1B6821880546A0
:10EE80008BB1B1F5917F05D20B4A4B1C55549BB207
:10EE9000238038BD0022084898470021064A55546F
:10EEA0000123238038BDB1F5917FEDD338BD00BF7C
:10EEB00048A1FF1FE2A2FF1FE8A2FF1F2DE9F843B0
:10EEC000214E224F3168012380463B70B1B1204D65
:10EED0004B8801EB8302013300240F2BC2F808801A
:10EEE0002C7004D84B8000233B70BDE8F88340238E
:10EEF0000B800320FFF780F93460F4E7DFF85490CB
:10EF000099F80030002BF0D0114D45F6215408E05F
:10EF1000013C12D02B7883B900F00AFB99F800303D
:10EF20007BB10320FFF7EEF80528F1D8FFF75CFF6F
:10EF3000014630600028EBD0CAE701232B70BDE802
:10EF4000F883BDE8F88300BF64A1FF1F38A1FF1F4D
:10EF500068A1FF1F1CA1FF1F1201F8B5D5B2A1B314
:10EF6000012943D04378044600781B0643EA004059
:10EF700040F4704045F004068F1E3043FFF79EFFBB
:10EF8000022F04F1020314D9053414F8023C14F8DA
:10EF9000032C14F8010C1B0443EA0223334343EA15
:10EFA0000060033FFFF78AFF022F234604F10304AA
:10EFB000EBD8022F23D0012F0DD045F4774040F03D
:10EFC0000500BDE8F840FFF779BF14482843BDE8C5
:10EFD000F840FFF773BF187845F4770545F006054C
:10EFE00045EA0020BDE8F840FFF768BF03780C4809
:10EFF00045EA03452843BDE8F840FFF75FBF1A78AC
:10F00000587845F0774545F0070545EA022545EA79
:10F010000040BDE8F840FFF751BF00BF06F0F70021
:10F0200007F000F738B5084B1C7824B9074D29685C
:10F0300009B14B8803B938BD9B000B800320FFF753
:10F04000DBF82C6038BD00BF38A1FF1F64A1FF1F93
:10F050002DE9F041AD4E33680746002B00F0928059
:10F060001D885A88910803EB81010432AA428C68FA
:10F0700042D25A8004F00F064FEA1428A449A6F1A0
:10F08000080208F00F00C4F30313062A00F101057B
:10F090000B701AD9B31E012B5FFA88F04ED9052EDA
:10F0A00048D0042E00F0A481731F022B7FD90F2EAD
:10F0B0000ED1F72842D8F02802D0964B1B883BB1DE
:10F0C000FFF7D8FE0020BDE8F08127B1BD4202D095
:10F0D0000020BDE8F081082EC4F3033300F08780E0
:10F0E000092E11D00A2E40F094800A2BF0D18A4BC1
:10F0F0008A4A1B68A02181E01846FFF795FE04208C
:10F10000FEF7E2FF3060B5E7092BE1D1270E00F0F2
:10F110007B81834B814A1B689021C4F307461170A1
:10F12000EDB2FCB2002B00F09D802246314628460D
:10F13000984797E0F02843D9F72841D0F1380E28B6
:10F14000C6D801A353F820F0FFF20000E3F200005C
:10F15000D1F20000D1F00000D1F00000C3F20000B5
:10F16000D1F00000A3F30000D1F000006DF3000027
:10F1700087F30000ABF20000D1F0000093F2000032
:10F1800077F20000674B1B78002BA1D00420FEF71C
:10F190009BFF0346306000289AD00588002D7FF43D
:10F1A00060AFFFF741FE35602846BDE8F081FFF70C
:10F1B00061FEC4F30740FFF75DFE072E02D1200E6B
:10F1C000FFF758FE534B584A198858481468584D51
:10F1D000524A017000270E0AF0201F802E70107016
:10F1E0000CB301225348A0470120BDE8F081082B51
:10F1F0007FF46EAF504B494A1B688021C4F3074629
:10F200001170EDB2240E6BB3284622463146984762
:10F2100028E00B2E11D10B2B7FF45AAF474B3F4AFE
:10F220001B68B021EAE7464B1B68002B00F0FB800F
:10F23000404898470120BDE8F0810C2E40F0008145
:10F240000C2B7FF445AF3F4B344A1B68C021117033
:10F25000EDB2C4F30746002B00F0C88028463146C3
:10F26000240E98473849314A314B0D7016701C7086
:10F270000120BDE8F081354B1B68002B00F0D680E3
:10F280009847C4F30746254BEDB2240E83F800805F
:10F29000E8E72F4B1B68002BF2D12E4B1B68A3B164
:10F2A000FE209847C4F30746EDE72B4B1B68002B65
:10F2B000E6D1284B1B6843B1FC209847C4F30746AE
:10F2C000E1E7264B1B68002BDAD1C4F30746DAE7E7
:10F2D000234B1B68C4F30746002BD4D03046984715
:10F2E000D1E7204B1A68002AEFD0260C630C06F0F9
:10F2F0007F0003F47E531843F6B29047C3E71A4BDE
:10F300001B68C4F30746002BE8D1BCE770A1FF1FC0
:10F31000E6A2FF1FE2A2FF1F4CA1FF1FE0A2FF1FFA
:10F3200080A1FF1F1CA1FF1F48A1FF1FE4A2FF1F18
:10F33000E5A2FF1FE8A2FF1F78A1FF1F7CA1FF1F0E
:10F3400060A1FF1F3CA1FF1FE7A2FF1F28A1FF1F15
:10F350002CA1FF1F30A1FF1F6CA1FF1F5CA1FF1F8D
:10F3600074A1FF1F44A1FF1F58A1FF1F3F4B1B6843
:10F37000002B85D13E4B1B68002BA6D0FA20984766
:10F38000C4F307467FE73B4B1B68002B7FF478AF45
:10F39000374B1B68002B98D0FB209847C4F30746D7
:10F3A00071E7354B1B68002B7FF46AAF304B1B684D
:10F3B000002B8AD0F8209847C4F3074663E70E2B4A
:10F3C0007FF486AE2D4A2E4B1268E0211970002A78
:10F3D00047D0260C610C06F07F0301F47E511943DF
:10F3E000EDB2A1F5005128469047F6B2240E39E758
:10F3F000FFF740FDC4F30740FFF73CFD200EFFF789
:10F4000039FD0020BDE8F0811E4B1D4A1B6880219C
:10F410001170EDB2C4F3074683B1314628463A462F
:10F4200098473C461EE70120BDE8F081104B1B6861
:10F43000002B3FF44AAFFF20984746E71C4611E7F0
:10F440000D2EBCD10D2B7FF443AE0F4B0C4A1B6825
:10F45000D0211170EDB2C4F30746002B7FF4FEAE4D
:10F46000C4E7C4F30746EDB2240EFBE654A1FF1F28
:10F4700030A1FF1F34A1FF1F24A1FF1F40A1FF1FC8
:10F48000E0A2FF1F78A1FF1F50A1FF1F38B5164D46
:10F490002868E0B101884488A14213DD03191B7A72
:10F4A00083B104F10803C2180C1B002302E012F818
:10F4B000011F21B10133A342F9D1204638BD1C46BA
:10F4C000204638BDFFF7B0FC0020286038BD074B50
:10F4D0001B780BB9002038BD0220FEF7F5FD28602F
:10F4E0000028D7D1F6E700BF8CA1FF1F1CA1FF1F8A
:10F4F0000D4B1B78BBB910B50C4C216803F0FF0213
:10F500004B883F2B07DC07330B4401F1470003F81E
:10F51000012F8342FBD140230B800120FEF76CFEBC
:10F520000023236010BD704784A1FF1F88A1FF1F27
:10F5300038B5224C237803B138BD01232370FFF77F
:10F54000A5FF70BB00F048F840BB00F0DBF810BB33
:10F55000FEF7F8FCE0B900232370EFF30583002BDE
:10F56000EAD1EFF3108172B6154B1868E0B1154C73
:10F570002278CAB945691D6001232370C5B1AA610B
:10F5800001B962B600254577836898472570D3E7AF
:10F5900000F020F8DFE700F01BF8D9E700F016F8DC
:10F5A000D3E7FFF71FFCCDE70029C5D162B638BD10
:10F5B000054B1D600029E5D1E3E700BF91A1FF1FC6
:10F5C000A89FFF1FAC9FFF1FA49FFF1F704700BF96
:10F5D000704700BF704700BF054A064B10781B7884
:10F5E000C0B2DBB2984238BF4030C01A704700BF8B
:10F5F00098A1FF1F99A1FF1FF0B4384B1A7912F0A0
:10F60000300F2CD072B6997D01F0FF0200293DD059
:10F6100062B6334F334938780D78334E1C46C0B24A
:10F62000EDB2431C402BE17928BF0023AB4202F12D
:10F63000FF32C9B21CBFF154184612F0FF02F0D1DC
:10F640002A4B1B68C2B23A704BB1A84236BFC5F113
:10F650004005401B40192728C4BF01221A701F49CA
:10F66000CA78D2B2150616D452060DD51B4B1B799B
:10F670005B0609D51E4B1F491B6800220A7003B1A7
:10F680001A70164B3C22DA70F0BC70474022D979D0
:10F690005A7462B6E3E70B791C06E5D5164B174E94
:10F6A0001C783378E4B2DBB29C420ED0144D01E0FA
:10F6B000A3420AD00133402B28BF00230879E85C1D
:10F6C000C0B2C871087D0728F2D9DBB20349337094
:10F6D0000B79180644BF7C23CB70C5E700A0064019
:10F6E00098A1FF1F99A1FF1FDCA1FF1F94A1FF1F7D
:10F6F00020A2FF1F1CA2FF1F24A2FF1F1DA2FF1F8D
:10F700009CA1FF1F054A064B10781B78C0B2DBB2E4
:10F71000984238BF4030C01A704700BF98A2FF1F00
:10F720002DA2FF1FF0B4384B1A7912F0300F2CD0F5
:10F7300072B6997D01F0FF0200293DD062B6334FC9
:10F74000334938780D78334E1C46C0B2EDB2431CB5
:10F75000402BE17928BF0023AB4202F1FF32C9B24E
:10F760001CBFF154184612F0FF02F0D12A4B1B685F
:10F77000C2B23A704BB1A84236BFC5F14005401B3A
:10F7800040192728C4BF01221A701F49CA78D2B273
:10F79000150616D452060DD51B4B1B795B0609D5F1
:10F7A0001E4B1F491B6800220A7003B11A70164BCA
:10F7B0003C22DA70F0BC70474022D9795A7462B6A4
:10F7C000E3E70B791C06E5D5164B174E1C7833780A
:10F7D000E4B2DBB29C420ED0144D01E0A3420AD049
:10F7E0000133282B28BF00230879E85CC0B2C87118
:10F7F000087D0728F2D9DBB2034933700B7918066C
:10F8000044BF7C23CB70C5E700B0064098A2FF1F21
:10F810002DA2FF1F58A2FF1F28A2FF1F9CA2FF1F9F
:10F820002CA2FF1FA0A2FF1F99A2FF1F30A2FF1F43
:10F8300070B584B072B6194B194D1A487022412622
:10F840000F2480211A702E701A46047019701378D4
:10F850001B06FCD5144B186862B6144B144C984226
:10F8600098BF00EB800001A998BF40000A22FDF775
:10F87000CFFE01A92046002311F8012B01333AB134
:10F880000A2B20F8022FF7D11623237004B070BD85
:10F890005B00DBB2237004B070BD00BF000002400B
:10F8A0000700024006000240080002407F969800D0
:10F8B0009893FF1FFFFFFFFF2DE9F043DFF8EC8077
:10F8C0008BB006460F4600F073F898F9003001330C
:10F8D00004460D4637D03046394600F0DFF900289F
:10F8E00031D02BA3D3E900233046394600F026FE61
:10F8F000814668BB28A3D3E900233046394600F08F
:10F90000FFFD00B398F90030254ACDF8209004247B
:10F9100000200021022BCDE90467CDE902670094A5
:10F920000192CDE906012CD0684600F0BDF940B344
:10F93000089B1BB101F0AAF9089B0360DDE90601F1
:10F940000BB0BDE8F083204629460BB0BDE8F0833C
:10F95000134A98F90030019203210022CDE904678F
:10F96000CDE90267009108922BB90E4B4FF060422F
:10F97000CDE90623D8E70C490020022BCDE906018A
:10F98000D2D101F083F922230360D1E7AFF30080E5
:10F99000EF39FAFE422E864051302DD5104987C0EE
:10F9A00068450100FFFFEF470000F07FAE93FF1FA7
:10F9B0002DE9F04FB04F21F00042BA4283B00C461F
:10F9C0004FEAD17605460DD9AC4FBA4225D9C1F3DD
:10F9D0001303034340F0EF800EB10020014603B053
:10F9E000BDE8F08FA64B9A4200F2CC80A54B9A421C
:10F9F00000F2DE808AA3D3E9002300F05DF9002243
:10FA0000A14B00F09BFD002800F00581284621460F
:10FA100000229D4B00F050F9E1E783A3D3E90023D6
:10FA200000F08CFD002840F0CB802846214680A3C2
:10FA3000D3E9002300F064FD0028CED1934B284683
:10FA400003EBC60821467CA3D3E9002300F0E6FAC5
:10FA5000D8E9002300F030F900F07AFD804600F08C
:10FA600077FA77A3D3E9002306460F4600F0D6FACB
:10FA700002460B462846214600F01CF972A3D3E942
:10FA80000023CDE900013046394600F0C7FA82462E
:10FA90008B4652465B46DDE9000100F00BF9054656
:10FAA0000C462A4623462846214600F0B7FA68A3AA
:10FAB000D3E9002306460F4600F0B0FA66A3D3E967
:10FAC000002300F0F7F832463B4600F0A7FA64A3A3
:10FAD000D3E9002300F0F0F832463B4600F09EFAEE
:10FAE00061A3D3E9002300F0E5F832463B4600F07D
:10FAF00095FA5FA3D3E9002300F0DEF832463B46D7
:10FB000000F08CFA02460B462846214600F0D2F857
:10FB100006460F462846214632463B46B8F1000FBE
:10FB200056D000F07BFA324604460D463B46002094
:10FB30004FF0804100F0BEF802460B4620462946B1
:10FB400000F096FB02460B465046594600F0B2F8CC
:10FB5000DDE9002300F0AEF80B4602464A490020DA
:10FB600000F0A8F86FF47F7398454FDA08F57A78BB
:10FB700001EB085100224FF0B87300F04FFA03B0C8
:10FB8000BDE8F08F424B9A423FF658AF414BF4002C
:10FB90002344D3E9002300F08DF83F4BC6F1010860
:10FBA0001C44CDE90001D4E900ABC6EB080870E7BE
:10FBB0004FF0000875E702460B4600F07DF80EE7AF
:10FBC00017A3D3E900231046194600F027FA06E7E9
:10FBD00000F024FA0022804689464FF080433046E8
:10FBE000394600F067F802460B464046494600F0A9
:10FBF0003FFB2A46234600F05DF802460B460020F4
:10FC0000214900F057F803B0BDE8F08F01EB08512F
:10FC100003B0BDE8F08F804643E700BFAFF300803C
:10FC20009C7500883CE4377EEF39FAFE422E864010
:10FC300051302DD5104987C0FE822B654715F73FFF
:10FC40000000E0FE422EE63F763C7935EF39EA3D92
:10FC5000D0A4BE726937663EF16BD2C541BDBB3ED2
:10FC60002CDE25AF6A56113F93BDBE166CC1663FB0
:10FC70003E5555555555C53F412E8640FFFFEF7FF8
:10FC8000422ED63FFFFF2F3E0000F03F704501009F
:10FC9000B1A2F03F904501008045010041F00041D4
:10FCA00001F58010C00F70470020704781F00041BF
:10FCB00002E000BF83F0004330B54FEA41044FEA51
:10FCC000430594EA050F08BF90EA020F1FBF54EAEC
:10FCD000000C55EA020C7FEA645C7FEA655C00F088
:10FCE000E2804FEA5454D4EB5555B8BF6D420CDD59
:10FCF0002C4480EA020281EA030382EA000083EADC
:10FD0000010180EA020281EA0303362D88BF30BD7B
:10FD100011F0004F4FEA01314FF4801C4CEA1131D1
:10FD200002D0404261EB410113F0004F4FEA033330
:10FD30004CEA133302D0524263EB430394EA050FBB
:10FD400000F0A780A4F10104D5F1200E0DDB02FA2A
:10FD50000EFC22FA05F2801841F1000103FA0EF2BE
:10FD6000801843FA05F359410EE0A5F120050EF184
:10FD7000200E012A03FA0EFC28BF4CF0020C43FAB5
:10FD800005F3C01851EBE37101F0004507D54FF0C2
:10FD9000000EDCF1000C7EEB00006EEB0101B1F512
:10FDA000801F1BD3B1F5001F0CD349085FEA300058
:10FDB0004FEA3C0C04F101044FEA445212F5800F63
:10FDC00080F09A80BCF1004F08BF5FEA500C50F100
:10FDD000000041EB045141EA050130BD5FEA4C0CE3
:10FDE000404141EB010111F4801FA4F10104E9D16C
:10FDF00091F0000F04BF01460020B1FA81F308BF63
:10FE00002033A3F10B03B3F120020CDA0C3208DD2E
:10FE100002F1140CC2F10C0201FA0CF021FA02F109
:10FE20000CE002F11402D8BFC2F1200C01FA02F179
:10FE300020FA0CFCDCBF41EA0C019040E41AA2BF9E
:10FE400001EB0451294330BD6FEA04041F3C1CDA66
:10FE50000C340EDC04F11404C4F1200220FA04F086
:10FE600001FA02F340EA030021FA04F345EA030130
:10FE700030BDC4F10C04C4F1200220FA02F001FAF2
:10FE800004F340EA0300294630BD21FA04F0294674
:10FE900030BD94F0000F83F4801306BF81F480110D
:10FEA0000134013D4EE77FEA645C18BF7FEA655C80
:10FEB00029D094EA050F08BF90EA020F05D054EA52
:10FEC000000C04BF1946104630BD91EA030F1EBF57
:10FED0000021002030BD5FEA545C05D1400049415B
:10FEE00028BF41F0004130BD14F580043CBF01F54E
:10FEF000801130BD01F0004545F0FE4141F4700134
:10FF00004FF0000030BD7FEA645C1ABF194610460E
:10FF10007FEA655C1CBF0B46024650EA013406BF0F
:10FF200052EA033591EA030F41F4002130BD00BFCE
:10FF300090F0000F04BF0021704730B54FF480648B
:10FF400004F132044FF000054FF0000150E700BF0C
:10FF500090F0000F04BF0021704730B54FF480646B
:10FF600004F1320410F0004548BF40424FF0000158
:10FF70003EE700BF42004FEAE2014FEA31014FEA9B
:10FF800002701FBF12F07F4393F07F4F81F06051EA
:10FF9000704792F0000F14BF93F07F4F704730B559
:10FFA0004FF4607401F0004521F0004120E700BFEC
:10FFB00050EA010208BF704730B54FF000050AE073
:10FFC00050EA010208BF704730B511F0004502D574
:10FFD000404261EB41014FF4806404F132045FEA76
:10FFE000915C3FF4DCAE4FF003025FEADC0C18BF1B
:10FFF00003325FEADC0C18BF033202EBDC02C2F111
:020000021000EC
:10000000200300FA03FC20FA02F001FA03FE40EAA2
:100010000E0021FA02F11444C1E600BF70B54FF0A2
:10002000FF0C4CF4E06C1CEA11541DBF1CEA135584
:1000300094EA0C0F95EA0C0F00F0DEF82C4481EAEC
:10004000030621EA4C5123EA4C5350EA013518BF0C
:1000500052EA033541F4801143F4801338D0A0FBF9
:1000600002CE4FF00005E1FB02E506F00042E0FBA6
:1000700003E54FF00006E1FB03569CF0000F18BFAC
:100080004EF0010EA4F1FF04B6F5007F64F5407454
:1000900004D25FEA4E0E6D4146EB060642EAC621E7
:1000A00041EA55514FEAC52040EA5E504FEACE2E54
:1000B000B4F1FD0C88BFBCF5E06F1ED8BEF1004F57
:1000C00008BF5FEA500E50F1000041EB045170BDD3
:1000D00006F0004646EA010140EA020081EA030117
:1000E000B4EB5C04C2BFD4EB0C0541EA045170BD13
:1000F00041F480114FF0000E013C00F3AB8014F18D
:10010000360FDEBF002001F0004170BDC4F10004D5
:10011000203C35DA0C341BDC04F11404C4F1200556
:1001200000FA05F320FA04F001FA05F240EA0200B1
:1001300001F0004221F0004110EBD37021FA04F6E7
:1001400042EB06015EEA430E08BF20EAD37070BDA1
:10015000C4F10C04C4F1200500FA04F320FA05F000
:1001600001FA04F240EA020001F0004110EBD37002
:1001700041F100015EEA430E08BF20EAD37070BD72
:10018000C4F1200500FA05F24EEA020E20FA04F34B
:1001900001FA05F243EA020321FA04F001F00041FA
:1001A00021FA04F220EA020000EBD3705EEA430E6B
:1001B00008BF20EAD37070BD94F0000F0FD101F09A
:1001C0000046400041EB010111F4801F08BF013CD3
:1001D000F7D041EA060195F0000F18BF704703F011
:1001E0000046520043EB030313F4801F08BF013D98
:1001F000F7D043EA0603704794EA0C0F0CEA135554
:1002000018BF95EA0C0F0CD050EA410618BF52EA0D
:100210004306D1D181EA030101F000414FF0000013
:1002200070BD50EA410606BF1046194652EA430621
:1002300019D094EA0C0F02D150EA013613D195EA95
:100240000C0F05D152EA03361CBF104619460AD1DD
:1002500081EA030101F0004141F0FE4141F47001E7
:100260004FF0000070BD41F0FE4141F4780170BDD7
:1002700070B54FF0FF0C4CF4E06C1CEA11541DBF3C
:100280001CEA135594EA0C0F95EA0C0F00F0A7F83E
:10029000A4EB050481EA030E52EA03354FEA01316B
:1002A00000F088804FEA03334FF0805545EA13137E
:1002B00043EA12634FEA022245EA111545EA106546
:1002C0004FEA00260EF000419D4208BF964244F1DD
:1002D000FD0404F5407402D25B084FEA3202B61AFC
:1002E00065EB03055B084FEA32024FF480104FF4D0
:1002F000002CB6EB020E75EB030E22BFB61A754644
:1003000040EA0C005B084FEA3202B6EB020E75EBD6
:10031000030E22BFB61A754640EA5C005B084FEA3E
:100320003202B6EB020E75EB030E22BFB61A75460B
:1003300040EA9C005B084FEA3202B6EB020E75EB16
:10034000030E22BFB61A754640EADC0055EA060ED7
:1003500018D04FEA051545EA16754FEA06164FEA1A
:10036000C30343EA52734FEAC2025FEA1C1CC0D1C6
:1003700011F4801F0BD141EA00014FF000004FF053
:10038000004CB6E711F4801F04BF01430020B4F114
:10039000FD0C88BFBCF5E06F3FF6AFAEB5EB030CCC
:1003A00004BFB6EB020C5FEA500C50F1000041EBC9
:1003B000045170BD0EF0004E4EEA113114EB5C0496
:1003C000C2BFD4EB0C0541EA045170BD41F4801169
:1003D0004FF0000E013C90E645EA060E8DE60CEA71
:1003E000135594EA0C0F08BF95EA0C0F3FF43BAF8E
:1003F00094EA0C0F0AD150EA01347FF434AF95EA45
:100400000C0F7FF425AF104619462CE795EA0C0F28
:1004100006D152EA03353FF4FDAE1046194622E7F5
:1004200050EA410618BF52EA43067FF4C5AE50EACF
:1004300041047FF40DAF52EA43057FF4EBAE12E7BF
:100440004FF0FF3C06E000BF4FF0010C02E000BFA0
:100450004FF0010C4DF804CD4FEA410C7FEA6C5C83
:100460004FEA430C18BF7FEA6C5C1BD001B050EA26
:10047000410C0CBF52EA430C91EA030F02BF90EA11
:10048000020F0020704710F1000F91EA030F58BFD0
:10049000994208BF90422CBFD8176FEAE37040F032
:1004A000010070474FEA410C7FEA6C5C02D150EAD0
:1004B000013C07D14FEA430C7FEA6C5CD6D152EA8B
:1004C000033CD3D05DF8040B704700BF8446104650
:1004D00062468C461946634600E000BF01B5FFF74F
:1004E000B7FF002848BF10F1000F01BD4DF808ED1F
:1004F000FFF7F4FF0CBF012000205DF808FB00BFF0
:100500004DF808EDFFF7EAFF34BF012000205DF849
:1005100008FB00BF4DF808EDFFF7E0FF94BF012096
:1005200000205DF808FB00BF4DF808EDFFF7CEFF97
:1005300094BF012000205DF808FB00BF4DF808EDD6
:10054000FFF7C4FF34BF012000205DF808FB00BFA7
:100550004FEA410212F5001215D211D56FF47873EB
:10056000B3EB625212D94FEAC12343F0004343EA8E
:10057000505311F0004F23FA02F018BF4042704769
:100580004FF00000704750EA013005D111F00040F3
:1005900008BF6FF0004070474FF00000704700BF89
:1005A0004FEA4102B2F1E04324BFB3F5001CDCF195
:1005B000FE5C0DD901F0004C4FEAC0024CEA5070CD
:1005C000B2F1004F40EB830008BF20F001007047FC
:1005D00011F0804F21D113F13872BCBF01F00040FF
:1005E000704741F480114FEA5252C2F11802C2F131
:1005F000200C10FA0CF320FA02F018BF40F00100B2
:100600004FEAC1234FEAD32303FA0CFC40EA0C0063
:1006100023FA02F34FEA4303CCE77FEA625307D1A0
:1006200050EA01331EBF4FF0FE4040F440007047D7
:1006300001F0004040F0FE4040F40000704700BF71
:1006400080F0004002E000BF81F0004142001FBF87
:100650005FEA410392EA030F7FEA226C7FEA236C90
:100660006AD04FEA1262D2EB1363C1BFD218414085
:1006700048404140B8BF5B42192B88BF704710F01B
:10068000004F40F4000020F07F4018BF404211F0BE
:10069000004F41F4000121F07F4118BF494292EA26
:1006A000030F3FD0A2F1010241FA03FC10EB0C0052
:1006B000C3F1200301FA03F100F0004302D54942DF
:1006C00060EB4000B0F5000F13D3B0F1807F06D38C
:1006D00040084FEA310102F10102FE2A51D2B1F184
:1006E000004F40EBC25008BF20F0010040EA030079
:1006F0007047490040EB000010F4000FA2F1010226
:10070000EDD1B0FA80FCACF1080CB2EB0C0200FAAF
:100710000CF0AABF00EBC25052421843BCBFD040FD
:100720001843704792F0000F81F4000106BF80F477
:1007300000000132013BB5E74FEA41037FEA226C3A
:1007400018BF7FEA236C21D092EA030F04D092F005
:10075000000F08BF0846704790EA010F1CBF002039
:10076000704712F07F4F04D1400028BF40F0004096
:10077000704712F100723CBF00F50000704700F0B6
:10078000004343F0FE4040F4000070477FEA2262DD
:1007900016BF08467FEA23630146420206BF5FEAAE
:1007A000412390EA010F40F4800070474FF00003AE
:1007B00004E000BF10F0004348BF40425FEA000C75
:1007C00008BF704743F0964301464FF000001CE01D
:1007D00050EA010208BF70474FF000030AE000BF73
:1007E00050EA010208BF704711F0004302D54042B1
:1007F00061EB41015FEA010C02BF84460146002023
:1008000043F0B64308BFA3F18053A3F50003BCFA3D
:100810008CF2083AA3EBC25310DB01FA02FC6344EA
:1008200000FA02FCC2F12002BCF1004F20FA02F2F1
:1008300043EB020008BF20F00100704702F12002E4
:1008400001FA02FCC2F1200250EA4C0021FA02F245
:1008500043EB020008BF20EADC7070474FF0FF0C4A
:100860001CEAD0521EBF1CEAD15392EA0C0F93EA45
:100870000C0F6FD01A4480EA010C400218BF5FEAE7
:1008800041211ED04FF0006343EA501043EA51115A
:10089000A0FB01310CF00040B1F5000F3EBF490054
:1008A00041EAD3715B0040EA010062F17F02FD2A58
:1008B0001DD8B3F1004F40EBC25008BF20F001003B
:1008C000704790F0000F0CF0004C08BF49024CEA52
:1008D000502040EA51207F3AC2BFD2F1FF0340EAE4
:1008E000C250704740F400004FF00003013A5DDC55
:1008F00012F1190FDCBF00F000407047C2F1000296
:10090000410021FA02F1C2F1200200FA02FC5FEA82
:10091000310040F1000053EA4C0308BF20EADC70CC
:10092000704792F0000F00F0004C02BF400010F43E
:10093000000F013AF9D040EA0C0093F0000F01F0EB
:10094000004C02BF490011F4000F013BF9D041EA0D
:100950000C018FE70CEAD15392EA0C0F18BF93EA0F
:100960000C0F0AD030F0004C18BF31F0004CD8D139
:1009700080EA010000F00040704790F0000F17BFC0
:1009800090F0004F084691F0000F91F0004F14D006
:1009900092EA0C0F01D142020FD193EA0C0F03D15E
:1009A0004B0218BF084608D180EA010000F0004061
:1009B00040F0FE4040F40000704740F0FE4040F43C
:1009C000400070474FF0FF0C1CEAD0521EBF1CEADB
:1009D000D15392EA0C0F93EA0C0F69D0A2EB0302F9
:1009E00080EA010C49024FEA402037D04FF0805393
:1009F00043EA111143EA10130CF000408B4238BF58
:100A00005B0042F17D024FF4000C8B4224BF5B1A65
:100A100040EA0C00B3EB510F24BFA3EB510340EAB3
:100A20005C00B3EB910F24BFA3EB910340EA9C0061
:100A3000B3EBD10F24BFA3EBD10340EADC001B01D1
:100A400018BF5FEA1C1CE0D1FD2A3FF650AF8B4275
:100A500040EBC25008BF20F0010070470CF0004C82
:100A60004CEA50207F32C2BFD2F1FF0340EAC250AD
:100A7000704740F400004FF00003013A37E792F06E
:100A8000000F00F0004C02BF400010F4000F013ACC
:100A9000F9D040EA0C0093F0000F01F0004C02BFC7
:100AA000490011F4000F013BF9D041EA0C0195E730
:100AB0000CEAD15392EA0C0F08D142027FF47DAFC9
:100AC00093EA0C0F7FF470AF084676E793EA0C0FB9
:100AD00004D14B023FF44CAF08466EE730F0004CB7
:100AE00018BF31F0004CCAD130F000427FF45CAF47
:100AF00031F000437FF43CAF5FE700BF4FF0FF3CB5
:100B000006E000BF4FF0010C02E000BF4FF0010C07
:100B10004DF804CD4FEA40024FEA41037FEA226CD0
:100B200018BF7FEA236C11D001B052EA530C18BFF2
:100B300090EA010F58BFB2EB030088BFC81738BF57
:100B40006FEAE17018BF40F0010070477FEA226C45
:100B500002D15FEA402C05D17FEA236CE4D15FEA41
:100B6000412CE1D05DF8040B704700BF8446084675
:100B70006146FFE70FB5FFF7C9FF002848BF10F136
:100B8000000F0FBD4DF808EDFFF7F4FF0CBF01207B
:100B900000205DF808FB00BF4DF808EDFFF7EAFF05
:100BA00034BF012000205DF808FB00BF4DF808EDC0
:100BB000FFF7E0FF94BF012000205DF808FB00BFB5
:100BC0004DF808EDFFF7D2FF94BF012000205DF83B
:100BD00008FB00BF4DF808EDFFF7C8FF34BF012048
:100BE00000205DF808FB00BF4FEA4002B2F1FE4F63
:100BF0000FD34FF09E03B3EB12620DD94FEA0023DF
:100C000043F0004310F0004F23FA02F018BF4042B7
:100C100070474FF00000704712F1610F01D142029E
:100C200005D110F0004008BF6FF0004070474FF052
:100C30000000704742000ED2B2F1FE4F0BD34FF0CE
:100C40009E03B3EB126209D44FEA002343F0004342
:100C500023FA02F070474FF00000704712F1610F65
:100C600001D1420202D14FF0FF3070474FF0000037
:100C7000704700BF0B460146184600F001B800BFA0
:100C800013460A460146022000F0ACBE014B18682C
:100C9000704700BFD897FF1F70B50F4E0F4D761BE2
:100CA000B61018BF002405D0013455F8043B98470E
:100CB000A642F9D10A4E0B4D761B03F073FCB61019
:100CC00018BF002406D0013455F8043B9847A642CB
:100CD000F9D170BD70BD00BFB0450100B045010045
:100CE000C4450100B0450100024B0146186800F000
:100CF0000BB800BFD897FF1F024B0146186800F0E1
:100D000035BF00BFD897FF1F2DE9F04F01F10B054C
:100D1000162D83B0064640F29F8035F0070500F19E
:100D2000BF80A94200F2BC8000F058FBB5F5FC7F03
:100D3000C0F09C826B0A00F0BA80042B00F2838121
:100D4000A80900F1390E4FEA4E033830C44F07EBC3
:100D50008303A3F108015C68A14207D1ACE0002A3B
:100D600080F2AC80E468A14200F0A680636823F0C2
:100D700003035A1B0F2AF2DDB9493C6901F1080E41
:100D8000744500F0B381636823F003035A1B0F2AF4
:100D900000F39981002AC1F814E0C1F810E080F254
:100DA0009E80B3F5007F80F06781DB0803F1010CC2
:100DB00001229B1002FA03F34A6851F83C80C4F800
:100DC000088001EBCC091A43A9F10803E3604A60EB
:100DD00041F83C40C8F80C40831001249C409442E8
:100DE00000F28A80144206D120F00300640014420D
:100DF00000F10400FAD007EBC009CC468046DCF8CD
:100E00000C108C4507D173E1002A80F28181C968FA
:100E10008C4500F06D814B6823F003035A1B0F2AA9
:100E2000F2DD0C46D1F80CC054F8088F4B1945F090
:100E300001054D6042F00101C8F80CC03046CCF805
:100E400008807B613B61C3F80CE0C3F808E059609F
:100E50009A5000F0C5FA1FE0102921D800F0BEFA20
:100E60001025062302207E4F07EB8303A3F108021F
:100E70005C68944200F045816368E168A56823F0EE
:100E80000303234430465A68E96042F001028D6052
:100E90005A6000F0A5FA0834204603B0BDE8F08F90
:100EA00000240C232046336003B0BDE8F08F80237C
:100EB0004FF0400E3F2049E770465DE72344E1686C
:100EC0005A68A56842F00102E96030468D605A60B8
:100ED00000F086FA0834204603B0BDE8F08F2344C2
:100EE00030465A6842F001025A6000F079FA08343C
:100EF000204603B0BDE8F08FBC68636823F00308A8
:100F0000A84504D3C5EB08030F2B00F38C80554B89
:100F1000DFF860911A68D9F8003001332A4404EBF5
:100F2000080A00F0608102F580520F3222F47F62DD
:100F300022F00F0211463046019200F04BFCB0F156
:100F4000FF3F8346019A00F05881824500F2FC8001
:100F5000454B1968DA451144196000F05381D9F8FE
:100F60000000DFF810E101301BBFCAEB0B0A51444F
:100F7000CEF800B019601BF0070100F01781C1F135
:100F80000800C1F58051834408315A44C2F30B0272
:100F9000C2EB010949463046019300F01BFC431C9B
:100FA000019B00F03F81CBEB00024A4442F001027A
:100FB0001968C7F808B04944BC42CBF8042019604E
:100FC000DFF8A49016D0B8F10F0F40F2FD806268F0
:100FD000A8F10C0323F00703E01802F001024FF020
:100FE000050E1A430F2B6260C0F804E0C0F808E059
:100FF00000F21C811D4BBC681A68914288BF1960C1
:101000001B4B1A689142626888BF196022F0030284
:101010009542A2EB050301D80F2B04DC304600F00B
:10102000DFF9002438E7621943F0010345F00105B8
:1010300065603046BA60536000F0D2F9083420464B
:1010400003B0BDE8F08F142B71D9542B00F2A480AB
:10105000280B00F16F0E4FEA4E036E3076E600BFAC
:10106000DC97FF1FACA2FF1FB0A2FF1FA8A2FF1FAB
:10107000A4A2FF1FE89BFF1F5A0A042A5ED9142A64
:1010800000F2B38002F15C0149005B3207EB810C96
:1010900057F82110DFF8DC81ACF1080C8C4500F02A
:1010A00088804A6822F00302934202D289688C4504
:1010B000F7D1D1F80CC07A68C4F80CC0A160CCF8A4
:1010C0000840CC6088E6631942F0010745F001054D
:1010D000656030464B610B61C3F80CE0C3F808E073
:1010E0005F609A50083400F07BF9D5E64A6873E6F1
:1010F00008F1010818F0030F0CF1080C7FF47FAE23
:1011000030E0DC68A34208BF02303FF435AEB3E6FE
:101110000B440C465A68C96854F8085F42F0010253
:101120005A603046E9608D6000F05AF9B4E603F188
:101130005C0E03F15B004FEA4E0307E69A0902F1E9
:10114000390149003832A1E7BC424A4B3FF400AFB5
:101150009C68626822F003025AE759F808399945F9
:1011600040F0828010F0030F00F1FF30F5D17B6872
:1011700023EA04037B6064009C423FF6BDAE002C72
:101180003FF4BAAE1C4240467FF435AE64001C42C8
:1011900000F10400FAD02EE6B3F5AA7F18D8E80BC8
:1011A00000F1780E4FEA4E037730CFE54FF48051CF
:1011B000EBE60121D8F80430921001FA02F21A434A
:1011C000C8F80420614677E70123CBF8043025E70F
:1011D00040F25452934220D8A80C00F17D0E4FEA01
:1011E0004E037C30B2E51032A4E6542A26D81A0BFE
:1011F00002F16F0149006E3248E7BC68626822F074
:10120000030205E7CAF30B0000287FF4A8AE4244AE
:10121000BB6842F001025A60ECE6FE234FF07F0EFD
:101220007E2093E501224FF00009C1E604F1080198
:10123000304600F09BFCD9F80010DBE6B2F5AA7F3F
:1012400005D8DA0B02F17801490077321EE740F247
:1012500054518A4205D89A0C02F17D0149007C3232
:1012600014E7FE217E2211E77B6884E7E808431C2F
:101270005B00F8E5DC97FF1F8842F0B50DD98B18AD
:1012800098420AD28118002A51D09A1A13F8014DB7
:1012900001F8014D9342F9D1F0BD0F2A48D941EA36
:1012A00000039B0746D100F1100401F1100315461D
:1012B00053F8106C44F8106C53F80C6C44F80C6C38
:1012C00053F8086C44F8086C103D53F8046C44F86B
:1012D000046C0F2D03F1100304F11004E8D8A2F1FF
:1012E000100323F00F0302F00F0E1033BEF1030FB3
:1012F0001944034421D91E1F0D467446043C55F879
:10130000047B46F8047F032CF8D8AEF1040424F0E3
:10131000030404342344214402F0030262B1013B7C
:101320000A4411F8014B03F8014F8A42F9D1F0BD8C
:101330000346F3E70346F2E7F0BD7246EEE700BF6F
:1013400070B4840746D0541E002A41D0CDB2034663
:1013500002E0621EE4B3144603F8015B9A07F8D179
:10136000032C2ED9CDB245EA05250F2C45EA0545BB
:1013700019D903F110022646103E0F2E42F8105CD8
:1013800042F80C5C42F8085C42F8045C02F110027E
:10139000F2D8A4F1100222F00F0204F00F04103270
:1013A000032C13440DD91E462246043A032A46F85C
:1013B000045BFAD8221F22F003020432134404F023
:1013C00003042CB1C9B21C4403F8011BA342FBD196
:1013D00070BC704714460346C2E700BF704700BFA9
:1013E000704700BF024B0A460146186800F002B879
:1013F000D897FF1F2DE9F04F174683B0002900F062
:10140000C1800E46814607F10B05FFF7E7FF56F84E
:1014100004EC162D2EF00304A6F1080840D8102283
:101420001546AF4241D8944275DAC94B996808EB2A
:1014300004008842416800F0D98021F00103034490
:101440005B68DB077DD51EF0010F35D03946484675
:10145000FFF75AFC0746E0B156F8043C23F00103BD
:101460004344A0F108029A4200F04481221F242A3A
:1014700000F23181132A00F20481034632461168DA
:1014800019605168596092689A603146484600F088
:101490006DFB4846FFF7A4FF384603B0BDE8F08F68
:1014A00025F00705002D2A46BBDA0C230020C9F8D9
:1014B000003003B0BDE8F08F56F8083CC3EB080AD3
:1014C000DAF8043023F0030C04EB0C039342BDDB89
:1014D0005746DAF80C1057F8080F221F242AC1606B
:1014E000886000F21781132A40F212813168CAF82D
:1014F00008107168CAF80C101B2A00F22B810836FC
:101500000AF110023168116071685160B168916030
:101510003E461C46D046631B0F2B1DD8D8F804301E
:1015200003F0010323434444C8F80430636843F0E4
:10153000010363604846FFF753FF304603B0BDE840
:10154000F08F21F003012144914221DBC3688268BE
:101550000C46D3609A60DEE7D8F8042008EB05015A
:1015600002F00102154343F001020B44C8F8045095
:101570004A605A6842F0010208315A60484600F059
:10158000F5FAD7E7114603B0BDE8F04FFFF7BCBB53
:101590001EF0010F7FF45AAF56F8083CC3EB080A5F
:1015A000DAF8043023F0030C01EB0C0E96458BDBCC
:1015B000C36882685746D3609A6057F8081FDAF804
:1015C0000C30CB60221F242A996000F29980132AE4
:1015D00062D93368CAF808307368CAF80C301B2A1D
:1015E00000F2A08008360AF1100356E021F0030B48
:1015F000A34405F11000834559DA1EF0010F7FF472
:1016000025AF56F8081CC1EB080ADAF8041021F0DF
:10161000030CE34458453FF757AF5746DAF80C1030
:1016200057F8080F221F242AC160886000F2B48096
:10163000132A40F2A5803168CAF808107168CAF808
:101640000C101B2A00F2AF8008360AF11002316834
:10165000116071685160B16891600AEB0501C5EBDA
:101660000B0242F0010299604A60DAF8043003F09C
:1016700001031D434846CAF80450FFF7B1FE38463F
:101680005CE733680360736843601B2A27D800F166
:10169000080306F10802F2E63B4632681A607268F7
:1016A0005A60B2689A603E467446D04633E708EB0B
:1016B0000501C5EB0B0B4BF0010299604A6056F82F
:1016C000043C03F001031D43484646F8045CFFF761
:1016D00087FE304632E73146FFF7CEFDD5E6B368E8
:1016E0008360F368C360242A28D000F1100306F158
:1016F0001002C4E650F8043C23F003031C440AE73C
:10170000314638467446D046FFF7B6FD3E4602E7FE
:101710003A46F7E6314638461C46D046FFF7ACFD60
:101720003E46F8E6B368CAF81030F368CAF81430D9
:10173000242A1BD010360AF11803AEE7336903617F
:101740007369436106F1180200F1180397E600BFC0
:10175000DC97FF1FB168CAF81010F168CAF81410BE
:10176000242A0FD010360AF11802CBE63369CAF8E2
:1017700018307369CAF81C3018360AF120038CE758
:101780003A4664E73269CAF818207269CAF81C2020
:1017900018360AF12002B5E6314638460193FFF7C4
:1017A0006BFD019B59E7B168CAF81010F168CAF8DF
:1017B0001410242A03D010360AF1180247E73269C0
:1017C000CAF818207269CAF81C2018360AF12002DB
:1017D0003DE700BF38B5074C0023054608462360A7
:1017E000FBF7E0FE431C00D038BD2368002BFBD084
:1017F0002B6038BD0CA4FF1FFFFFFFFFFFFFFFFFA3
:1018000090F800F06DE9024520F007016FF0000C40
:1018100010F0070491F820F040F049804FF00004E8
:101820006FF00700D1E9002391F840F000F10800C3
:1018300082FA4CF2A4FA8CF283FA4CF3A2FA8CF3FB
:101840004BBBD1E9022382FA4CF200F10800A4FA62
:101850008CF283FA4CF3A2FA8CF3E3B9D1E90423B6
:1018600082FA4CF200F10800A4FA8CF283FA4CF3ED
:10187000A2FA8CF37BB9D1E9062301F1200182FAA7
:101880004CF200F10800A4FA8CF283FA4CF3A2FAAD
:101890008CF3002BC6D0002A04BF04301A4612BABB
:1018A000B2FA82F2FDE8024500EBD2007047D1E9BE
:1018B000002304F00305C4F100004FEAC50514F04D
:1018C000040F91F840F00CFA05F562EA05021CBF1E
:1018D00063EA050362464FF00004A9E7002A41D0FD
:1018E00040EA010313F00303F0B425D1032A23D9FE
:1018F00004680D68AC421FD1043A35D0A4F101351B
:1019000025EA040414F0803F31D1071D0D1D0DE0C0
:1019100057F8043B0E68A3F10134B34224EA0304F0
:101920000AD1043A20D014F0803F23D1032A29465B
:10193000384605F10405EBD803780C789C4202F197
:10194000FF320CD182B114B916E06AB17BB110F844
:10195000013F11F8014FA34202F1FF32F5D0181BED
:10196000F0BC7047104670471046F0BC70471846F0
:10197000F0BC70470020F3E72046F1E740EA01039E
:101980009B0770B42BD1032A29D90C460346214664
:1019900054F8046BA6F1013525EA060515F0803FE1
:1019A00006D1043A032A43F8046B2146EFD8A2B1CA
:1019B0000C781C70013A013301313CB16AB111F865
:1019C000014B03F8014B013A002CF7D12AB11A441C
:1019D000002103F8011B9A42FBD170BC70470346FB
:1019E000E5E700BF2DE9F047254C2568D5F84841CB
:1019F0000646884692469946C4B360681F2817DC9D
:101A0000431C76B104EB80050122C5F888A0D4F808
:101A1000881182401143022EC4F88811C5F808913C
:101A20001ED00230636044F820800020BDE8F087BB
:101A3000144B03B34FF4C870FFF756F90446D0B106
:101A4000D5F84831002780E88800C5F84841384675
:101A50000123C4F88871C4F88C71002EE1D0D1E75D
:101A6000D4F88C110A43C4F88C21DAE705F5A67482
:101A7000C5F84841C1E74FF0FF30BDE8F08700BF2F
:101A8000A0450100E90C0100024B13B1024800F02F
:101A900005B8704700000000A91A010000230146A4
:101AA0001A461846FFF79EBF38B5074D074C2C1B4A
:101AB000A41005D0013C55F8043D9847002CF9D1FD
:101AC000BDE8384002F07EBD0000000000000000CC
:101AD000F8B5234F0C460646FFF780FCBB685D68EF
:101AE00025F00305291B01F6EF7121F47F6121F038
:101AF0000F01A1F58054B4F5805F07DB002130466B
:101B0000FFF768FEBB682B44984204D03046FFF7CD
:101B100067FC0020F8BD61423046FFF75BFE0130F4
:101B20000DD0104BBA6819682D1B45F001053046E1
:101B3000091B55601960FFF753FC0120F8BD002117
:101B40003046FFF747FEBA68831A0F2BDEDD064CDE
:101B50000449246843F00103001B53600860D5E783
:101B6000DC97FF1FB0A2FF1FE89BFF1F002945D095
:101B70002DE9F0410D468046FFF730FC55F8047C16
:101B80006A4927F00103A5F10804E2188E6850683D
:101B9000B24220F0030062D0FE0750600BD455F82B
:101BA000087CE41B01F1080EA56875453B446FD025
:101BB000E768EF60BD6015186D68ED0742D543F02A
:101BC00001026260E350B3F5007F18D2DB085A1CB3
:101BD0004D6851F83270A76001209B1000FA03F3A2
:101BE00001EBC2001D430838E0604D6041F832400F
:101BF000FC604046BDE8F041FFF7F2BB70475A0A6F
:101C0000042A53D89A0902F139077F0002F13805F6
